:100000000C94F8130C9422140C9422140C942214C3
:100010000C9422140C9422140C9422140C94221488
:100020000C9422140C9422140C9422140C94221478
:100030000C9422140C94EE730C9422140C9422143D
:100040000C9422140C94A8710C9423C20C942214C6
:100050000C94123B0C94083B0C9422140C94221424
:100060000C9422140C9422140C9422140C94221438
:100070000C9422140C9422140C9422140C94221428
:100080000C9422140C9422140C9422144E414E49C8
:100090004E495459494E46CDCCCC3D0AD7233C1746
:1000A000B7D13877CC2B329595E6241FB14F0A0093
:1000B0000020410000C84200401C4620BCBE4CCA83
:1000C0001B0E5AAEC59D7400407A10F35A00A07200
:1000D0004E18090010A5D4E80000E8764817000083
:1000E000E40B54020000CA9A3B000000E1F5050051
:1000F0000080969800000040420F000000A086019A
:10010000000000102700000000E803000000006469
:1001100000000000000A00000000000100000000D4
:10012000002C76D888DC674F0823DFC1DFAE59E1A9
:10013000B1B796E5E3E453C63AE651997696E8E618
:10014000C28426EB898C9B62ED407C6FFCEFBC9CEB
:100150009F40F2BAA56FA5F490055A2AF75C936BFD
:100160006CF9676DC11BFCE0E40D47FEF520E6B5B8
:1001700000D0ED902E0300943577050080841E0892
:100180000000204E0A000000C80C333333330F98B0
:100190006E12831141EF8D2114893BE65516CFFE77
:1001A000E6DB18D1844B381BF77C1D901DA4BBE403
:1001B00024203284725E228100C9F124ECA1E53D45
:1001C00027434F4D4D554E49434154494F4E0044EE
:1001D000525952554E004552524F525300494E46C5
:1001E0004F004543484F00486F74656E6420496472
:1001F0006C652054696D656F757400486F74656E29
:10020000642049646C652054696D656F75740A00DB
:100210002121204B494C4C20636175736564206239
:100220007920746F6F206D75636820696E616374E7
:100230006976652074696D65202D2063757272651D
:100240006E7420636F6D6D616E643A200053544F7D
:10025000505045442E20005072696E7465722073B0
:10026000746F707065642064756520746F206572AA
:10027000726F72732E2046697820746865206572EB
:10028000726F7220616E6420757365204D39393943
:1002900020746F20726573746172742E2028546507
:1002A0006D70657261747572652069732072657313
:1002B00065742E20536574206974206166746572BC
:1002C0002072657374617274696E67290A004E6FDB
:1002D00020436865636B73756D2077697468206C63
:1002E000696E65206E756D6265722C204C61737449
:1002F000204C696E653A20004E6F20436865636B41
:1003000073756D2077697468206C696E65206E75F1
:100310006D6265722C204C617374204C696E653A75
:100320002000636865636B73756D206D69736D6123
:100330007463682C204C617374204C696E653A209C
:10034000004C696E65204E756D6265722069732080
:100350006E6F74204C617374204C696E65204E750D
:100360006D6265722B312C204C617374204C696E68
:10037000653A20004D3131300053657269616C205F
:10038000737461747573206D69736D617463680A49
:100390000053442072656164206572726F720A00B6
:1003A0004D6564696120496E7365727465640050BF
:1003B0006C65617365205265736574005052494ED7
:1003C0005445522048414C5445440025533A202579
:1003D0005300706F7765726F6666004B494C4C45F1
:1003E000442E20005072696E7465722068616C74CE
:1003F00065642E206B696C6C28292063616C6C65C8
:1004000064210A006563686F3A004572726F723A40
:10041000000A4D6561737572656420706F696E7452
:10042000733A0A00357835206D6573682E205A209E
:100430006F66667365743A2000206E6F7420656E77
:1004400074657265642E0A0050726F62696E67206F
:10045000506F696E740025532025692F256900208F
:100460006F6620004D424C2047323920706F696E14
:10047000742000290A004A206F7574206F6620726C
:10048000616E67652028302D00290A0049206F75AC
:1004900074206F662072616E67652028302D0047DA
:1004A00032384C30004D6573682070726F62696E2F
:1004B0006720646F6E65004D6573682070726F62AF
:1004C000696E6720646F6E652E0A005374617274E2
:1004D000206D6573682070726F62696E672077693E
:1004E00074682022473239205331222066697273A2
:1004F000742E0A004732395332004732384C300AE2
:10050000473239533200686173206E6F2064617422
:10051000612E0A004D65736820426564204C657643
:10052000656C696E67200053206F7574206F6620BC
:1005300072616E67652028302D35292E0A0020490A
:100540006E76616C6964206578747275646572207A
:1005500000536C6565702E2E2E004D6573682070FB
:100560006F696E74206F7574206F662072616E679C
:10057000650A00436C69636B20746F205265737564
:100580006D652E2E2E004E6F204D6F76652E004528
:100590006E642066696C65206C6973740A0042653C
:1005A00067696E2066696C65206C6973740A004E19
:1005B0006F206D656469610A00706175736500285C
:1005C0006E6F2066696C65290043757272656E7482
:1005D0002066696C653A20005344207072696E741D
:1005E000696E67206279746520004E6F74205344F1
:1005F000207072696E74696E670A002E0A00446585
:100600006C6574696F6E206661696C65642C204648
:10061000696C653A200046696C652064656C657498
:1006200065643A002569730025696D2025697300AA
:100630002569682025696D20256973002569642076
:100640002569682025696D20256973002569792051
:10065000256964202569682025696D202569730056
:100660005072696E742074696D653A20006F6B007A
:100670006F666600E201DD01D601CF01C10144458C
:100680004255473A0020573A0042656420436F6F55
:100690006C696E672E2E2E00426564204865617479
:1006A000696E672E2E2E00544D334420456E6465CE
:1006B0007233204F46462E004649524D574152450F
:1006C0005F4E414D453A4D61726C696E20322E305D
:1006D0002E375F4457372E3320544D334420453353
:1006E000454D444E4E202841707220323420323025
:1006F00032312031373A33353A32392920534F5588
:100700005243455F434F44455F55524C3A687474B9
:1007100070733A2F2F6769746875622E636F6D2F3F
:10072000496E73616E6974794175746F6D61746936
:100730006F6E2F4D61726C696E2F747265652F43F9
:100740007265616C6974794477696E5F322E30200E
:1007500050524F544F434F4C5F56455253494F4EA2
:100760003A312E30204D414348494E455F5459504F
:10077000453A544D334420456E64657233204558E4
:100780005452554445525F434F554E543A312055CB
:100790005549443A63656465326132662D3431618E
:1007A000322D343734382D396231322D633535638B
:1007B00036326633363766660A002F2F004D3134E5
:1007C0003520533C696E6465783E206F7574206FE8
:1007D000662072616E67652028302D31290A00205D
:1007E0005200416363656C65726174696F6E3A2093
:1007F00050005741524E494E4721204C6F77205AA6
:10080000204A65726B206D6179206C65616420748B
:100810006F20756E77616E746564207061757365A5
:10082000732E0A004D32303620580020204D61785A
:100830003A2000200020204D696E3A2000536F6658
:100840007420656E6473746F70733A200046523A78
:100850000020466C6F773A20004D424C2041646A7C
:10086000757374205A0020643A0020693A002070A1
:100870003A00496E76616C696420657874727564BB
:1008800065720A0064697300656E0043290A00619D
:10089000626C656420286D696E2074656D7020003F
:1008A000436F6C642065787472756465732061723F
:1008B0006520004F4646004F4E00426564204C655F
:1008C00076656C696E6720004661696C65642074AA
:1008D0006F20656E61626C6520426564204C6576B0
:1008E000656C696E670A004D657368204265642017
:1008F0004C6576656C20646174613A0A00496E76D5
:10090000616C6964206D6573682E0A004D657368BB
:1009100020706F696E74206F7574206F662072612D
:100920006E67650A004D34323120696E636F7272F2
:1009300065637420706172616D6574657220757392
:100940006167650A004F6666736574732041707055
:100950006C696564004572723A20546F6F2066615D
:10096000722100546F6F206661722066726F6D2075
:100970007265666572656E636520706F696E740A74
:1009800000454550524F4D204F4B0A004D38340022
:10099000446F6E65207072696E74696E6720666957
:1009A0006C650A004D3737004D333100496E766172
:1009B0006C69642065787472756465720A002057EA
:1009C0003A00436F6F6C696E672E2E2E004865618A
:1009D00074696E672E2E2E00452025530023646512
:1009E00066696E652044454641554C545F004B6432
:1009F00020004B6920004B70200050494420417575
:100A0000746F74756E652066696E697368656421BC
:100A10002050757420746865206C617374204B706D
:100A20002C204B6920616E64204B6420636F6E73D1
:100A300074616E74732066726F6D2062656C6F777F
:100A400020696E746F20436F6E666967757261749A
:100A5000696F6E2E680A00504944204175746F74A6
:100A6000756E65206661696C6564212074696D65C9
:100A70006F75740A00504944204175746F74756E27
:100A800065206661696C6564212054656D706572CE
:100A9000617475726520746F6F20686967680A00F9
:100AA000204B643A2000204B693A2000204B703ADA
:100AB000200020436C617373696320504944200A0D
:100AC000002054753A2000204B753A2000206D61BB
:100AD000783A2000206D696E3A200020643A2000A8
:100AE00020626961733A2000504944204175746F57
:100AF00074756E652073746172740A0050494420E5
:100B00004175746F74756E65206661696C656421EA
:100B10002054656D706572617475726520746F6FB5
:100B200020686967680A00504944204175746F74F1
:100B3000756E65206661696C656421204261642080
:100B40006865617465722069640A005049442041F7
:100B500075746F74756E65004572723A20757466AF
:100B60003820666F6E74206E6F7420696E697469C8
:100B7000616C697A65642E004572723A20757466FC
:100B80003820666F6E74206E6F7420696E697469A8
:100B9000616C697A65642E004572723A20757466DC
:100BA0003820666F6E74206E6F7420696E69746988
:100BB000616C697A65642E0042656400456E636C01
:100BC0006F73757265002568753A25303268750057
:100BD00025303268753A2530326875002020202093
:100BE0002020200020202020003FFFF0380070301F
:100BF000FC3020FC102078102030102C00D02E313A
:100C0000D02F7BD02F7BD02E31D02C00D020301095
:100C100020781020FC1030FC303800703FFFF03F8F
:100C2000FFF03800703186302387102787902F8798
:100C3000D02F03D0203010207810207810203010D2
:100C40002F03D02F87D02787902387103186303805
:100C500000703FFFF004104002082002082004103A
:100C600040082080104100104100082080041040FE
:100C70000000001FFFF81FFFF863616E63656C00E2
:100C80005072696E742041626F72746564004D32F7
:100C9000350050617573696E672E2E2E0072657374
:100CA000756D65004D32340046696C2E20446961D3
:100CB0002E004F6666004F6E004520696E206D6DF8
:100CC0005E33005654726176204D696E00566D6930
:100CD0006E00566D6178204500566D6178205A008F
:100CE000566D6178205900566D6178205800416D2D
:100CF0006178204500416D6178205A00416D61782E
:100D0000205900416D6178205800412D5472617660
:100D1000656C00412D5265747261637400416363B8
:100D2000656C0056652D4A65726B00565A2D4A65F2
:100D3000726B0056592D4A65726B0056582D4A65E4
:100D4000726B00452073746570732F6D6D005A20AF
:100D500053746570732F6D6D0059205374657073F3
:100D60002F6D6D00582053746570732F6D6D0041A9
:100D70006476616E6365642053657474696E67732D
:100D8000003F0043616E63656C00496E6974004DFD
:100D900034323800496E697469616C697A6520453E
:100DA0004550524F4D0046696C616D656E7400533D
:100DB000746570732F6D6D004A65726B00416363DB
:100DC000656C65726174696F6E0056656C6F6369FE
:100DD00074790053657420486F6D65204F666673A3
:100DE00065747300436F6E66696775726174696FCD
:100DF0006E004C6576656C696E6720446F6E652188
:100E0000004D6F7665205A00473239533200000C8E
:100E10000F00FE07022503BB017FFE08FE08FE054A
:100E2000080806000040F0C888889878100508086F
:100E3000060000C0F88888888888F805050506003F
:100E4000012030F830200508080600002070F82046
:100E5000202020E00509090600FF2070A8A8B88816
:100E6000887020070505070001D86C366CD8050985
:100E7000090600FFF8A88888888888A8F8050A0A63
:100E80000600FE205050505088A8A8887003030325
:100E900006000340A040FFFFFFFFFFFFFFFFFFFF33
:100EA000FFFFFFFFFFFFFFFFFFFFFFFF0000000648
:100EB00005FF010707060200808080808000800314
:100EC0000303060105A0A0A005060606000050F8D1
:100ED0005050F8500509090600FF2070A8A070289E
:100EE000A87020050707060000C8C8102040989881
:100EF00005070706000040A0A040A8906801030372
:100F00000602058080800309090601FF2040408019
:100F100080804040200309090601FF8040402020D6
:100F20002040408005070706000020A8702070A818
:100F3000200505050600012020F8202002030306F5
:100F400001FFC04080050101060003F8020202060D
:100F50000100C0C00507070600000810102040402F
:100F600080050707060000708898A8C888700307E6
:100F70000706010040C040404040E005070706006A
:100F800000708808102040F8050707060000F808E0
:100F9000103008887005070706000010305090F8E0
:100FA0001010050707060000F880F0080888700593
:100FB0000707060000304080F088887005070706A4
:100FC0000000F80810102020200507070600007018
:100FD0008888708888700507070600007088887800
:100FE000081060020505060100C0C000C0C002066E
:100FF000060601FFC0C000C04080030505060101D0
:101000002040804020050303060002F800F8030595
:10101000050601018040204080050707060000709A
:101020008810202000200507070600007088B8A857
:10103000B88070050707060000708888F8888888DF
:10104000050707060000F04848704848F005070704
:101050000600007088808080887005070706000001
:10106000F04848484848F0050707060000F8808027
:10107000F08080F8050707060000F88080F0808087
:101080008005070706000070888080988870050733
:1010900007060000888888F8888888030707060103
:1010A00000E04040404040E00507070600003810DF
:1010B00010101090600507070600008890A0C0A0DF
:1010C0009088050707060000808080808080F805F2
:1010D000070706000088D8A88888888805070706BB
:1010E00000008888C8A8988888050707060000704F
:1010F000888888888870050707060000F08888F0CF
:1011000080808005070706000070888888A890689E
:10111000050707060000F08888F0A09088050707FB
:1011200006000070888070088870050707060000B8
:10113000F820202020202005070706000088888846
:1011400088888870050707060000888888885050BE
:101150002005070706000088888888A8A85005078A
:101160000706000088885020508888050707060079
:101170000088885020202020050707060000F80876
:1011800010204080F80309090601FFE0808080807C
:10119000808080E005070706000080404020101096
:1011A000080309090601FFE020202020202020E07C
:1011B0000503030600052050880501010600FEF81E
:1011C00003030306010580402005050506000070A5
:1011D000087888780507070600008080F0888888EE
:1011E000F005050506000070808088700507070679
:1011F00000000808788888887805050506000070D2
:1012000088F08070050707060000304840E0404045
:10121000400507070600FE70888888780870050773
:10122000070600008080F088888888030707060189
:10123000004000C0404040E00409090601FE1000E3
:10124000301010101090600507070600008080889D
:1012500090E09088030707060100C04040404040EE
:10126000E0050505060000D0A8A8A8A80505050604
:101270000000B0C8888888050505060000708888C9
:1012800088700507070600FEF0888888F0808005D2
:1012900007070600FE78888888780808050505068F
:1012A0000000B0C8808080050505060000788070C9
:1012B00008F00507070600002020F8202020180568
:1012C0000505060000888888986805050506000061
:1012D00088888850200505050600008888A8A85041
:1012E0000505050600008850205088050707060000
:1012F000FE88888850204080050505060000F8100B
:101300002040F80309090601FF204040408040408A
:1013100040200109090602FF808080808080808053
:10132000800309090601FF80404040204040408082
:1013300005030306000248A890FF41425300504CA9
:1013400041004E65787420506F696E7400256920E5
:101350002F20257500473239533100473239533237
:1013600000436C69636B20746F20426567696E008F
:10137000486F6D696E672058595A0053746F7265D3
:101380002053657474696E6773004C6F61642053F9
:10139000657474696E677300426564205A004F6615
:1013A00066004F6E00426564204C6576656C696E20
:1013B00067004C6576656C20426564004D6F74690A
:1013C0006F6E00426564004E6F7A7A6C650046610C
:1013D0006E20537065656400436F6E666967757251
:1013E0006174696F6E00526573746F726520446535
:1013F0006661756C7473004C6F616420536574741E
:10140000696E67730053746F7265205365747469F5
:101410006E67730050726568656174202420436FA5
:101420006E6600416476616E636564205365747412
:10143000696E6773004D61696E003F004261636BC6
:101440000053746F70004D3231005072696E742019
:1014500066726F6D204D656469610052656C6561EF
:101460007365204D65646961004D323200436F6ED3
:1014700066696775726174696F6E0054656D706539
:10148000726174757265004D6F74696F6E0052659C
:1014900073756D65205072696E7400417474616378
:1014A00068204D656469610054756E650053746F02
:1014B00070205072696E74005061757365205072AF
:1014C000696E7400496E666F2053637265656E00C5
:1014D00043616E6E6F7420656E7465722073756201
:1014E0006469723A2000022E2E0001526566726510
:1014F0007368004D61696E002100486F74656E6409
:1015000020746F6F20636F6C64004261636B0050E6
:10151000726F63656564004D6F74696F6E00446936
:101520007361626C65205374657070657273004DF1
:10153000383400426564204C6576656C696E6700DE
:101540004175746F20486F6D6500473238004D61FA
:10155000696E0050726568656174202420456E6470
:1015600000507265686561742024204265640054EF
:10157000656D7065726174757265003E133A134350
:101580006F6F6C646F776E00507265686561742070
:10159000240046616E2053706565640042656400F6
:1015A0004E6F7A7A6C65004D61696E0042616279B6
:1015B00073746570205A00466C6F770046616E2028
:1015C000537065656400426564004E6F7A7A6C659D
:1015D00000426564205A005370656564004D61697E
:1015E0006E00486F6D696E67204661696C656400C6
:1015F0006F70656E00545249474745524544003A62
:1016000020007A5F6D696E00795F6D696E00785FAA
:101610006D696E005265706F7274696E6720656ED9
:101620006473746F70207374617475730A0020742E
:101630006F6F206C6F6E6720657874727573696F59
:101640006E2070726576656E7465640A0020636F43
:101650006C6420657874727573696F6E2070726542
:1016600076656E7465640A000000000000000000EA
:10167000000000005761726E696E673A20486F6D16
:10168000696E672042756D702044697669736F7268
:10169000203C20310A0002020400007A4300007A54
:1016A0004300007A430000004100000041000000B8
:1016B0004000007A4300007A4300007A43000000B3
:1016C00000000000000000000053657474696E673C
:1016D000732053746F72656400454550524F4D201E
:1016E000496E697469616C697A65640A003B20001F
:1016F00020440020490020204D333031205000503C
:1017000049442073657474696E67733A002046001B
:1017100020420020480020204D3134352053004D18
:101720006174657269616C206865617475702070A0
:101730006172616D65746572733A002020473239B9
:10174000205334205A00204A0020204732392053A9
:101750003320490020204D3432302053004D657332
:101760006820426564204C6576656C696E673A0056
:1017700020204D323036205800486F6D65206F664E
:10178000667365743A0020580020530020204D32C3
:101790003035204200416476616E6365643A2042D0
:1017A0003C6D696E5F7365676D656E745F74696DBE
:1017B000655F75733E20533C6D696E5F6665656459
:1017C000726174653E20543C6D696E5F747261761F
:1017D000656C5F66656564726174653E20583C6D3A
:1017E00061785F785F6A65726B3E20593C6D617805
:1017F0005F795F6A65726B3E205A3C6D61785F7AF3
:101800005F6A65726B3E20453C6D61785F655F6A1B
:1018100065726B3E0020540020520020204D323073
:1018200034205000416363656C65726174696F6E4A
:101830002028756E6974732F7332293A20503C70DA
:1018400072696E745F616363656C3E20523C7265C1
:1018500074726163745F616363656C3E20543C74B1
:10186000726176656C5F616363656C3E0020204D3C
:101870003230312058004D6178696D756D204163BB
:1018800063656C65726174696F6E2028756E69742A
:10189000732F7332293A0020204D32303320580004
:1018A0004D6178696D756D206665656472617465FA
:1018B000732028756E6974732F73293A0053746509
:1018C00070732070657220756E69743A0020440050
:1018D00020204D3230302053002044697361626C07
:1018E00065640A0046696C616D656E742073657489
:1018F00074696E67733A0020204D313439204320DB
:101900003B20556E69747320696E2043656C736962
:1019100075730A0020286D6D290020204732312080
:101920002020203B20556E69747320696E206D6DF8
:101930000000803B4400803B4400002041000096B2
:10194000420000A0420000A0420000C8430000BEC8
:1019500042D0070000D0070000640000004B0000E8
:101960000024F4D43050C38E20C2A24017828B7062
:1019700011127A910D816CD90AA861E108C75866E5
:1019800007615143061E4B5D05C145A7041A41116D
:1019900004093D9803713931034036DB0265339108
:1019A00002D4305402802E1D02632CEE01752AC52C
:1019B00001B028A001102781018F2564012B244B41
:1019C00001E0223401AC211F018D200D01801FFC9C
:1019D00000841EED00971DDF00B81CD200E61BC678
:1019E00000201BBC00641AB200B219A8000A19A09A
:1019F000006A189900D117910040178B00B5168422
:101A00000031167E00B31579003A157300C7146FC4
:101A10000058146A00EE1366008813630025135EF5
:101A200000C7125B006C12570015125400C111510F
:101A30000070114F0021114B00D61049008D104746
:101A4000004610440002104200C00F4000800F3ECC
:101A500000420F3C00060F3B00CB0E3800930E37C0
:101A6000005C0E3500270E3400F30D3200C10D313D
:101A700000900D3000600D2E00320D2D00050D2C54
:101A800000D90C2B00AE0C2900850C29005C0C271A
:101A900000350C27000E0C2600E80B2400C40B2494
:101AA00000A00B23007D0B23005A0B2100390B21D2
:101AB00000180B2000F80A1F00D90A1E00BB0A1EDE
:101AC000009D0A1D00800A1D00630A1C00470A1BB6
:101AD000002C0A1B00110A1A00F7091A00DD091967
:101AE00000C4091900AB091900920917007B0918F5
:101AF00000630917004C0916003609160020091664
:101B0000000A091500F5081500E0081400CC0814B7
:101B100000B8081400A4081400900813007D0812EF
:101B2000006B081300580812004608120034081110
:101B300000230811001208110001081100F007101D
:101B400000E0071000D0071000C0071000B0070F1A
:101B500000A107100091070E0083070F0074070F04
:101B60000065070E0057070E0049070E003B070DE2
:101B7000002E070E0020070D0013070D0006070DAD
:101B800000F9060C00ED060D00E0060C00D4060C72
:101B900000C8060C00BC060C00B0060C00A4060B26
:101BA0000099060C008D060B0082060B0077060BD1
:101BB000006C060B0061060A0057060B004C060A73
:101BC0000042060A0038060A002E060A0024060A09
:101BD000001A060A001006090007060A00FD05099A
:101BE00000F4050900EB050900E2050900D9050923
:101BF00000D0050900C7050900BE050900B50508A4
:101C000000AD050800A50509009C0508009405081D
:101C1000008C050800840508007C05080074050890
:101C2000006C050700650508005D050700560508FE
:101C3000004E050700470507004005080038050766
:101C400000310507002A050700230507001C0506CB
:101C500000160507000F0507000805060002050726
:101C600000FB040600F5040700EE040600E8040685
:101C700000E2040700DB040600D5040600CF0406DA
:101C800000C9040600C3040600BD040600B704062C
:101C900000B1040500AC040600A6040600A004057B
:101CA000009B04060095040500900406008A0405C4
:101CB0000085040500800406007A0405007504050B
:101CC00000700405006B040500660405006104054E
:101CD000005C04050057040500520405004D04058E
:101CE0000048040500430405003E0404003A0405CE
:101CF0000035040500300404002C0405002704040A
:101D000000230405001E0404001A04040016040540
:101D100000110404000D0404000904050004040477
:101D20000000040400FC030400F8030400F40304AE
:101D300000F0030400EC030400E8030400E40304DF
:101D400000E0030400DC030400D8030400D403040F
:101D500000D0030400CC030400C8030300C5030340
:101D60000024F404D9201BC40C5C0E9804C4095F41
:101D70000265077101F405F900FB04B3004804870C
:101D800000C10369005803550003034500BE023A31
:101D9000008402310053022A002902250004022097
:101DA00000E4011C00C8011900AF011700980114DC
:101DB0000084011300710110006101100051010E37
:101DC0000043010D0036010B002B010B0020010B1D
:101DD00000150109000C01090003010800FB0008BF
:101DE00000F3000800EB000700E4000600DE000638
:101DF00000D8000600D2000600CC000500C7000590
:101E000000C2000500BD000400B9000400B50004D4
:101E100000B1000400AD000400A9000400A5000307
:101E200000A20003009F0004009B00030098000331
:101E3000009500020093000300900003008D000253
:101E4000008B00030088000200860002008400036B
:101E500000810002007F0002007D0002007B000282
:101E60000079000200770001007600020074000291
:101E70000072000100710002006F0002006D00019D
:101E8000006C0002006A00010069000200670001A6
:101E900000660001006500010064000200620001AC
:101EA0000061000100600001005F0002005D0001B0
:101EB000005C0001005B0001005A000100590001B4
:101EC00000580001005700010056000100550001B4
:101ED00000540001005300000053000100520001B3
:101EE0000051000100500001004F0001004E0000B1
:101EF000004E0001004D0001004C0001004B0000AD
:101F0000004B0001004A00010049000100480000A8
:101F100000480001004700010046000000460001A3
:101F2000004500000045000100440001004300009E
:101F30000043000100420000004200010041000097
:101F40000041000100400001003F0000003F00018F
:101F5000003E0000003E0001003D0000003D000189
:101F6000003C0000003C0000003C0001003B000081
:101F7000003B0001003A0000003A00010039000077
:101F8000003900010038000000380000003800016E
:101F90000037000000370001003600000036000066
:101FA000003600010035000000350000003500015A
:101FB0000034000000340000003400010033000051
:101FC0000033000000330001003200000032000046
:101FD000003200010031000000310000003100013A
:101FE000003000000030000000300001002F000031
:101FF000002F0000002F0000002F0001002E000025
:10200000002E0000002E0001002D0000002D000019
:10201000002D0000002D0001002C0000002C00000D
:10202000002C0000002C0001002B0000002B000001
:10203000002B0000002B0001002A0000002A0000F5
:10204000002A0000002A00010029000000290000E9
:1020500000290000002900000029000100280000DC
:1020600000280000002800000028000000280001CF
:1020700000270000002700000027000000270000C4
:1020800000270001002600000026000000260000B6
:1020900000260000002600010025000000250000A9
:1020A000002500000025000000250000002500019B
:1020B0000024000000240000002400000024000090
:1020C0000024000100230000002300000023000082
:1020D0000023000000230000002300000023000173
:1020E0000022000000220000002200000022000068
:1020F0000022000000220001002100000021000059
:10210000002100000021000000210000002100004B
:10211000002100010020000000200000002000003D
:10212000002000000020000000200000002000002F
:1021300000200001001F0000001F0000001F000021
:10214000001F0000001F0000001F0000001F000112
:10215000001E0000001E0000001E0000001E000007
:1021600000043700001E290000511B000058100019
:102170000010090000CC04000078020000410100BA
:102180000020436F756E7420583A00426564004524
:102190003100626564002C2073797374656D20735F
:1021A000746F7070656421204865617465725F4961
:1021B000443A200048656174696E67204661696C25
:1021C00065640048656174696E67206661696C6565
:1021D00064004D3131322053687574646F776E003E
:1021E0001000C90210012C014001220170011801E8
:1021F000B0010E01F00104015002FA00B002F0003B
:102200003003E600D003DC009004D2007005C80063
:10221000A006BE000008B400B009AA00D00BA000C0
:10222000600E960060118C00001582002019780065
:10223000C01D6E00A0226400B0275A00902C5000F0
:1022400000314600E0343C0010383200903A28005B
:10225000603C1E00A03D1400803E0A00203F0000AC
:10226000544845524D414C2052554E41574159001A
:10227000546865726D616C2052756E61776179008A
:102280004572723A204D415854454D50004D4158C9
:1022900054454D50207472696767657265640045E6
:1022A00072723A204D494E54454D50004D494E549E
:1022B000454D502074726967676572656400202F10
:1022C000002042403A0020403A007C3C3E5E2B3DDC
:1022D0003F2F5B5D3B2C2A225C0043616E6E6F7466
:1022E000206F70656E2073756264697220005344BC
:1022F0002063617264206F6B0A006F70656E526FAD
:102300006F74206661696C65640A00766F6C756D28
:10231000652E696E6974206661696C65640A004E99
:102320006F20534420636172640A000A4D32340006
:102330004D3233202573002E0A006F70656E2066C3
:1023400061696C65642C2046696C653A20004669B9
:102350006C652073656C65637465640A002053695D
:102360007A653A200046696C65206F70656E656419
:102370003A2000454E4420535542524F5554494E41
:10238000450A002220706F73002220706172656E12
:10239000743A2200535542524F5554494E452043FA
:1023A000414C4C207461726765743A220053756227
:1023B00063616C6C204F766572666C6F7700457850
:1023C000636565646564206D617820535542524FA2
:1023D0005554494E452064657074683A00577269D7
:1023E00074696E6720746F2066696C653A200066B8
:1023F0007265736800646F696E67002066696C655A
:102400003A20004E6F7720002F6175746F25632E80
:1024100067006001F4017001EA019001E001B00180
:10242000D601D001CC010002C2013002B801600225
:10243000AE019002A401D0029A0120039001700322
:102440008601C0037C0130047201A00468012005EC
:102450005E01B005540160064A0120074001F00703
:102460003601F0082C01100A2201500B1801C00C93
:102470000E01500E04013010FA002012F00050142A
:10248000E600C016DC007019D200501CC800501FB6
:10249000BE007022B400B025AA00F028A000202CB5
:1024A0009600302F8C0010328200A0347800F03675
:1024B0006E00E0386400803A5A00403B5500E03B33
:1024C0005000F03C4600C03D3C00603E3200E03E23
:1024D0002800303F1E00503F1900703F1400A03FFD
:1024E0000A00C03F0000D03FF6FFE03FECFF202095
:1024F000506C616E6E657242756666657242797483
:1025000065733A20002046726565204D656D6F72D7
:10251000793A2000436F6D70696C65643A204170B0
:102520007220323420323032310A00204C61737410
:1025300020557064617465643A20323032312D3038
:10254000342D3138207C20417574686F723A2054E4
:10255000696E794D616368696E657333440A003250
:102560002E302E375F4457372E330A004D61726C80
:10257000696E0020536F66747761726520526573CF
:1025800065740A00205761746368646F6720526540
:102590007365740A002042726F776E206F75742025
:1025A00052657365740A002045787465726E616CBB
:1025B0002052657365740A00506F77657255700A12
:1025C0000073746172740A004732385859004D31F3
:1025D000303031006F6B006572726F7220777269F4
:1025E00074696E6720746F2066696C650A00446FB9
:1025F0006E6520736176696E672066696C652E0A68
:10260000004D323900456E6473746F70730025534A
:1026100020256320256320256320256300205A3A66
:102620000020593A0020583A00656E6473746F7048
:1026300073206869743A2000000000010200090A52
:102640000000000004030807000000000000000074
:102650000000000000000000004D6F76652025732B
:102660006D6D004D6F766520302E316D6D004D6FB4
:10267000766520316D6D004D6F76652031306D6D62
:10268000004D6F76652041786973004578747275E6
:10269000646572004D6F7665205A004D6F76652037
:1026A00059004D6F76652058005072696E7420662F
:1026B000726F6D204D6564696100FFFFFF486F6DAB
:1026C0006520257325732573204669727374002273
:1026D0000A00556E6B6E6F776E20636F6D6D616E65
:1026E000643A202200544D334420456E64657233B1
:1026F0002052656164792E005072696E74696E674C
:102700002E2E2E005072696E7420506175736564B0
:1027100000204500205A00205900204D3932205811
:102720000020453A00205A3A0020593A00583A0011
:102730004572726F722077726974696E6720746F68
:1027400020454550524F4D210A0020746F6F206C78
:102750006F6E6720657874727573696F6E20707222
:102760006576656E7465640A0020636F6C6420652D
:102770007874727573696F6E2070726576656E74A9
:1027800065640A00526573656E643A200000002299
:1027900000250028002B0000002100240027002A2B
:1027A00000020202020202020204040404040404FD
:1027B00004030303030303030301010101010101F6
:1027C000010102040810204080010204081020408A
:1027D000800102040810204080804020100804027C
:1027E000012F2F616374696F6E3A000087D65ADD3E
:1027F00011241FBECFEFD0E4DEBFCDBF12E0A0E0BA
:10280000B1E0E4E1F7ED01E00BBF02C007900D92EB
:10281000AE31B107D9F727E1AEE1B2E001C01D92B8
:10282000A93BB207E1F713E1C7EFD3E104C0219759
:10283000FE010E94E1E8C63FD107C9F70E94ABD76D
:102840000C947DEB0C9400008F929F92AF92BF92FC
:10285000CF92DF92EF92FF92CF936B017C0120E049
:1028600030E0A9010E94FCE187FD9FC06DEB77E39A
:1028700086E095E3A70196010E94F3E86B017C01D5
:1028800020E030E040E251E40E9462E220E030E0EB
:1028900048EC52E40E9462E24B015C0120E030E02F
:1028A000A901C701B6010E94FCE120E030E040EA46
:1028B00050E487FF04C020E030E040EA50ECC5015E
:1028C000B4010E94F3E820E030E040E251E40E94CD
:1028D00076E90E94E8E96B017C018BE2F7FE09C012
:1028E000F094E094D094C094C11CD11CE11CF11C64
:1028F0008DE28093D503C701B60120E137E240E0C5
:1029000050E00E94C2E88AE0882E912CA12CB12CC4
:10291000CA01B901A50194010E94C2E8605D6093FB
:10292000D603C701B60128EE33E040E050E00E9434
:10293000C2E8CA01B901A50194010E94C2E8605D24
:102940006093D703C701B60124E630E040E050E0D1
:102950000E94C2E8CA01B901A50194010E94C2E81F
:10296000605D6093D8038EE28093D903C701B601FE
:10297000A50194010E94C2E8C62FCA01B901A501B0
:1029800094010E94C2E8605D6093DA03C05DC09369
:10299000DB0385ED93E0CF91FF90EF90DF90CF9038
:1029A000BF90AF909F908F9008956DEB77E386E096
:1029B00095EB60CF8F929F92AF92BF92CF92DF92B2
:1029C000EF92FF92CF936B017C0120E030E0A901F0
:1029D0000E94FCE187FDAAC06DEB77E386E095E3FA
:1029E000A70196010E94F3E86B017C0120E030E032
:1029F000A9010E94FCE187FF9EC0C701B601905863
:102A000020E030E040E251E40E9462E220E030E069
:102A100040E251E40E9462E220E030E040EA50E40B
:102A20000E94F3E820E030E040E251E40E9476E9C1
:102A30000E94E8E96B017C0180E28093D50360E2AB
:102A400080E1C81687E2D806E104F1048CF0C701E2
:102A5000B60120E137E240E050E00E94C2E8CA013E
:102A6000B9012AE030E040E050E00E94C2E8605D39
:102A70006093D60360E288EEC81683E0D806E104CE
:102A8000F1048CF0C701B60128EE33E040E050E0DD
:102A90000E94C2E8CA01B9012AE030E040E050E0FB
:102AA0000E94C2E8605D6093D70360E284E6C816C6
:102AB000D104E104F1048CF0C701B60124E630E052
:102AC00040E050E00E94C2E8CA01B9012AE030E0CB
:102AD00040E050E00E94C2E8605D6093D8038AE065
:102AE000882E912CA12CB12CC701B601A50194010F
:102AF0000E94C2E8C62FCA01B901A50194010E9433
:102B0000C2E8605D6093D9038EE28093DA03C05D12
:102B1000C093DB0385ED93E0CF91FF90EF90DF90C2
:102B2000CF90BF90AF909F908F9008956DEB77E31B
:102B300086E095EB55CF20E030E040E251E4C7015C
:102B4000B60162CFCF93DF93EC01CB01BA010E94B3
:102B500003E220E030E040E251E40E9476E920E028
:102B600030E0A9010E94F3E8688379838A839B831C
:102B7000DF91CF9108950E9403E220E030E040E22F
:102B800051E40E9476E920E030E0A9010E94F3E8D8
:102B90000C94DA14CF93DF93EC01CB01BA010E94BD
:102BA00003E220E030E048EC52E40E9476E920E0C5
:102BB00030E0A9010E94F3E8688379838A839B83CC
:102BC000DF91CF9108950E9403E220E030E048ECCD
:102BD00052E40E9476E920E030E0A9010E94F3E887
:102BE0000C942414CF93DF93EC01CB01BA010E9423
:102BF00003E220E030E0A9010E94F3E868837983D2
:102C00008A839B83DF91CF910895CF93DF93EC016B
:102C1000CB01BA010E9403E220E030E0A9010E944A
:102C2000F3E8688379838A839B83DF91CF9108954A
:102C3000CF93DF93EC01CB01BA010E9403E22AE0BB
:102C400037ED43E25DE30E9476E920E030E0A90140
:102C50000E94F3E80E94EFE9688379838A839B836B
:102C6000DF91CF910895CF93DF93EC01CB01BA01AF
:102C70000E9403E22AE037ED43E25DE30E9476E939
:102C800020E030E0A9010E94F3E8688379838A8319
:102C90009B83DF91CF910895CF93DF93EC01CB011C
:102CA000BA010E9403E220E030E04AE754E40E94C7
:102CB00076E920E030E0A9010E94F3E86883798397
:102CC0008A839B83DF91CF910895FC0184910895BD
:102CD000FC0180810895FC0180E09191992329F005
:102CE000907C9038D1F38F5FF8CF08951198000051
:102CF000000087FD52C0419800000000119A0000BA
:102D0000000011980000000086FD53C041980000AB
:102D10000000119A0000000011980000000085FDDD
:102D200046C0419800000000119A00000000119870
:102D30000000000084FD39C0419800000000119A95
:102D40000000000011980000000083FD2CC0419895
:102D500000000000119A000000001198000000001F
:102D600082FD1FC0419800000000119A0000000081
:102D700011980000000081FD12C041980000000081
:102D8000119A000000001198000000004198000016
:102D90000000119A000000000895419AADCF419AB9
:102DA000EDCF419AE0CF419AD3CF419AC6CF419A15
:102DB000B9CF419AACCF90E080E00895CF93DF93F4
:102DC000DB01F9019C919130C1F0943080F0945076
:102DD0009C938830D1F480819181009771F00197A4
:102DE00091838083480F591FEA01188206C08C35F1
:102DF00039F49C5F9C93943041F4DF91CF91089516
:102E00008B3339F781E08C93F8CF20813181B90180
:102E10006F5F7F4F71836083420F531FEA01888386
:102E2000808191818F3591056CF7E7CF0F931F93C8
:102E300081E00091C2161091C3162091C416309102
:102E4000C5164091BE165091BF166091C016709184
:102E5000C116041715072607370708F480E01F91ED
:102E60000F910895282F90914003833021F495FD10
:102E70000FC094FD0FC0892F90E0B0E0A0E004C027
:102E8000B695A795979587952A95D2F7817008955D
:102E900081E0089580E0089580915301882341F0F6
:102EA0006091D0037091D10341E081E00C940CBC9F
:102EB000089563E972E084E690E00E949A946AEBD8
:102EC00072E084E690E00C949A9481110C94591766
:102ED00068EB71E084E190E00C949A94CF93DF93D7
:102EE00000D000D0CDB7DEB70E94EFE90E9401E22A
:102EF00069837A838B839C83CE0101960E94C09064
:102F00000F900F900F900F90DF91CF9108950E9436
:102F100003E22AE037ED43E25DE30E9476E920E038
:102F200030E0A9010E94F3E80C946E17CF92DF9273
:102F3000EF92FF92CF93DF9300D000D0CDB7DEB7F2
:102F40006B017C0120E030E0A9010E94FCE187FDDB
:102F50001BC06DEB77E386E095E3A70196010E9425
:102F6000F3E869837A838B839C83CE0101960E9468
:102F7000C0900F900F900F900F90DF91CF91FF9026
:102F8000EF90DF90CF9008956DEB77E386E095EBBF
:102F9000E4CF0E9403E22AE037ED43E25DE30E94C2
:102FA00076E920E030E0A9010E94F3E80C9496173E
:102FB0000E9403E220E030E0A9010E94F3E80C94B3
:102FC0009617CF92DF92EF92FF926B017C0120E087
:102FD00030E0A9010E94FCE187FD26C06DEB77E39C
:102FE00086E095E3A70196010E94F3E86B017C015E
:102FF00020E030E0A9010E94FCE120E030E040E068
:103000005FE387FF04C020E030E040E05FEBC701F2
:10301000B6010E94F3E80E94E8E9CB01FF90EF902F
:10302000DF90CF900C945E926DEB77E386E095EBAA
:10303000D9CF0E9403E220E030E0A9010E94F3E82A
:103040000C94E1170E9403E220E030E04AE754E4E8
:103050000E9476E920E030E0A9010E94F3E80C9498
:10306000C794EF92FF920F931F9381E8E82E8DE0B3
:10307000F82E04E91DE030E020E045E75DE163E87B
:103080007DE08AE89DE00E94A0C41F910F91FF900F
:10309000EF9008950E9469740C9465170E941C8F2C
:1030A0000C9459170C947A770C947A770C947A775D
:1030B0000C947A770C942C770C942C770C942C77B6
:1030C0000C942C770E9458A60C946517AF92BF926F
:1030D000CF92DF92EF92FF920F931F93CF93DF93E4
:1030E0006B01E9014A3009F4B8C0453109F06AC002
:1030F000DB011296ED91FC91F280C681D781139A83
:1031000088E28A950000E9F7BF2CB29420EFB22242
:1031100030E1A32EAF0C48E2E42E88EF0E94761631
:103120008E2D8A950000E9F7BFE1BF1508F481C034
:103130008F2D807780680E9476168B2D0E947616E0
:103140008E2D8A950000E9F780E80E94761680E0CF
:103150000E9476168E2D8A950000E9F78AEF0E946C
:1031600076168E2D8A950000E9F78E01005F1F4FBD
:103170008881807F0E94761689918295807F0E9447
:103180007616C017D107A1F78E2D8A950000E9F7B2
:10319000F394E0E1BE0EFA10C0CF1398D601129658
:1031A000CD91DC91CE010E946DC28111EEC1DF9103
:1031B000CF911F910F91FF90EF90DF90CF90BF9034
:1031C000AF900895FB0102811381423309F498C145
:1031D00008F49CC1463409F489C1473409F48CC110
:1031E0004B3329F589812B81D80112966C91129766
:1031F00013964C91213009F4DFC1233009F0A9C1A5
:1032000038EF380F582F91E0431708F490E041E071
:10321000531708F040E031E0561708F430E0592F1A
:10322000542B352309F0BDC1942309F0BAC181E0C4
:10323000BECF80EE8F0D8068807F0E9476168F2D26
:103240008295807F0E9476168E2D8A950000E9F780
:1032500080E80E94761680E87BCF0B9A1398399A03
:103260004198099A119A139A88E28A950000E9F721
:1032700088E790E0CEE9DFE0FE013197F1F70197B2
:10328000D9F788EF0E94761618E2812F8A95000000
:10329000E9F780E20E94761680E00E947616812F80
:1032A0008A950000E9F780E00E94761680E80E9487
:1032B0007616812F8A950000E9F780E00E94761645
:1032C00080E10E947616812F8A950000E9F7CE01F1
:1032D0000197F1F7CE010197F1F7CE010197F1F7D0
:1032E000CE010197F1F7CE010197F1F7CE010197D9
:1032F000F1F7CE010197F1F7CE010197F1F7CE0179
:103300000197F1F7CE010197F1F7CE010197F1F79F
:10331000CE010197F1F7CE010197F1F7CE010197A8
:10332000F1F72197F1F780E20E94761680E40E947F
:103330007616812F8A950000E9F780E20E947616C2
:1033400080E60E9476161A950000E9F710E0D0E0BA
:10335000C8E28D2F807780680E947616812F0E94A8
:1033600076168C2F8A950000E9F780E80E94761681
:1033700080E00E9476168C2F8A950000E9F78AEF8C
:103380000E9476168C2F8A950000E9F780E211984A
:1033900000000000419800000000119A00000000A9
:1033A000119800000000419800000000119A0000F0
:1033B0000000119800000000419800000000119AE0
:1033C000000000001198000000004198000000007B
:1033D000119A0000000011980000000041980000C0
:1033E0000000119A000000001198000000004198B0
:1033F00000000000119A0000000011980000000079
:10340000419800000000119A00000000119800008F
:103410000000419800000000119A0000000011987F
:1034200000000000419800000000119A0000000018
:10343000119800000000419800000000119A00005F
:103440000000119800000000419800000000119A4F
:1034500000000000119800000000419800000000EA
:10346000119A00000000119800000000419800002F
:103470000000119A0000000011980000000041981F
:1034800000000000119A00000000119800000000E8
:10349000419800000000119A0000000011980000FF
:1034A0000000419800000000119A000000009C2FCD
:1034B0009A950000E9F7815009F069CF88EF0E94E2
:1034C00076168C2F8A950000E9F7DF5F105FD03207
:1034D00009F03FCF80E00E94761680EC0E947616BD
:1034E000CA950000E9F7139881E061CED8011596DE
:1034F0008C91888381E05BCEF80181818883FACF4B
:10350000B901C8010E948AC281E051CE443171F0F4
:10351000473109F08CCE1882F80182818983858138
:1035200081508A8383818B8381E041CED8011596B7
:103530004C91159750E0440F551F70E060E01696CF
:103540008D919C910E941EEBC8010E9483C281E074
:103550002ECE481708F46BCE861708F468CEFA8092
:10356000E12CD12C243070F41DC0BE01C8010E9492
:103570008AC2898198819D0D98838E0D8983FF0C65
:1035800009F455CEF7FEF6CFF0CF4D8150E0440F51
:10359000551F70E060E08E819F810E941EEB81E0EC
:1035A00006CEFA8030E0F901EE58FE4FD080225965
:1035B0003E4FF901E080E6CF58E0580F382F23CE78
:1035C00020914803022E000C330B8217130641F0A2
:1035D000809348036EE07EE08AE495E10C9442C655
:1035E0000895EF92FF920F931F93CF93DF93EC0117
:1035F0008B017A018A859B858617970731F0888130
:1036000099810E9442C61B870A87B70188819981E8
:103610000E94E2BC2E813F81820F932F911D9F83D8
:103620008E8390E080E0DF91CF911F910F91FF900A
:10363000EF9008959F92AF92BF92CF92DF92EF9258
:10364000FF920F931F93CF93DF93EC018B01942E86
:10365000A52E8A859B858617970731F088819981E9
:103660000E9442C61B870A8788859985019649F57D
:10367000BC800A818E81080FC880D980D6015596FA
:10368000ED91FC91C6010995B80EE92CFA2C10E0D9
:10369000F70121917F01211127C08E819F81810F28
:1036A000911D9F838E8390E080E0DF91CF911F91E9
:1036B0000F91FF90EF90DF90CF90BF90AF909F90D1
:1036C00008950E811F81692D7A2D888199810E942C
:1036D000E2BC800F912F911D288539852817390765
:1036E00038F681E090E0E1CF4B2D602FC6010E94BB
:1036F0009AC6080F180FCCCFDF92EF92FF920F936C
:103700001F93CF93DF93EC01D62E1CAD0BAD7C0144
:1037100084E0E80EF11CE98DFA8DC7010995412F6F
:10372000480F2D2D602FC7010E949AC69BAD890FAF
:103730008BAF81E090E0DF91CF911F910F91FF90CF
:10374000EF90DF900895CF92DF92EF92FF920F9368
:103750001F93CF93DF93CDB7DEB72C970FB6F894B6
:10376000DEBF0FBECDBFF0908115E0908215209195
:103770004A0321111DC048E75BE06E2D8F2D0E948A
:1037800006C790E080E0F80EF0928115E092821575
:1037900099272C960FB6F894DEBF0FBECDBFDF91F0
:1037A000CF911F910F91FF90EF90DF90CF900895F0
:1037B000C0904E15D0904F152AE435E13A83298305
:1037C0002F2D30E03C832B832E2D30E03E832D8344
:1037D00018861F827A8769871C861B860AE11BE18F
:1037E0009E012F5F3F4F45E656E1BC01C6010E9496
:1037F00053B6B6018AE495E10E9442C68F8198854E
:10380000C2CFEF92FF920F931F93CF937C01009151
:10381000430310914403C0E0F701EC0FF11D6081F8
:10382000662351F0062E000C770BC8010E9443EB73
:10383000892B49F4CF5FF0CF80E0CF911F910F919A
:10384000FF90EF90089581E0F8CF682F880F770BF5
:1038500080914303909144030E9443EBFC0181E07B
:10386000309709F480E0309781F0918120ED290FA5
:103870002A3030F09E3251F4928190539A3098F46D
:103880003196F0933503E093340308959D3211F09F
:103890009B3249F4928120ED290F2A3088F39E3221
:1038A00011F49381EACFF0E0E0E0EBCF80913403B4
:1038B00090913503009731F04AE050E070E060E00D
:1038C0000C941EE060E070E0CB0108958091340319
:1038D00090913503009731F04AE050E070E060E0ED
:1038E0000C94F0DE60E070E0CB0108950E94661C4D
:1038F000CB0108950F931F93CF9380913403909140
:1039000035030097E9F0FC018F01C1912C2F2F7D29
:1039100081F0C53411F0C536B9F7F801108270E0B6
:1039200060E00E9492DDF801C083CF911F910F915A
:10393000089570E060E0CF911F910F910C9492DD9B
:1039400060E070E0CB01F1CFCF93DF93CDB7DEB76E
:1039500020E24F8158856E818D810E9469BCDF9184
:10396000CF9108958F929F92AF92BF92EF92FF9264
:103970000F931F93CF93DF93EC018B01E42EF22E74
:1039800080914415909145158C179D0709F43EC010
:103990002091CA0327FD1092CA032AE9C239D2072F
:1039A00009F03FC08450944371F40E9482C16E516B
:1039B0007B4F8F4F9F4F6093CC037093CD038093C9
:1039C000CE039093CF03D0934515C093441530E0B8
:1039D00020E00093CE051093CF052093D0053093BF
:1039E000D105E092C705F092C805C450D44321F434
:1039F0001092C6051092CB0382E08093530181E0C0
:103A00008093DE051092D4031092C505DF91CF910B
:103A10001F910F91FF90EF90BF90AF909F908F906C
:103A2000089524E3C430D20771F682599A4919F0F7
:103A3000C4E0D4E3C8CF0E9482C18090CC039090B0
:103A4000CD03A090CE03B090CF03681979098A09FD
:103A50009B0997FFEDCF809194058770873041F7E0
:103A6000C0E7D6E6B0CF80911E1590911F15891B37
:103A70008F7051F480910006813031F08091C6162C
:103A800082FB882780F9089581E00895E091CB03B7
:103A9000E63010F581E08E0F8093CB034091CE0588
:103AA0005091CF056091D0057091D1059091C705D7
:103AB0008091C80528E0E29FF0011124E656FC4FF2
:103AC00020914415309145153183208342835383DF
:103AD0006483758396838783089520E040E070E0D7
:103AE00060E084E094E30C94B21CCF930E941C8F9E
:103AF0000E946974C82F882319F080E00E9484A076
:103B00008C2F0E946517CF910C946D1DE091CB0313
:103B1000EE2389F0E150E093CB0388E0E89FF001C9
:103B20001124E656FC4F6281738127814681808192
:103B300091810C94B21C0C946D1D8091D203811163
:103B400006C01092C6050E94861D0E9459178091DA
:103B50005301882331F041E062EF7DE081E00E9473
:103B60000CBC82E08093530108954F925F926F9254
:103B70007F928F929F92AF92BF92CF92DF92EF92FD
:103B8000FF920F931F93CF93DF930E94331D782EE4
:103B90000E9495BDC091C70515E0711001C016E0E7
:103BA0006C2E85E0582E5C0E05E00C1B84E0F82E90
:103BB000FC1A83E0E82EEC1A82E0982E9C1A9FE80B
:103BC000A92E9DE0B92E23EDC22E2DE0D22E81E04C
:103BD000882E8C1A4C2E4194C11132C08091C90597
:103BE000882389F080915301882309F447C081E03C
:103BF0009091C905911180E024E044EE5DE0642DD0
:103C00000E9469BC3BC08091C4051092C405882302
:103C100049F30E94861D8091DE05882319F3DF9108
:103C2000CF911F910F91FF90EF90DF90CF90BF90B9
:103C3000AF909F908F907F906F905F904F9008957E
:103C4000C13009F05BC08091C905813009F443C0DF
:103C500080915301882391F01F92DF92CF928F922F
:103C600081E09091C905913009F080E08F930E9426
:103C7000A41C0F900F900F900F900F90711079C0AF
:103C8000C53009F076C08091C905853009F49EC021
:103C9000809153018111ABC0D6E081E08D0F8C1370
:103CA00013C09091C9059C1709F4CCC080915301B1
:103CB000882351F06C2F661981E09C1380E023E08B
:103CC00044E95DE00E9469BCCF5FC51185CFDE5F2E
:103CD000D093C805A4CF8091C4051092C405882351
:103CE00009F4B6CFB092A205A092A1050E946D1D65
:103CF0008091DE05882309F4ABCF91CFC23009F063
:103D0000C2C08091C905823081F08091530188231F
:103D100009F4B4CF81E09091C905923009F080E0B8
:103D200023E04AEC5DE0692D6BCF8091C4051092D1
:103D3000C405882351F38EE496E20E94FB9480919F
:103D4000DE05882311F36BCF8091C9058330F1F034
:103D500080915301882309F491CF81E09091C905A6
:103D6000933009F080E023E04DEB5DE06E2D0E9482
:103D700069BC1C1309C08091C905811709F444C0AE
:103D800080915301811151C0D12F87CF8091C405FB
:103D90001092C4058823E1F28EE198E20E94FB9420
:103DA0008091DE058823A1F23ACF8091C40510925C
:103DB000C405882309F472C087E19BE20E94FB944A
:103DC0008091DE05882309F469C029CF8091C4055C
:103DD0001092C405882309F45BCF85EF9CE20E9412
:103DE000FB948091DE05882309F452CF18CF81E03F
:103DF0009091C905953009F080E023E04FEA5DE03D
:103E0000602F0E9469BC48CF8091C4051092C40500
:103E1000882309F4B5CF84E29EE20E94FB9480914E
:103E2000DE05882309F4ACCFFACE6C2F661981E049
:103E30009091C9059C1380E023E046EA5DE00E9472
:103E400069BCA2CF8091C4051092C405882309F4EF
:103E50002DCF0E94461D20E040E070E060E081E34D
:103E600098E1DF91CF911F910F91FF90EF90DF903C
:103E7000CF90BF90AF909F908F907F906F905F900A
:103E80004F900C94B21CC33009F45ECFC43009F0DB
:103E9000F5CE8091C905843009F487CF8091530114
:103EA000882309F4EBCE81E09091C905943009F0A4
:103EB00080E023E048EB5DE06F2D59CFCF93DF9397
:103EC000CDB7DEB78D8190919612891768F08093F7
:103ED00096129E01285F3F4F4E815F816AE270E03B
:103EE0008BE692E10E94C3E1DF91CF9108950F9399
:103EF0001F93CF93DF938C016F3F19F410929612AA
:103F000060E020919612862F062E000C990B281740
:103F1000190609F0F4F460939612C8010E9449E171
:103F2000800F911FEC01C01BD10BCB32D1053CF0AF
:103F30000197FC012491207C2038D1F3F3CFDD27B9
:103F4000AE01B8018BE692E10E946AE1C559DD4EEF
:103F50001882DF91CF911F910F910895CF93809197
:103F60009203811109C082E99CE09093D103809370
:103F7000D00381E0809392030E94461D20E040E040
:103F800070E060E08CE497E10E94B21CC1E0C09355
:103F9000C6050E949E771092C6050E94861DC0939A
:103FA000C60560E084E097E20E94771F8EE89CE0FF
:103FB0009093A2058093A105CF910895109291034B
:103FC000109252018091C61680648093C61689E7CC
:103FD0009CE00E9480B560E080E89CE00E94771F32
:103FE0000C946D1D0F931F930E9482C100918D034D
:103FF00010918E0320918F0330919003601B710B01
:10400000820B930B97FD0CC089B183FB882780F945
:1040100091E089274A9B8260309B846080938C0367
:1040200080918C03817090918C0391FD82609091BE
:104030008B03981749F0813009F148F0823079F00C
:10404000833091F080938B031F910F9108959130ED
:1040500079F09230B9F790918A0391500CC099236E
:1040600039F09330C1F3EECF9130A9F3923051F78C
:1040700090918A039F5F90938A03E4CF992359F329
:10408000933001F7F5CFCF92DF92EF92FF92CF936B
:10409000C82F0E9482C16B017C0124EA30E74DE702
:1040A0005FE360911B0170911C0180911D01909153
:1040B0001E010E94FCE187FD18C08AEF90E0A0E09D
:1040C000B0E08C0D9D1DAE1DBF1D80937A039093B3
:1040D0007B03A0937C03B0937D03C0931901CF9120
:1040E000FF90EF90DF90CF90089580E090E0DC01AA
:1040F000E8CFCF9380914B03811154C0109281156A
:10410000109282151092831510924F1510924E1531
:1041100010925115109250151092531581E0809312
:10412000521582E280935415109259151092581529
:10413000EDE6F5E12BE735E18FEF81932E173F0791
:10414000E1F7C1E0C0936A152EE037EA30936015BD
:1041500020935F15C093611510926215109263153C
:1041600090E490936415109265152CED36EA309327
:104170007C1520937B1521E131E030934D15209380
:104180004C159EE19093711591E1909372159CE10D
:1041900090936F1580936E1580936D150E94CBC21E
:1041A000C0934B0381E080934A0386EC9BE090939D
:1041B00098148093971410929A141092991453980B
:1041C0005B9A52985A9A3898409A0E94F21F10921D
:1041D0008A03CF910895FC01A081B1811C92A28134
:1041E000B3818C918F5F8C930280F381E02D90815D
:1041F0008CE0989F800D1124E6E4F5E113AE84AFC6
:104200000895FC0180E09491992331F0907C9038DE
:1042100009F08F5F3196F7CF0895AF92BF92CF929A
:10422000DF92EF92FF920F931F93CF93DF93EC01F6
:104230005B018A01FB01099587FD16C0C82ED12CB0
:10424000F12CE12C2196F801C082D182E282F38226
:10425000CE01DF91CF911F910F91FF90EF90DF90F2
:10426000CF90BF90AF900895982F907E903CA9F486
:104270008F7190E0B0E0A0E06C017D0156E0CC0CC5
:10428000DD1CEE1CFF1C5A95D1F7CE010196F501FD
:1042900009958F73C82A2296D6CF982F907F903E8B
:1042A00011F58F7090E0B0E0A0E06C017D0136E088
:1042B000CC0CDD1CEE1CFF1C3A95D1F7CE0101960B
:1042C000F50109958F73C82A46E0CC0CDD1CEE1C65
:1042D000FF1C4A95D1F7CE010296F50109958F731F
:1042E000C82A2396B0CF982F987F903F79F5877092
:1042F00090E0B0E0A0E06C017D0186E0CC0CDD1C1C
:10430000EE1CFF1C8A95D1F7CE010196F5010995A7
:104310008F73C82A96E0CC0CDD1CEE1CFF1C9A950E
:10432000D1F7CE010296F50109958F73C82A26E0D0
:10433000CC0CDD1CEE1CFF1C2A95D1F7CE01039698
:10434000F50109958F73C82A24967DCF982F907C0C
:10435000903841F4807C803869F42196CE01F501D3
:104360000995F8CF8E7F8D3F28F02196CE01F5017B
:104370000995F8CFC12CD12C760165CF9CE0899F9F
:10438000802D112491E0980F909349032CE0280F81
:104390002093E40530E02E5F3F4F40917E15421799
:1043A000130619F014F080E00895209180159217FB
:1043B000D0F7662341F08E5F0E94ECC38091E40544
:1043C0008E5F0E94ECC38091E40590917E15891761
:1043D00050F32091801590914903291720F31092F2
:1043E00081158093821581E00895CF92DF92EF923C
:1043F000FF920F931F93CF93DF93CDB7DEB72C9728
:104400000FB6F894DEBF0FBECDBF6F3F71058105BB
:10441000910509F0D0F486E495E10E947C1BE091BF
:104420004E15F0914F153196849190E02C960FB671
:10443000F894DEBF0FBECDBFDF91CF911F910F91DA
:10444000FF90EF90DF90CF900895F0908115E0906D
:10445000821520914A0321110FC048E95BE06E2DBF
:104460008F2D0E9406C790E080E0F80EF092811533
:10447000E09282159927DACFC0904E15D0904F1553
:104480002AE435E13A8329832F2D30E03C832B83C6
:104490002E2D30E03E832D8318861F822FEF3FEFB5
:1044A0003A8729871C861B860AE11BE19E012F5F44
:1044B0003F4FAB01BC01C6010E948FB5B6018AE433
:1044C00095E10E9442C68F819885CFCFAF92BF926F
:1044D000CF92DF92EF92FF920F931F93CF93DF93D0
:1044E00000D000D0CDB7DEB77C01062F6A01122FB5
:1044F00086E0A82EB12C11160CF040C0AE014F5F23
:104500005F4F65E676E1C7010E940D217C0169815C
:104510007A818B819C81611571058105910571F10D
:104520006D3371058105910509F450C06E37710531
:104530008105910509F44AC06A327105810591052A
:1045400069F507FF12C08CEB9BE00E3F11F088EB82
:104550009BE026E01202B00111240E94A31B66E03A
:1045600070E00E94AEE8161B61C065E470E080E078
:1045700090E00E94F521115059F510E0812F0F9025
:104580000F900F900F90DF91CF911F910F91FF909F
:10459000EF90DF90CF90BF90AF9008956432710597
:1045A0008105910579F4C114D10461F026E012026D
:1045B000B0011124C6010E94A31BB5010E94AEE800
:1045C000161B99CF0E94F521115095CF07FDBBCF47
:1045D00061E089819A81AB81BC81CD97A105B1054C
:1045E00009F460E0600F6A30ACF01150862F6AE089
:1045F0000E948CE8092F682F880F770B605D7F4F32
:10460000072E000C880B990B0E94F521112309F449
:10461000B4CF602F062E000C770B605D7F4F072E06
:10462000000C880B990B0E94F5211150112309F4FD
:10463000A4CF86E01802B0011124C7010E94A31B79
:1046400066E070E00E94AEE8161B98CF6FEF7FEF38
:104650000C94A31BCF92DF92EF92FF920F931F93C4
:10466000CF93DF93CDB7DEB72C970FB6F894DEBFAC
:104670000FBECDBFF0908115E090821520914A03C6
:1046800021111DC048E55BE06E2D8F2D0E9406C7ED
:1046900090E080E0F80EF0928115E0928215992763
:1046A0002C960FB6F894DEBF0FBECDBFDF91CF9131
:1046B0001F910F91FF90EF90DF90CF900895C090E1
:1046C0004E15D0904F152AE435E13A8329832F2DDA
:1046D00030E03C832B832E2D30E03E832D831886E3
:1046E0001F827A8769871C861B860AE11BE19E016F
:1046F0002F5F3F4F48E656E1BC01C6010E9453B60A
:10470000B6018AE495E10E9442C68F819885C2CFA6
:104710006FEF7FEF0C942A23AF92BF92CF92DF927C
:10472000EF92FF920F931F93CF93DF935C016B0186
:104730000E940121E82EC6010E946B16F12C03E1B4
:1047400010E0081B1109C5E20E151F050CF4CFE19E
:104750008C2F90E09C012E5F3F4F40917E154217B9
:10476000130609F0CCF50997209180152817190632
:104770009CF14091E6055091E7056091E5051092A6
:104780008115C093821525E1C5010E946622D1E002
:10479000C114D104B1F06AE370E080E090E00E94BF
:1047A000F5210E151F05D4F4C45F80917E15C8173E
:1047B00040F0209180154C2F4950550B24171506B9
:1047C0007CF4DF91CF911F910F91FF90EF90DF90DC
:1047D000CF90BF90AF900895D0E0DACFDD2389F37A
:1047E000802F880F080F000F00938115C09382154A
:1047F00060E270E080E090E00E94F521C601DF9168
:10480000CF911F910F91FF90EF90DF90CF90BF90CD
:10481000AF900C948823CF92DF92EF92FF92CF93C8
:10482000DF9300D000D0CDB7DEB78091C4051092E1
:10483000C405882331F18091D3038F5F8093D30324
:104840008931E0F081E08093D20320E040E070E025
:1048500060E08DE99DE10E94B21C88E09EE09093AB
:10486000A2058093A1050F900F900F900F90DF91FC
:10487000CF91FF90EF90DF90CF9008950E9456A0C7
:10488000F2CF6091CE057091CF058091D0059091C7
:10489000D105611571058105910509F43EC00E949D
:1048A00003E22DEC3CEC4CEC5CE30E9462E22091D4
:1048B0004C0B30914D0B40914E0B50914F0B0E9481
:1048C000F3E86B017C0120E030E040E850EC0E940E
:1048D000FCE187FD53C020E030E040E850E4C70130
:1048E000B6010E9476EA18160CF44FC0C0924C0B29
:1048F000D0924D0BE0924E0BF0924F0B8EE891E070
:104900000E94618582E0809353011092CE0510923F
:10491000CF051092D0051092D105809153018823C4
:1049200009F4A1CFC0904C0BD0904D0BE0904E0BF2
:10493000F0904F0B20E030E0A901C701B6010E94C2
:10494000FCE127E137EB41ED58E387FF04C027E1A5
:1049500037EB41ED58EBC701B6010E94F3E86983DC
:104960007A838B839C836BE2CE0101960E944391F4
:10497000BC0181E09EE00E948C2375CFC12CD12C1C
:1049800090E8E92E90ECF92EB1CFC12CD12C80E823
:10499000E82E80E4F82EAACF0F931F93CF93DF93D6
:1049A000FC01EB018091CE059091CF05A091D0053F
:1049B000B091D105B7FF08C01092CE051092CF0577
:1049C0001092D0051092D1058091D2059091D30517
:1049D000A091D405B091D5054091CE055091CF0559
:1049E0006091D0057091D10584179507A607B70788
:1049F00044F48093CE059093CF05A093D005B09357
:104A0000D105809153018823E1F06091CE0570912A
:104A1000CF058091D0059091D1050091D6051091D8
:104A2000D7052091D8053091D905600F711F821FDD
:104A3000931F0995BC018091DC059091DD050E94D2
:104A40008C238091C405811108C08091CB058823F7
:104A5000D1F1809153018823B1F18091DA059091D1
:104A6000DB050097B1F04091CE055091CF056091E4
:104A7000D0057091D1050091D6051091D7052091F0
:104A8000D8053091D905400F511F621F731FFE01D9
:104A90000995E091CC05F091CD05309741F08091DA
:104AA000CB05811103C08091C405811109958091C6
:104AB000C4051092C405882331F0DF91CF911F9176
:104AC0000F910C94861DDF91CF911F910F91089546
:104AD00062EA75E18BEB95E10C94CC246AEC75E10C
:104AE00083EE95E10C94CC2465E076E189E198E1D0
:104AF0000C94CC2468E176E187E897E10C94CC240F
:104B000063E376E189EC97E10C94CC2462EF75E1E4
:104B100088ED97E10C94CC246CE476E182E298E194
:104B20000C94CC248F929F92AF92BF92CF92DF923F
:104B3000EF92FF920F931F93CF93DF93CDB7DEB722
:104B40002C970FB6F894DEBF0FBECDBF982F862FDF
:104B50005A017901D02E692F0E94BE21882309F4C1
:104B600087C010914A03C701002381F10E940121EF
:104B7000C82E80904E1590904F15111143C01FEF15
:104B800023E12C194091E6055091E7056091E50578
:104B9000C5010E946622CC2009F46AC0B6E08B9F52
:104BA000500111246AE370E080E090E00E94F5215A
:104BB00057E0A516B10408F442C060E270E080E05E
:104BC00090E00E94F521A81AB90AF2CF0E946B1654
:104BD000C82E80904E1590904F15112381F2FE0142
:104BE00033968AE0DF011D928A95E9F78AE495E120
:104BF0009A83898301EF1AE19E012F5F3F4F48E6B8
:104C000056E112C0FE0133968AE0DF011D928A95BB
:104C1000E9F78AE495E19A83898301EF1AE19E011D
:104C20002F5F3F4F45E656E1B701C4010E9453B6DE
:104C3000B4018AE495E10E9442C61F81A1CF409150
:104C4000E405212F30E0A6E0CA9EC00111242E5FAA
:104C50003F4F281739070CF49C0180E8821B809392
:104C6000811540938215C701DD20A9F00E942623FB
:104C70002C960FB6F894DEBF0FBECDBFDF91CF915B
:104C80001F910F91FF90EF90DF90CF90BF90AF906A
:104C90009F908F9008950E948823EACF7F928F92F1
:104CA0009F92AF92BF92CF92DF92EF92FF920F93BB
:104CB0001F93CF93DF930E9495BDC091C70565E018
:104CC000862E8C0ED6E0DC1B85E0D82EDC1A84E024
:104CD000C82ECC1A83E0B82EBC1A82E0A82EAC1ADB
:104CE00081E0982E9C1A7C2E7194C11134C0809161
:104CF000C9058823B1F080915301882359F081E0E0
:104D00009091C905911180E024E04FE65DE0672DA8
:104D10000E9469BCCF5FC811E8CF87E08093C805C7
:104D20000CC08091C4051092C405882321F30E9411
:104D3000861D8091DE058823F1F2DF91CF911F91CE
:104D40000F91FF90EF90DF90CF90BF90AF909F902A
:104D50008F907F900895C130E9F58091C905813029
:104D6000E9F0809153018823A9F211E08091C905EF
:104D7000813009F010E06091200B7091210B80913F
:104D8000220B9091230B0E94961700E09C0147EEA6
:104D90005CE0692D812F0E949225BCCF8091C405D3
:104DA0001092C4058823E9F20E9416BDE12C1CE391
:104DB000F12E0CE116E420E030E040E85FE360E231
:104DC0007BE087EE9CE00E94EBBD8091DE058823AE
:104DD00041F2B3CFC23009F006C18091C9058230DB
:104DE000D9F080915301882309F494CF11E0809188
:104DF000C905823009F010E06091240B7091250BF9
:104E00008091260B9091270B0E94961700E09C0141
:104E100040EE5CE06A2DBECF8091C4051092C405BF
:104E20008823F9F20E9416BDE12C1CE3F12E0CE15F
:104E300016E420E030E040E85FE364E27BE080EEEF
:104E40009CE00E94EBBD8091DE05882351F275CF76
:104E50008091C9058330D9F080915301882309F4EA
:104E600059CF11E08091C905833009F010E06091BD
:104E7000280B7091290B80912A0B90912B0B0E948B
:104E8000961700E09C0149ED5CE06B2D83CF80918B
:104E9000C4051092C4058823F9F20E9416BDE12CC6
:104EA0001CE3F12E0CE116E420E030E040E85FE383
:104EB00068E27BE089ED9CE00E94EBBD8091DE051D
:104EC000882351F23ACF8091C9058430D9F080917E
:104ED0005301882309F41ECF11E08091C905843065
:104EE00009F010E060912C0B70912D0B80912E0B2E
:104EF00090912F0B0E94961700E09C0142ED5CE020
:104F00006C2D48CF8091C4051092C4058823F9F216
:104F10000E9416BDE12C1CE3F12E0CE116E420E00A
:104F200030E040E85FE36CE27BE082ED9CE00E94D1
:104F3000EBBD8091DE05882351F2FFCE8091C9053B
:104F40008530D9F080915301882309F4E3CE11E034
:104F50008091C905853009F010E060913C0B70919B
:104F60003D0B80913E0B90913F0B0E94961700E005
:104F70009C014DEC5CE06D2D0DCF8091C40510922D
:104F8000C4058823F9F20E9416BDE12C1CE3F12E22
:104F90000CE116E420E030E0A9016CE37BE08DEC4D
:104FA0009CE00E94EBBD8091DE05882359F2C5CEBE
:104FB0008091C4051092C405882329F10E9416BD72
:104FC000E12C1CE3F12E0CE116E420E030E0A90115
:104FD00060E47BE083EC9CE00E94EBBD8091DE0509
:104FE000882389F0AACEC33009F432CFC43009F443
:104FF0006ACFC53009F4A2CFC63009F08BCE8091BC
:10500000C9058630A9F280915301882309F482CE24
:1050100011E08091C905863009F010E06091400BE5
:105020007091410B8091420B9091430B0E94961717
:1050300000E09C0143EC5CE06D2FACCE2F923F92E0
:105040004F925F926F927F928F929F92AF92BF9298
:10505000CF92DF92EF92FF920F931F93CF93DF9344
:10506000CDB7DEB72C970FB6F894DEBF0FBECDBF1D
:10507000C090000BD090010BE090020BF090030B5E
:105080008091040B9091050BA091060BB091070B3A
:105090008C159D05AE05BF0510F4D701C601C09063
:1050A000FC0AD090FD0AE090FE0AF090FF0ABC01D5
:1050B000CD016C157D058E059F0510F4C701B60165
:1050C0000E9401E22B013C010E9495BD2091C70581
:1050D0002B872E83822F8B5F8D8387E0922F821BFD
:1050E0008F8386E0821B888785E0821B898784E026
:1050F000821B8A8783E0282E221A82E0382E321AF9
:1051000091959C872B85211142C08091C9058823E8
:10511000C9F080915301882359F081E09091C9052D
:10512000911180E024E04FE65DE06C850E9469BC4F
:105130008B858F5F8B879D819813E4CF88E0809368
:10514000C8050CC08091C4051092C405882309F3DA
:105150000E94861D8091DE058823D9F22C960FB619
:10516000F894DEBF0FBECDBFDF91CF911F910F919D
:10517000FF90EF90DF90CF90BF90AF909F908F9077
:105180007F906F905F904F903F902F9008958B8508
:10519000813009F089C08091C9058130F9F0809192
:1051A0005301882329F211E08091C905813009F06B
:1051B00010E06091300B7091310B8091320B909127
:1051C000330B0E94961761E02E81621B00E09C0168
:1051D0004DE15DE0812F0E949225AACF8091C40508
:1051E0001092C4058823D9F20E9416BD2AE037ED3B
:1051F00043E25DE3C301B2010E9462E220E030E0DD
:10520000A9010E94F3E84B015C0120E030E040E09E
:105210005FE40E94FCE187FD05C0812C912CA12C4C
:105220003FE4B32E2AE037ED43E25DE36091300BBB
:105230007091310B8091320B9091330B0E9462E29E
:1052400020E030E0A9010E94F3E820E030E040E8EF
:105250005FE30E94F2E80E94EFE969837A838B831F
:105260009C83C501B4010E94E8E97B018C0121E027
:10527000E21AF10801091109912C812C20E8A22ED3
:1052800025E2B22EC980DA8021E030E040E050E033
:1052900060E37BE08DE19DE00E9422BD8091DE0510
:1052A000882309F47CCF5ACF8B85823009F08EC1D8
:1052B0008091C9058230D9F080915301882309F487
:1052C00037CF11E08091C905823009F010E060917C
:1052D000340B7091350B8091360B9091370B0E94F7
:1052E000961700E09C0143E15DE0632D73CF809150
:1052F000C4051092C4058823F9F20E9416BD60917E
:10530000080B7091090B80910A0B90910B0B0E9476
:1053100001E27B018C0120E030E048EC52E464E3E0
:105320007BE083E19DE00E94EBBD8091DE05882358
:1053300019F214CF8091C9058330D9F080915301BF
:10534000882309F4F5CE11E08091C905833009F076
:1053500010E06091380B7091390B80913A0B90916D
:105360003B0B0E94961700E09C014AE05DE0622D35
:1053700031CF8091C4051092C4058823F9F20E94B0
:1053800016BD2AE037ED43E25DE3C301B2010E949E
:1053900062E220E030E0A9010E94F3E84B015C01E9
:1053A00020E030E040E05FE40E94FCE187FD05C0C2
:1053B000812C912CA12C9FE4B92E2AE037ED43E2F9
:1053C0005DE36091380B7091390B80913A0B9091AD
:1053D0003B0B0E9462E220E030E0A9010E94F3E86A
:1053E00020E030E040E85FE30E94F2E80E94EFE94D
:1053F00069837A838B839C83C501B4010E94E8E9A9
:105400007B018C0121E0E21AF10801091109912CBC
:10541000812C80E8A82E85E2B82EC980DA8021E0B0
:1054200030E040E050E068E37BE08AE09DE00E94ED
:1054300022BD8091DE05882309F480CF8FCE809134
:10544000C9058430E9F080915301882309F470CEB6
:1054500011E08091C905843009F010E06091FC0AE8
:105460007091FD0A8091FE0A9091FF0A0E9401E26C
:105470000E946E1700E09C0143E05DE06A85AACEC1
:105480008091C4051092C4058823E9F20E9416BDDC
:1054900000E618E124E630E040E050E06CEF7AE00E
:1054A00083E09DE00E9488BE8091DE05882359F24A
:1054B00055CE8091C9058530E9F08091530188234C
:1054C00009F436CE11E08091C905853009F010E06D
:1054D0006091000B7091010B8091020B9091030B76
:1054E0000E9401E20E946E1700E09C014CEF5CE01C
:1054F000698570CE8091C4051092C4058823E9F2B5
:105500000E9416BD0EE518E124E630E040E050E0D0
:1055100060E07BE08CEF9CE00E9488BE8091DE051D
:10552000882359F21BCE8091C9058630E9F080911D
:105530005301882309F4FCCD11E08091C905863020
:1055400009F010E06091040B7091050B8091060B3F
:105550009091070B0E9401E20E946E1700E09C01EF
:1055600045EF5CE0688536CE8091C4051092C40595
:105570008823E9F20E9416BD0CE518E12AE030E02C
:1055800040E050E064E07BE085EF9CE00E9488BE54
:105590008091DE05882359F2E1CD8091C4051092F7
:1055A000C405882339F10E9416BD0AE518E124E6F6
:1055B00030E040E050E068E07BE08EEE9CE00E944E
:1055C00088BE8091DE058823A9F0C8CD2B852330C5
:1055D00009F4B0CE243009F432CF253009F469CF74
:1055E000263009F4A0CF273009F0A2CD8091C9055B
:1055F000873099F280915301882309F499CD11E005
:105600008091C905873009F010E06091080B709116
:10561000090B80910A0B90910B0B0E9401E20E94F2
:105620006E1700E09C014EEE5CE06F81D3CD3F929F
:105630004F925F926F927F928F929F92AF92BF92A2
:10564000CF92DF92EF92FF920F931F93CF93DF934E
:105650000E9495BDC091C705A5E04A2E4C0ED4E02E
:10566000DC1B83E0782E7C1A82E0682E6C1A81E0C5
:10567000582E5C1A3C2E3194C11138C08091C90556
:105680008823B1F080915301882359F081E09091F3
:10569000C905911180E024E04FE65DE0632D0E9492
:1056A00069BCCF5FC411E8CF85E08093C8050CC00A
:1056B0008091C4051092C405882321F30E94861DA1
:1056C0008091DE058823F1F2DF91CF911F910F9138
:1056D000FF90EF90DF90CF90BF90AF909F908F9012
:1056E0007F906F905F904F903F900895C13009F088
:1056F0005BC08091C9058130E9F080915301882316
:1057000081F211E08091C905813009F010E06091CB
:105710000F067091100680911106909112060E945A
:10572000E11700E09C014BE35DE0652D812F0E94B5
:105730009225B7CF8091C4051092C4058823E9F261
:105740000E9416BD20E030E0A90160910F06709123
:10575000100680911106909112060E94F3E820E055
:1057600030E040E85FE30E94F2E80E94EFE9912C0C
:10577000812CE4E7AE2EE5E2BE2E6B011DEDE12E9D
:1057800013E0F12E00E010E021E030E040E050E0D6
:105790006FE076E08BE39DE00E9422BD8091DE0504
:1057A000882309F4AACF90CFC23009F0F8C08091C5
:1057B000C9058230D9F080915301882309F471CF53
:1057C00011E08091C905823009F010E06091130664
:1057D0007091140680911506909116060E94E117AB
:1057E00000E09C0143E35DE0662DA0CF8091C405FD
:1057F0001092C4058823F9F20E9416BD20E030E023
:10580000A90160911306709114068091150690917C
:1058100016060E94F3E820E030E040E85FE30E94D3
:10582000F2E80E94EFE9912C812C44E7A42E45E296
:10583000B42E6B011DEDE12E13E0F12E00E010E01F
:1058400021E030E040E050E063E176E083E39DE07A
:105850000E9422BD8091DE05882309F4ACCF34CFAD
:105860008091C9058330D9F080915301882309F4D0
:1058700018CF11E08091C905833009F010E06091E4
:105880001706709118068091190690911A060E94C9
:10589000241400E09C014BE25DE0672D47CF80912E
:1058A000C4051092C4058823F9F20E9416BD20E0B9
:1058B00030E048EC52E46091170670911806809130
:1058C000190690911A060E9462E220E030E0A901D8
:1058D0000E94F3E820E030E040E251E40E94F2E868
:1058E0000E94EFE9912C812C2EE6A22E25E2B22E09
:1058F0006B011EEAE12E12E8F12E01E010E02AE031
:1059000030E040E050E067E176E08BE29DE00E940D
:1059100022BD8091DE05882309F4A6CFD5CE8091E3
:10592000C4051092C405882309F444C00E9416BD22
:1059300020E030E048EC52E460911B0670911C06B8
:1059400080911D0690911E060E9462E220E030E0E8
:10595000A9010E94F3E820E030E040E251E40E9417
:10596000F2E80E94EFE9912C812C8EE6A82E85E2C8
:10597000B82E6B011EEAE12E12E8F12E01E010E0D4
:105980002AE030E040E050E06BE176E083E29DE029
:105990000E9422BD8091DE05882361F095CEC33040
:1059A00009F45ECFC43009F07CCE8091C905843003
:1059B00009F4B5CF80915301882309F472CE11E028
:1059C0008091C905843009F010E060911B06709148
:1059D0001C0680911D0690911E060E94241400E072
:1059E0009C0143E25DE06D2FA1CEBF92CF92DF928A
:1059F000EF92FF920F931F93CF93DF930E9495BD79
:105A0000C091C70585E0C82ECC0ED4E0DC1B13E0A6
:105A10001C1B82E0F82EFC1A81E0E82EEC1ABC2E4A
:105A2000B194C11130C08091C9058823B1F0809133
:105A30005301882359F081E09091C905911180E0CC
:105A400024E04FE65DE06B2D0E9469BCCF5FCC1176
:105A5000E8CF85E08093C8050CC08091C405109202
:105A6000C405882321F30E94861D8091DE058823CA
:105A7000F1F2DF91CF911F910F91FF90EF90DF90A6
:105A8000CF90BF900895C130B9F58091C90581309C
:105A9000F1F0809153018823C9F2DD24D3948091E1
:105AA000C905813009F0D12C6091100B7091110B58
:105AB0008091120B9091130B0E94DA1400E09C016C
:105AC00044E65DE06E2D8D2D0E949225BFCF809122
:105AD000C4051092C4058823E1F20E9416BD48E572
:105AE00058E160E17BE084E69DE00E9408BF809180
:105AF000DE05882371F2BDCFC23009F07FC08091EE
:105B0000C9058230E1F080915301882309F49ECFCA
:105B1000DD24D3948091C905823009F0D12C6091A5
:105B2000140B7091150B8091160B9091170B0E941E
:105B3000DA1400E09C0149E55DE06F2DC4CF80914F
:105B4000C4051092C4058823F1F20E9416BD46E5F3
:105B500058E164E17BE089E59DE00E9408BF809107
:105B6000DE05882381F285CF8091C9058330E1F07D
:105B700080915301882309F469CFDD24D394809167
:105B8000C905833009F0D12C6091180B7091190B65
:105B900080911A0B90911B0B0E94DA1400E09C017B
:105BA0004EE45DE0612F8FCF8091C4051092C40553
:105BB0008823F1F20E9416BD44E558E168E17BE0DC
:105BC0008EE49DE00E9408BF8091DE05882381F26B
:105BD00050CF8091C4051092C4058823C9F00E945B
:105BE00016BD42E558E16CE17BE083E49DE00E9454
:105BF00008BF8091DE05882359F03BCFC33009F4FC
:105C0000B3CFC43009F022CF8091C905843009F3A5
:105C100080915301882309F419CFDD24D394809116
:105C2000C905843009F0D12C60911C0B70911D0BBB
:105C300080911E0B90911F0B0E94DA1400E09C01D2
:105C400043E45DE06D2F3FCF2F923F924F925F92E2
:105C50006F927F928F929F92AF92BF92CF92DF927C
:105C6000EF92FF920F931F93CF93DF930E9495BD06
:105C7000C091C70535E0432E4C0E43E0342E57E368
:105C8000652E5FE5752ED1E0DC1B2C2E219482E081
:105C9000582E5C1AC11141C08091C9058823F1F0CA
:105CA00080915301882359F081E09091C9059111A9
:105CB00080E024E04FE65DE0622D0E9469BC8091A7
:105CC0000604882309F4C3C0C23009F45CC083E031
:105CD000CF5FC411DFCF8093C8050CC08091C4058D
:105CE0001092C4058823E1F20E94861D8091DE0592
:105CF0008823B1F2DF91CF911F910F91FF90EF9028
:105D0000DF90CF90BF90AF909F908F907F906F90DB
:105D10005F904F903F902F900895C13081F6809111
:105D2000C9058130C9F080915301882341F281E097
:105D30009091C905913009F080E09091060426EB1E
:105D40003CE0911102C022EB3CE001E049EB5CE059
:105D50006D2F0E949225B3CF809106049091C405C7
:105D60001092C4059923F9F28C278093060430928F
:105D700053016114710411F00E94375F8091DE05B8
:105D8000882389F2B7CF8091C9058230F1F08091E4
:105D90005301882309F49BCF11E08091C90582301B
:105DA00009F010E0609102047091030480910404F2
:105DB000909105040E94C79400E09C0148EA5CE0D1
:105DC000652D812F0E94922582CF8091C40510926B
:105DD000C4058823E1F20E9416BD20E030E04AE7C6
:105DE00054E4609102047091030480910404909142
:105DF00005040E9462E220E030E0A9010E94F3E87D
:105E000020E030E84BEB54E40E94F2E80E94EFE916
:105E100087E3882E8FE5982E9CE8A92E95E2B92E6F
:105E20006B0116EDE12E16E0F12E00E010E02CEDF6
:105E300035E040E050E062E074E088EA9CE00E94D7
:105E400022BD8091DE05882309F4A1CF53CF82E0E3
:105E50003FCFE6E4F5E183AF64AFCA010C94882339
:105E60000F931F93CF9310924203109241032FE39D
:105E70002093470310924603109245039C01F901B9
:105E800090812F5F3F4F9032D1F39E34C9F48181CE
:105E900090ED980F9A3020F08D3211F08B3281F412
:105EA00032969F012F5F3F4F808180538A3008F4E4
:105EB00068C09F012F5F3F4F8081803209F463C02B
:105EC000F093F205E093F1058F010F5F1F4FC08142
:105ED0006AE270E0C8010E9443EB009731F0FC01D8
:105EE000319780818032E1F31182CD3429F0C435BD
:105EF00019F0C73409F041C0F80180810F5F1F4FCE
:105F00008032D1F380538A30C0F5C093470330E02C
:105F100020E06AE0AF014F5F5F4F629FC001639F67
:105F2000900D11249C01205331098081280F311DCF
:105F300087FD3A95FA01808180538A3058F3309377
:105F4000460320934503CA01FC010196408140327B
:105F5000D9F3F0934403E0934303CD3401F52E319C
:105F6000310539F090F42731310519F02C31310524
:105F7000B1F4F0934203E0934103CF911F910F914D
:105F80000895F9018ECFF90194CF2537310538F006
:105F90002737310570F3203A83E0380751F350E09A
:105FA00040E0CF0101966081662309F45AC0613256
:105FB00091F4CD3481F42032310569F49093420399
:105FC0008093410363E270E00E9443EB0097A9F2E3
:105FD000FC011082D2CFFC01DF018D91803271F083
:105FE00090ED980F9A3008F18E3251F491819053D0
:105FF0009A30D8F041155105E1F414C0FD01ECCF01
:106000008D3211F08B3259F4918160ED690F6A3055
:1060100060F09E3221F4928190539A3030F0411515
:10602000510519F4AF014150510981548A3108F4E6
:10603000B8CFDF01FD018D91882309F4B2CF90ED37
:10604000980F9A30B8F393ED980F923098F38B3203
:1060500089F3CF0101966081603209F0A2CFFC0183
:10606000F8CF509342034093410387CF0E94661CB0
:1060700097FD0CC00E94661C6F3F7105810591055C
:1060800009F034F40E94661C862F089580E008957C
:106090008FEF08958091340390913503892B41F05F
:1060A0000E94363091E0811101C090E0892F08955F
:1060B00091E0FCCF0E94251C882341F081E02091D3
:1060C000340330913503232B09F480E00895CF93F6
:1060D000DF93EB010E945A30882319F00E94661C5E
:1060E000EB01CE01DF91CF910895CF93DF93C82FBD
:1060F000D62F0E945A30882321F0DF91CF910C9443
:106100004A308C2F0E94251C811101C08D2FDF91F8
:10611000CF91089510926B0410926C0410926D044C
:1061200010926E04E7E0F4E084E6DF011D928A95A8
:10613000E9F70895909101049817B1F00E949E77B5
:1061400080910104882341F084E49BE00E94D7778A
:10615000109201040C94538681E08093010484E43E
:106160009BE00E94BF77F6CF08959091010481E0F3
:1061700089270C949A30EF92FF920F931F93CF933D
:10618000DF9307E014E0C5E07801D5E0F701619105
:106190007191819191917F0120E030E0A9010E94ED
:1061A000FCE181110EC0D15089F7C1500C5E1F4F28
:1061B000C111EACFDF91CF911F910F91FF90EF9026
:1061C000089581E0F7CFEFE6F0E080818260808380
:1061D00008954F925F926F927F928F929F92AF92AB
:1061E000BF92CF92DF92EF92FF920F931F93CF93C4
:1061F000DF9300D000D0CDB7DEB70E9482C14B0143
:106200005C01809119018F3F09F441C00E9482C155
:10621000C0907A03D0907B03E0907C03F0907D03E4
:106220006C197D098E099F0997FD31C080911E155B
:1062300090911F158F5F8F70891749F1E0911901B7
:1062400080E090E0A8E4B3E4E43050F424E0E29F7E
:10625000F0011124EA58FE4F80819181A281B3811F
:1062600089839A83AB83BC83C12CD12C76018E01A8
:106270000F5F1F4F20E53BE04CE45BE068E47BE010
:1062800084E49BE00E9439B98FEF809319010E944A
:10629000F21F80918C0382FF33C0809189038111AA
:1062A00031C091E090938903809191038927809375
:1062B000C4051092910383E08093530110928C03E4
:1062C0000E9482C16C507E4F8F4F9F4F60938D0311
:1062D00070938E0380938F039093900368E873E12B
:1062E00082E090E00E949A9416E0115059F00E94CA
:1062F0003E9462E070E080E090E00E94E7C0F5CF5D
:10630000109289038091850390918603A091870361
:10631000B0918803A5019401281B390B4A0B5B0B34
:10632000DA01C901B7FF05C08091D403882309F4BD
:10633000C6C1D501C4018C599F4FAF4FBF4F809349
:10634000850390938603A0938703B093880360919D
:106350008A03062E000C770B77FF03C071956195B9
:10636000710990918A0380918403981365C063300A
:1063700008F062C010928A0380918A03809384039C
:10638000643008F069C08091C4058111E7C0809134
:106390004415909145158450944341F480911A011D
:1063A000882309F4EDC0815080931A010E94C579B9
:1063B000C0903306D0903406E0903506F090360653
:1063C00081110E94E330D701C6013AE0B695A79546
:1063D000979587953A95D1F7009741E0A407B105C5
:1063E00020F08FEF9FEFA0E0B0E096958795209189
:1063F00053012111D7C03091D40331118EC1809146
:106400004415909145158450944309F46DC18091D1
:10641000C605811169C18091800390918103A0918B
:106420008203B0918303881A990AAA0ABB0AB7FCAF
:1064300069C10E946D1D66C1633009F09DCF8091D6
:106440008A0387FD07C081E0880F880F80938A0345
:1064500064E092CF8FEFF8CF8091E30521E030E048
:1064600040E050E0882309F456C0C090DF05D0908A
:10647000E005E090E105F090E205C114D104E104EB
:10648000F104E9F170E090E080E00E9401E220E098
:1064900030E040E85EE30E9462E22B013C01C5016E
:1064A000B4016C197D098E099F090E9401E29B01CC
:1064B000AC01C301B2010E9476E920E030E04AE776
:1064C00054E40E9462E26B017C0120E030E042E093
:1064D00053E40E9476EA24E630E040E050E087FF93
:1064E00012C020E030E040EA52E4C701B6010E9449
:1064F00076EA2AE030E040E050E087FF04C021E087
:1065000030E040E050E08092DF059092E005A092FC
:10651000E105B092E205A0918A030A2E000CBB0BA4
:106520000E94EAE824E030E040E050E00E94C2E847
:106530008091CE059091CF05A091D005B091D10565
:10654000820F931FA41FB51F8093CE059093CF0594
:10655000A093D005B093D10510928A03D501C40150
:106560008856954CAF4FBF4F809380039093810323
:10657000A0938203B093830381E08093530107CFFC
:106580008CE080931A0180917E0390917F030097A5
:1065900029F0019790937F0380937E0381E080939D
:1065A000530104CF009741F040917E0350917F0347
:1065B0004817590708F023CF8091D40381111DC0DB
:1065C000223038F0243008F44CC0243011F41092FA
:1065D000530180918315811105C081E0809383155B
:1065E0000E94CBC280914C1590914D150E94A4C27F
:1065F00081E08093CA058093D40383E00E94E01A6F
:1066000081E080936A15E0914415F0914515099554
:106610001092CA058091D403811127C01092C4053D
:1066200080914415909145158450944309F0EFCE24
:106630000E9482C1DC01CB0188199909AA09BB0912
:10664000C0907E03D0907F03F12CE12CC816D906B0
:10665000EA06FB0608F0D3CE90937F0380937E0377
:10666000CECE81E080935301B4CF8AE495E10E94BD
:1066700010C691E0811101C090E09093D40388236B
:1066800069F2809144159091451584509443B9F472
:106690000E9482C1DC01CB0188199909AA09BB09B2
:1066A000C0907E03D0907F03F12CE12CC816D90650
:1066B000EA06FB0620F490937F0380937E030F90FD
:1066C0000F900F900F90DF91CF911F910F91FF903E
:1066D000EF90DF90CF90BF90AF909F908F907F9082
:1066E0006F905F904F90089548E9840E4AE3941E9E
:1066F000A11CB11C8092800390928103A09282031E
:10670000B09283038091D4038111D9CF809153013A
:106710008130A9F610925301D2CF009709F46DCFC2
:1067200043CF8091EC059091ED05892B79F4809110
:10673000EC059091ED05892B49F42091EC05309101
:10674000ED0581E0232B19F480E0089581E00895A0
:10675000CF92DF92EF92FF926B017C0183E3C81628
:10676000D104E104F10470F082E3C81AD108E10811
:10677000F10862E370E080E090E00E94E7C00E94D0
:106780005586ECCFC701B6010E94E7C0FF90EF909D
:10679000DF90CF900C9455865E9A809194058E7F01
:1067A000809394055E9A809194058D7F80939405E3
:1067B000159A809194058B7F809394055E9A089535
:1067C0009091C61693FB882780F993FF06C081E05D
:1067D0009091BB14911101C080E008950E94B7BA56
:1067E0000E94E033882351F08091C61682FD06C0D6
:1067F00084EA9CE09093A2058093A1058DE99CE03A
:106800000E9480B50C9487904F925F926F927F9216
:106810008F929F92AF92BF92CF92DF92EF92FF92B0
:106820000F931F93CF93DF9300D000D01F92CDB76B
:10683000DEB71092E3058091C4051092C405882349
:10684000E9F020E040E070E060E082E99AE90F9032
:106850000F900F900F900F90DF91CF911F910F919C
:10686000FF90EF90DF90CF90BF90AF909F908F9070
:106870007F906F905F904F900C94B21C20911F01FD
:10688000309120014091CE055091CF05CA01820F71
:10689000931F2436310509F015C44730510544F0E3
:1068A00006978A3091050CF01CC48AE090E023C45E
:1068B00006964A3F5F4FACF38091CA05882309F4DE
:1068C000C0C120910106309102064091030650910B
:1068D00004066091440B7091450B8091460B90919A
:1068E000470B0E94F3E84B015C01209105063091B3
:1068F000060640910706509108066091480B70917A
:10690000490B80914A0B90914B0B0E94F3E86983ED
:106910007A838B839C832091090630910A064091EB
:106920000B0650910C0660914C0B70914D0B8091B1
:106930004E0B90914F0B0E94F3E82B013C0120E09D
:1069400030E040E251E40E9462E220E030E048ECB6
:1069500052E40E9462E26B017C0120E030E0A90178
:10696000C301B2010E94FCE120E030E040EA50ECBB
:1069700087FD04C020E030E040EA50E4C701B601E2
:106980000E94F3E820E030E040E251E40E9476E922
:106990000E94E8E92B013C0180E277FE09C0709477
:1069A000609450944094411C511C611C711C8DE2F8
:1069B0008093D50360E2F0E14F16F7E25F066104D1
:1069C00071048CF0C301B20120E137E240E050E0F5
:1069D0000E94C2E8CA01B9012AE030E040E050E07C
:1069E0000E94C2E8605D6093D60360E228EE421622
:1069F00023E05206610471048CF0C301B20128EE59
:106A000033E040E050E00E94C2E8CA01B9012AE048
:106A100030E040E050E00E94C2E8605D6093D70340
:106A2000C301B20124E630E040E050E00E94C2E839
:106A30006AE0C62ED12CE12CF12CCA01B901A701C4
:106A400096010E94C2E8605D6093D803C301B20161
:106A5000A70196010E94C2E86D83CA01B901A7018E
:106A600096010E94C2E8CD80CC2009F454C38EE286
:106A70008093D903605D6093DA032C2D205D209311
:106A8000DB0365ED73E082E793E00E944EEB20E0CC
:106A900030E0A901C501B4010E94FCE120E030E032
:106AA00040E05FEB87FD04C020E030E040E05FE3C2
:106AB000C501B4010E94F3E80E94E8E9CB010E94FD
:106AC000DF91BC018DE693E00E944EEB20E030E0C8
:106AD000A90169817A818B819C810E94FCE120E07F
:106AE00030E040E05FEB87FD04C020E030E040E0B4
:106AF0005FE369817A818B819C810E94F3E80E9427
:106B0000E8E9CB010E94DF91BC0188E693E00E9496
:106B10004EEB4091CA034F774983411127C00E9431
:106B2000E033882319F18091BE169091BF16A09191
:106B3000C016B091C1160097A105B105B9F0BC010E
:106B4000CD016D597F4F8F4F9F4F24E630E040E0DD
:106B500050E00E9444E86091C2167091C316809183
:106B6000C4169091C5160E9444E829830E943A9069
:106B7000B62E872E982EA92E6D8380911801C9807C
:106B80008C15C1F0C092180128E4C29EB0011124F6
:106B900090E080E00E9401E22AE037ED43E25CE30E
:106BA0000E9462E20E94EFE960936703C110C5C2D0
:106BB0001092620380911701CD80C81609F441C07C
:106BC000B09217016B2D782D892D9A2D20E13EE092
:106BD00040E050E00E9444E869012CE3422E512C31
:106BE000612C712C6B2D782D892D9A2DA30192018A
:106BF0000E9444E8CA01B901A30192010E9444E83D
:106C000024E6C216D10408F0BFC27F936F93DF92CF
:106C1000CF9280ED9BE09F938F9382E593E09F93CB
:106C20008F930E9493E10FB6F894DEBF0FBECDBFE5
:106C300085E0982F990F990F891B880F80588093B2
:106C400051030E9482C100914D0310914E03209187
:106C50004F03309150036B017C01C01AD10AE20A44
:106C6000F30A9701860137FD11C020914C0320954E
:106C700020934C036A547C4F8F4F9F4F60934D037A
:106C800070934E0380934F0390935003D0904C0326
:106C9000D98281E00E94E01A80917E15843158F4F7
:106CA00080918015883038F025E53CE04CE068E0C4
:106CB00080E50E9443C380917E158431A0F48091C9
:106CC0008015823080F0E980EE2031F08091370627
:106CD0002FE13CE0811102C029EE3BE042E162E09D
:106CE00088E60E9443C380917E158C3108F0D0C0A5
:106CF000E090A514F090A614883028F58091A71490
:106D00009091A8140E945E92FC01808193E08032F1
:106D100029F4818192E0803209F491E043E050E06F
:106D2000491B51094E0F5F1F892F880F880F981B31
:106D3000892F67E0815F0E94292F69E070E080E081
:106D400090E00E94F52180917E158C3130F5809184
:106D50008015843110F1C7010E945E92FC01808190
:106D600093E0803229F4818192E0803209F491E04D
:106D700043E050E0491B51094E0F5F1F892F880FD8
:106D8000880F981B892F6CE1815F0E94292F69E091
:106D900070E080E090E00E94F521E090A905F0907D
:106DA000AA0580917E15883028F58091AB059091D9
:106DB000AC050E945E92FC01808193E0803229F450
:106DC000818192E0803209F491E043E050E0491B78
:106DD00051094E0F5F1F892F880F880F981B892F2D
:106DE00067E0865A0E94292F69E070E080E090E019
:106DF0000E94F52180917E158C3130F580918015AF
:106E0000843110F1C7010E945E92FC01808193E001
:106E1000803229F4818192E0803209F491E043E0EC
:106E200050E0491B51094E0F5F1F892F880F880FB3
:106E3000981B892F6CE1865A0E94292F69E070E027
:106E400080E090E00E94F52180917E158C3100F564
:106E5000809180158431E0F0809137068823C1F05D
:106E600024E6829FC001112481589F4F6FEF70E08C
:106E70000E94AEE8CB010E945E92AC016CE187E615
:106E80000E94292F65E270E080E090E00E94F521E9
:106E90000E94E033882369F180917E15843348F5A0
:106EA000809180158A3228F107E028E04AE26AE200
:106EB0008AE495E10E944CC405E022E04CE262E3E2
:106EC0008AE495E10E944CC46AE08AE20E9405C40B
:106ED00060914C1570914D1582E3809366158BE29D
:106EE0008093671526E635E142E38AE495E10E9446
:106EF000A0C280917E15853340F480918015813346
:106F000020F06AE486E30E9405C480917E158433F4
:106F100068F480918015823348F002E02091670385
:106F200042E367E38AE495E10E944CC480917E15B8
:106F30008033D8F4809180158832B8F08091620354
:106F4000882361F042E653E060E387E30E94292F43
:106F500065E270E080E090E00E94F52142E553E0B8
:106F600060E3809151030E94292F80917E15873222
:106F700008F055C0809180158F3108F450C083E02F
:106F80008093811546E24093821568E570E080E0C9
:106F900090E00E94F5218BE08093811566E260937A
:106FA0008215C980CC2009F404C18DE693E00E94CB
:106FB000882388E280938115F6E2F093821569E5D3
:106FC00070E080E090E00E94F52180E380938115DD
:106FD00096E2C92EC0928215D980DD2009F40AC13B
:106FE00088E693E00E9488238DE480938115F6E281
:106FF000F09382156AE570E080E090E00E94F52150
:1070000085E58093811586E2C82EC0928215D980CD
:10701000DD2009F412C182E793E00E948823809169
:107020007E15833338F5809180158B3218F183E01B
:107030000E94E01A83E08093811583E38093821598
:1070400066E070E080E090E00E94F52181E00E941F
:10705000E01A80911F01909120010E945E92AC0184
:1070600063E38CE00E94292F65E270E080E090E00D
:107070000E94F52180917E15813408F007C180912E
:107080008015863308F402C1109281158EE3809337
:1070900082158BE692E10E946B16898360E870E0AE
:1070A0008BE692E10E942A23F981F53108F0EEC0C7
:1070B00060E270E080E090E00E94F52129812F5F7E
:1070C0002983F2CF243631054CF48536910504F539
:1070D0008A30910534F48AE090E009C08436910545
:1070E000BCF0883EE3E09E0714F087EE93E028179B
:1070F000390709F4E1CB9093200180931F0110928E
:10710000CE051092CF051092D0051092D105D4CBA8
:1071100084E690E0F0CF662351F08EE28093D903AD
:10712000605D6093DA0380E28093DB03AACC80E2A7
:107130008093DA038093D903F6CF498180E2443605
:1071400028F0842F64E60E9480E8805D8093D90354
:10715000698190E26A3040F02AE0862F622F0E9417
:1071600080E80E9480E8905D9093DA0389816AE06C
:107170000E9480E8905D9093DB0369ED73E082E606
:1071800093E00E944EEB16CD7F936F93DF92CF92E8
:1071900086EC9BE09F938F9382E593E09F938F9380
:1071A0000E9493E10FB6F894DEBF0FBECDBF86E01C
:1071B00040CD87E00E944B8580FF13C00DE613E0B1
:1071C000F80161918F01662309F4F3CE6F320CF060
:1071D0006FE3062E000C770B880B990B0E94F521AC
:1071E000EFCF8091940580FDE0CE84EE9BE00E947D
:1071F0002623DFCE87E00E944B85869580FF13C053
:1072000008E613E0F80161918F01662309F4ECCEE2
:107210006F320CF06FE3062E000C770B880B990B86
:107220000E94F521EFCF80919405869580FDD8CE00
:1072300084EE9BE00E942623D7CE87E00E944B85F8
:107240008695869580FF17C082E793E09A838983AD
:10725000E981FA816191FA83E983662309F4DFCE3B
:107260006F320CF06FE3062E000C770B880B990B36
:107270000E94F521EDCF809194058695869580FD3D
:10728000CACE8CED9BE00E942623C9CE0F900F90B2
:107290000F900F900F90DF91CF911F910F91FF9062
:1072A000EF90DF90CF90BF90AF909F908F907F90A6
:1072B0006F905F904F9008950E94E033882339F0DB
:1072C0008091C61682FB882780F991E0892708956E
:1072D00081E008959091C00095FFFCCF8093C60097
:1072E0000895CF93DF93EC018991882319F00E94D0
:1072F0006A39FACF8DE00E946A398AE0DF91CF9136
:107300000C946A39CF93DF93EC01FE0184912196AE
:10731000882319F00E946A39F8CFDF91CF91089540
:10732000E0913E0C81E6E89FF0011124E056F34F16
:107330008081811107C084ED95E20E9482398AE044
:107340000C946A3908950E946A3989E394E00C9498
:107350008239AF92BF92CF92DF92EF92FF920F935A
:107360001F93CF93DF9384E294E00E94823960916F
:107370006B0470916C0480916D0490916E0445E0F3
:107380000E948F7081E194E00E948239C0E0D9E0D0
:10739000D15021F080E20E946A39FACF8C2F0E94EE
:1073A00094C7CF5FC53099F78AE00E946A3907E039
:1073B00014E0C0E080E20E946A398C2F0E9494C7DA
:1073C0005801D5E080E20E946A39F501C080D18081
:1073D000E280F380A7019601C701B6010E94F4EA9A
:1073E00081112CC020E030E0A901C701B6010E9444
:1073F00076EA87FD03C08BE20E946A3945E0C70147
:10740000B6010E948F70D15084E1A80EB11CD11139
:10741000D9CF8AE00E946A39CF5F0C5F1F4FC53019
:1074200049F68AE0DF91CF911F910F91FF90EF9085
:10743000DF90CF90BF90AF900C946A39F12C80E22E
:107440000E946A39F3948DE3F8E0FF12F9CFDBCFA5
:10745000CF92DF92EF92FF926A017B010E94823904
:1074600042E0C701B601FF90EF90DF90CF900C94FF
:107470008F70CF93DF93EB010E948239CE01DF91B1
:10748000CF910C9430B78AE094E00C94823984E078
:1074900094E00C948239CF9384E50E945A30C0E086
:1074A0008823D9F00E943630C82F1816B4F40E94F1
:1074B000473A8DE40E946A398091450390914603D2
:1074C0000E949BC76C2FCC0F770B8EE395E00E9438
:1074D000393A8AE00E946A39CFEF8C2FCF91089514
:1074E000EC018B01F42E0E94E0710E94433A84EE7D
:1074F00093E00E9482390115110511F408E516E2A6
:10750000209711F4CBEDD3E00E9479201F930F93C5
:10751000DF93CF938BEC93E09F938F93D1E0DF9336
:107520000E945E1F0E946D1DC0914B15C695C695A9
:107530008DB79EB707960FB6F8949EBF0FBE8DBF4E
:1075400080918315811104C0D09383150E94CBC212
:1075500080914C1590914D150E94A4C2DC2FDD0F37
:107560001D2F1C0F83E00E94E01A4BE652E16C2FA6
:1075700080E00E94292F10928115D09382158CEB08
:1075800093E00E94262310928115109382158FEAB2
:1075900093E00E9426238AE495E10E9410C681119F
:1075A000E1CF82ED93E00E9480B589EE93E030E672
:1075B000019729F0232F2A950000E9F7F9CFF894D5
:1075C00089EE93E038EE019729F0232F2A950000E9
:1075D000E9F7F9CF0E94E071FF2021F00E94CC333F
:1075E000A895FECF5E9AFCCF8091540B9091550BDD
:1075F0002FEF3FEF981751F0E92FF0E0EC5AF44FDE
:10760000228130E09F5F9F779093550BC9010895C9
:107610001F920F920FB60F9211240F900FBE0F9072
:107620001F9018951F920F920FB60F9211240BB650
:107630000F922F933F934F935F938F939F93EF936B
:10764000FF938091C6004091550B9091540B31E00F
:10765000390F3F77209121032C3008F072C0E22FC0
:10766000F0E0EB5CF44C0C94E1E8413B683B773B89
:10767000823B893BA13B8D3BA13B913B953BA13B91
:10768000993B803229F0E8F48A3011F08D30F1F422
:10769000431731F0E92FF0E0EC5AF44F8283932F37
:1076A0009093540BFF91EF919F918F915F914F9128
:1076B0003F912F910F900BBE0F900FBE0F901F9018
:1076C00018958D3481F021E08E3471F02BE00CC0E0
:1076D0008A3338F48033E0F68032D1F28D32B1F75C
:1076E000D7CF8D3499F722E020932103D1CF813376
:1076F00029F0843329F0803249F7CACF23E0F4CF50
:1077000028E0F2CF24E0803379F326E0813361F37F
:10771000DDCF25E08833D1F6E7CF27E08233B1F61D
:10772000E3CF29E0813391F6DFCF2AE0803371F691
:10773000DBCF8A3019F08D3009F0AACF10922103E7
:10774000A7CF8A3019F08D3009F0A2CF509184155F
:107750005523A1F3273049F02A3059F0253071F72D
:107760001092520110929103E9CF21E0209371040D
:10777000E5CF21E020937004E1CF8EBD0DB407FE6C
:10778000FDCF08958FEF8EBD0DB407FEFDCF8EB5F2
:107790000895909164009B7F90936400982F906A65
:1077A00096959CBD80FD03C091E0863009F490E081
:1077B0009DBD0895CF92DF92EF92FF92CF936B0120
:1077C0007C01C42F4A3069F4F7FE0BC0F094E094BA
:1077D000D094C094C11CD11CE11CF11C8DE20E940C
:1077E0006A394C2FC701B601CF91FF90EF90DF901F
:1077F000CF900C942DC7CF92DF92EF92FF926A0147
:107800007B010E9482394AE0C701B601FF90EF90E8
:10781000DF90CF900C94DA3B2F923F924F925F9281
:107820006F927F928F929F92AF92BF92CF92DF9290
:10783000EF92FF920F931F93CF93DF93CDB7DEB7F5
:10784000EB970FB6F894DEBF0FBECDBF85E40E9464
:107850005A30882321F00E94761C811183C283E56F
:107860000E945A30882309F45EC00E94761C9A83D5
:10787000898383E40E945A30A5E07A2E882319F088
:107880000E94761C782E60E085E50E9475308FABF3
:1078900060E08BE49BE00E94771F49815A81BA0126
:1078A000550F880B990B0E9403E2162F7D838E8360
:1078B000292E0E9482C16B877C878D879E8760916D
:1078C0005001709151016F507109072E000C880B07
:1078D000990B0E9403E29B01AC01612F7D818E8197
:1078E000922D0E9476EA18161CF58CEF9AE00E9401
:1078F0008239EB960FB6F894DEBF0FBECDBFDF9195
:10790000CF911F910F91FF90EF90DF90CF90BF909C
:10791000AF909F908F907F906F905F904F903F902F
:107920002F900C94B7BA24EB30E03A832983A1CF8F
:107930008B859C85AD85BE85805B9C43AF4FBF4FDB
:107940008BAB9CABADABBEAB88EE9AE00E948239AC
:107950000E94E0718FE78093A91481E08093520127
:107960008B849C84AD84BE848AA69BA6ACA6BDA64F
:107970001C8E1D8E1E8E1F8E18A219A21AA21BA26B
:1079800019821A821B821C822FE730E040E050E00F
:107990002F87388B498B5A8B1F8230E43D8B4CE10B
:1079A0004E8B56E45F8B188E198E1A8E1B8EFFE756
:1079B000CF2ED12CE12CF12C1EA61FA618AA19AA95
:1079C0001AAA1DA21EA21FA218A68CA31C8A1B8A7B
:1079D000312C00E01AAE1BAEA72D770CBB0BB9AF54
:1079E000A8AF80915201882309F48BC00E9482C104
:1079F0002B013C01B0917204B9A7BB2309F46BC001
:107A00000E9493726091A5147091A614072E000C29
:107A1000880B990B0E9403E2362E072F8AAF9BAF8B
:107A2000288D398D4A8D5B8D0E9476EA181634F4C4
:107A3000388E098F2AAD2A8F3BAD3B8F2F813D8930
:107A40004E895F89632D702F8AAD9BAD0E94FCE14A
:107A500087FF06C03F820D8B4AAD4E8B5BAD5F8BBF
:107A60008CA1232D302F4AAD5BAD612F7D81882302
:107A700009F494C18E81922D0E94FCE187FF2BC0F6
:107A8000B301A201481959096A097B09DB01CA013E
:107A900088589341A109B109B7FD1DC08F85988908
:107AA000A989BA898C199D09AE09BF09B595A79511
:107AB000979587958093A9144DA35EA36FA378A78C
:107AC000188F9D81998FAE81AA8F2B8E4B865C86F5
:107AD0006D867E861CA220E030E040EF51E4612FED
:107AE0007D818E81922D0E94F3E8232D302F4AADA7
:107AF0005BAD0E94FCE187FF22C085E79AE00E940F
:107B00008239109252010E94E071F3CE4BEEC42EE6
:107B1000D12CE12CF12C95C184E190E0A0E0B0E003
:107B20008F87988BA98BBA8B34E1C32ED12CE12C93
:107B3000F12C95C1CF86D88AE98AFA8A90C1D301FF
:107B4000C2012AA53BA54CA55DA5821B930BA40BE6
:107B5000B50BB7FD4CC080E00E9433718AE00E94F3
:107B60006A39D301C2018053984FAF4FBF4F8AA7E4
:107B70009BA7ACA7BDA79EA5911167C02FA538A94B
:107B800049A95AA9632D702F8AAD9BAD0E9476EA50
:107B900018160CF046C020E030E040E050E4632DC1
:107BA000702F8AAD9BAD0E94F3E86FA778AB89ABCD
:107BB0009AABA3019201205B3C434F4F5F4F2BAB2D
:107BC0003CAB4DAB5EAB20E030E040EC50E4612FCD
:107BD0007D818E81922D0E94F2E8232D302F4AADB7
:107BE0005BAD0E94FCE1881F8827881F8EA78B85CC
:107BF0009C85AD85BE8588169906AA06BB0610F43D
:107C0000D501C401481A590A6A0A7B0A31E84316A9
:107C10003FE4530632E16306710480F187E59AE0A0
:107C20006ECFD301C2012BA93CA94DA95EA9821B2D
:107C3000930BA40BB50B44EB51E263EC71E2B7FD7F
:107C4000D6CF80E00E94AB72D2CF20E030E040EF90
:107C500051E4612F7D818E81922D0E94F2E89B017B
:107C6000AC01632D702F8AAD9BAD0E94FCE187FFB4
:107C7000BECF40E652E260E772E2E3CF48AD59ADD5
:107C80008B899C89481759070CF069C003970CF43D
:107C900066C08AEF99E00E9482398DED99E00E94DA
:107CA000823949815A816B817C8186EF99E00E94FB
:107CB000283A8AE00E946A398DED99E00E94823963
:107CC00048A159A16AA17BA182EF99E00E94283ABC
:107CD0008AE00E946A398DED99E00E9482394C8DCC
:107CE0005D8D6E8D7F8D8EEE99E00E94283A8AE040
:107CF0000E946A399FA9992309F4FBCD29813A8111
:107D00004B815C812093AA143093AB144093AC1444
:107D10005093AD142CEA35EC47E25EE368A179A1FB
:107D20008AA19BA10E9462E26093AE147093AF148B
:107D30008093B0149093B1142CEA35EC47E25EE3E3
:107D40006C8D7D8D8E8D9F8D0E9476E96093B2142F
:107D50007093B3148093B4149093B514CACD0E9459
:107D6000E9303FCE87E29BE0EB960FB6F894DEBF9A
:107D70000FBECDBFDF91CF911F910F91FF90EF907C
:107D8000DF90CF90BF90AF909F908F907F906F903B
:107D90005F904F903F902F900C9482398E81922D5E
:107DA0000E9476EA18160CF096CED301C2012B85FC
:107DB0003C854D855E85821B930BA40BB50BAC01F6
:107DC000BD01485853416109710977FD84CE4B8943
:107DD0005C89452B09F4FEC08DA09EA0AFA0B8A47D
:107DE000880E991EAA1EBB1E2DA13EA14FA158A50B
:107DF000281B390B4A0B5B0BC701B6010E9434E804
:107E0000A50194010E94C2E8CF84D888E988FA8845
:107E1000C20ED31EE41EF51E54E1C516D104E104C2
:107E2000F1040CF479CE8CEEC816D104E104F1040F
:107E30000CF06CCE90E8C916D104E104F1040CF406
:107E400079CECF86D88AE98AFA8A2EEF30E040E0F0
:107E500050E02C193D094E095F0969017A014F85EF
:107E6000588969897A8980EE9AE00E94FB3BB701C4
:107E7000A6018BED9AE00E94FB3B4F815D896E89E4
:107E80007F8984ED9AE00E94283A488D598D6A8D49
:107E90007B8D8DEC9AE00E94283AAB89BC891397C0
:107EA0000CF498C0C701B6010E9403E220E030E064
:107EB00040E850E40E9462E269837A838B839C836A
:107EC0002F813D894E895F89688D798D8A8D9B8D43
:107ED0000E94F2E82BED3FE049E450E40E9462E2A8
:107EE00020E030E040E05FE30E9462E29B01AC01F1
:107EF00069817A818B819C810E9476E96F83788782
:107F000089879A87C501B4010E9403E22FE632E116
:107F100043E85AE30E9462E24B015C012AE939E935
:107F200049E15FE36F81788589859A850E9462E2E5
:107F300069837A838B839C839B01AC010E94F3E865
:107F4000A50194010E9476E968A379A38AA39BA363
:107F500029813A814B815C81C501B4010E9462E2B2
:107F600020E030E040E05EE30E9462E26C8F7D8FB3
:107F70008E8F9F8F4F81588569857A8587EC9AE02F
:107F80000E94283AB501A40181EC9AE00E94283AA7
:107F90008AE00E946A3982EB9AE00E948239498124
:107FA0005A816B817C818CEA9AE00E94283A48A130
:107FB00059A16AA17BA186EA9AE00E94283A4C8DD9
:107FC0005D8D6E8D7F8D80EA9AE00E94283A8AE06E
:107FD0000E946A398F859889A989BA898C0D9D1D5F
:107FE000AE1DBF1DB595A795979587958093A9144C
:107FF0002B893C892F5F3F4F3C8B2B8B1F833D810F
:108000003D8B4E814E8B2F8A5301420159A55CA3B3
:1080100062CDCF93DF93EB010E948239CE01DF91D5
:10802000CF910C94B7CB4F925F926F927F928F92C9
:108030009F92AF92BF92CF92DF92EF92FF920F93F7
:108040001F93CF93DF9300D01F92CDB7DEB78091FF
:108050003D0C803108F0C7C131E6E32E80913D0C24
:10806000803108F0F8C08091540B9091550B891B1A
:108070008F7709F4F0C00E94F43A97FF0BC00E947A
:10808000433A89E793E00E9482398091540B8093B0
:10809000550BE4CF8A3019F08D3009F0D3C010921F
:1080A0003C0C8091DA0B9091DB0BFC01EA52F44F0F
:1080B0001682892B19F40E945586D0CF1092DB0BC3
:1080C0001092DA0B0CED1BE0F8018191803209F47B
:1080D00046C08E3409F0A1C064E773E0C8010E9475
:1080E00079E16C01892B41F06EE470E0C8010496DF
:1080F0000E9443EB009709F4C8014AE050E070E0A9
:1081000060E001960E94F0DE4B015C018091D60B8D
:108110009091D70BA091D80BB091D90B0196A11DCE
:10812000B11D88169906AA06BB0629F060E081E415
:1081300093E0CD2851F16AE270E0C8010E9472EB31
:108140009C01009729F1982F901BF12C992349F05D
:108150009150F801E90FF11D8081F826F7CF8F01CA
:10816000B3CF4AE050E070E060E0C90101960E94A0
:10817000F0DE4F2C512C712C612C64157505860591
:10818000970551F060E082E293E00E94B0B866CFBC
:1081900060E088EF92E0F9CF8092D60B9092D70BF7
:1081A000A092D80BB092D90B8091A4058130E1F058
:1081B00067E470E0C8010E9443EB0097A9F04AE031
:1081C00050E070E060E001960E94F0DE62307105E0
:1081D0008105910548F487E592E00E94823960E0CC
:1081E0008DE492E00E94771F8091DC0B8B3309F4C1
:1081F00035CF80913D0C803108F030CF80913F0C1D
:108200008E9DC00111246CED7BE0805C934F0E9439
:108210004EEB80E00E947CB821CF8091C61680FF93
:10822000C3CF61E076E2C8010E9479E1009731F0A6
:10823000FC01838180538A3008F0B6CF60E08EEC79
:1082400092E0A3CF2AED3BE04CED5BE06CE37CE0F9
:108250000E94DE1603CF8091C61682FFC4C01A8228
:10826000198281E6F82E90E1B92E29E6A22E80919E
:108270003D0C803108F0B7C00E9416178111B3C0C1
:1082800041E050E0BE016D5F7F4F88EB94E10E94BA
:108290003ACD0B8110E0019711F00FEF1FEF8091A5
:1082A000C0149091C114A091C214B091C3148093D2
:1082B000C2169093C316A093C416B093C5160E941D
:1082C00016170F3F100749F4811107C00E94433A67
:1082D00081E993E00E948239CACF40913F0C242F5C
:1082E00030E00A3061F00D3051F0882309F46DC0A0
:1082F00089819A81009719F001969A838983109257
:108300002E0389819A81F29EF001F39EF00D1124D3
:10831000E35CF34FDF01A80FB91F13961C92892B62
:10832000B9F50E9455860E941617882309F49FCF3D
:108330000E949E7788EB94E10E94496C8091BD1663
:108340008823F1F181508093BD168A9DC0011124CC
:1083500062E0835E9A4F0E9471CFE091BD1624E0E7
:10836000E29FF0011124E75EFA4F40815181628162
:1083700073814093C2165093C3166093C4167093D2
:10838000C51688EB94E10E9412CC0E94B0C76FCF53
:108390001A82198283818D3479F48481823361F465
:1083A0008581853349F4868180538A3028F0809115
:1083B000C6168B7F8093C61681E00E947CB8B3CF2F
:1083C0000E94A1C7B092A40552CF4F9DA0011124D5
:1083D000405C534F9E012F5F3F4F6EE273E0802F52
:1083E0000E94DE1644CF0E9482C14B015C01809145
:1083F0003C0390913D03A0913E03B0913F03009751
:10840000A105B10551F14091E8055091E905609150
:10841000EA057091EB05840F951FA61FB71FA501F4
:108420009401281B390B4A0B5B0BDA01C901B7FD1C
:1084300014C00E94433A6091F1057091F20580E109
:1084400092E00E9409408AE00E946A3940E070E0B0
:1084500060E090E080E00E94703A80910B01909182
:108460000C01A0910D01B0910E01892B8A2B8B2B51
:1084700079F090911E1580911F15981709F4FCC092
:108480008092E8059092E905A092EA05B092EB058A
:108490000E9482C16B017C0180919103811108C00F
:1084A00020911E1590911F1581E0291301C080E0D5
:1084B0002091A5143091A61491E089272A3A31051C
:1084C0000CF480E091E040912A0350912B036091DD
:1084D0002C0370912D03452B462B472B09F490E07C
:1084E000981789F0882309F401C1D701C601805685
:1084F0009444A24FBF4F80932A0390932B03A093E1
:108500002C03B0932D034090500B5090510B609072
:10851000520B7090530B209126033091270340910A
:10852000280350912903C301B2010E94FCE1882372
:1085300019F180912A0390912B03A0912C03B09103
:108540002D034092260350922703609228037092D5
:108550002903892B8A2B8B2B09F449C0D701C6012B
:1085600080569444A24FBF4F80932A0390932B03CD
:10857000A0932C03B0932D0380912A0390912B0399
:10858000A0912C03B0912D030097A105B10579F1BD
:10859000C81AD90AEA0AFB0AF7FC29C010922A0372
:1085A00010922B0310922C0310922D038BEF91E06D
:1085B0000E94823960E087EE91E00E94771F8091EF
:1085C000A7149091A8141816190624F490E080E0DE
:1085D0000E944AA08091AB059091AC05181619062F
:1085E00034F41092AC051092AB050E946A6280913F
:1085F0002F0390913003A0913103B0913203A50174
:108600009401281B390B4A0B5B0BDA01C901B7FD3A
:108610008FC090911E1580911F15F0903706981706
:1086200049F0E0911F153BE4E39FF0011124EF5660
:10863000F94FF0800E9482C1FF2009F4D1C000915F
:108640002203109123032091240330912503011567
:1086500011052105310509F04DC06C597F4F8F4F31
:108660009F4F60932203709323038093240390937E
:108670002503FF24FA9444C00E9482C10091E805BA
:108680001091E9052091EA053091EB05C0900B01AE
:10869000D0900C01E0900D01F0900E010C0D1D1D0D
:1086A0002E1D3F1D601B710B820B930B97FF03C0A8
:1086B00010923303EDCE809133038111E9CE81E036
:1086C000809333035E9A809194058E7F8093940506
:1086D0005E9A809194058D7F80939405159A809180
:1086E00094058B7F809394055E9AD2CE80E090E0D3
:1086F000DC0101CF601B710B820B930B97FDB9CF8F
:108700000F2D10E084E00E943AB8F11072C060E0D2
:1087100084E00E948BC044E6840E911CA11CB11C15
:1087200080922F0390923003A0923103B0923203D3
:108730000E9455868091A4058823F1F110910801CB
:108740001130B1F18091C61680628093C61681E027
:108750008093080164EF71E080E090E00E94A8330C
:108760000E94D2D18091C61683FFA5C0123028F492
:1087700060E080EA93E00E94771F01E083E080934D
:1087800053010E9482C16C597F4F8F4F9F4F60935E
:108790008503709386038093870390938803002357
:1087A00039F0123029F481E08093BC160E942DD25A
:1087B0000E943E940E94E9300F900F900F90DF913D
:1087C000CF911F910F91FF90EF90DF90CF90BF90CE
:1087D000AF909F908F907F906F905F904F90089593
:1087E0001092220310922303109224031092250367
:1087F00087CF0F3F110511F461E08ACFECE3F6E279
:10880000E491E150EA3008F051C0F0E0E65FFB4B44
:108810000C94E1E8144419441E4428445644564438
:1088200032443A4442444C4484B5806884BDF7BC29
:1088300072CF84B5806284BDF8BC6DCF809180001A
:10884000806880938000109389000093880063CF34
:108850008091800080628093800010938B00009351
:108860008A0059CF8091B00080688093B000F09268
:10887000B30051CF8091B00080628093B000F0923D
:10888000B40049CF8091900080688093900010934D
:108890009900009398003FCF809190008062809370
:1088A000900010939B0000939A0035CF003811057B
:1088B0000CF0A2CF2CCF00E0112309F479CF5ECFCA
:1088C0002F923F924F925F926F927F928F929F92E0
:1088D000AF92BF92CF92DF92EF92FF920F931F93CE
:1088E000CF93DF93CDB7DEB764970FB6F894DEBFB2
:1088F0000FBECDBF8091FB0A83FDB0C10E944B3AF1
:10890000898787FDABC189E40E945A30882309F426
:1089100097C10E94363090E01816190614F481E0D1
:1089200090E026E0289FF001299FF00D1124E255E8
:10893000FA4F808191811B8A0E944AA02091A7143E
:108940003091A8148091A5149091A61482179307D2
:108950008CF48DEC99E09F938F9388ED99E09F9331
:108960008F931F920E945E1F0F900F900F900F9099
:108970000F9005C02B8982EC99E0222361F381E0FE
:10898000809352011C821D821E821F821A861B86C2
:108990001C861D861F862CE3288B3CE1398B46E420
:1089A0004A8B212C312C50E85A838FEB8B83198210
:1089B00091E09E87812C912C540101C01E8600916C
:1089C000A7141091A814B801012E000C880B990B64
:1089D0000E9403E2D62EE72EF82E988791014A8155
:1089E0005B810E94FCE1882391F08091A514909115
:1089F000A6143B893111E7C041E0498308171907E4
:108A00000CF019822D2C3E2CFA8258855B830E9433
:108A100082C16B017C01DC01CB012A853B854C8541
:108A20005D85821B930BA40BB50BB7FD2FC0D7013F
:108A3000C60188519C4FAF4FBF4F8A879B87AC8739
:108A4000BD8789850E9433718EEB99E00E9482393F
:108A500081149104A104B10409F4E0C0C501B4017A
:108A60006053784F8F4F9F4F6C197D098E099F0976
:108A700028EE33E040E050E00E9444E8CA01B9012A
:108A80004AE00E94DA3B8AE00E946A390E94134061
:108A90000E9482C16093E8057093E9058093EA051E
:108AA0009093EB056091A5147091A614072E000C0D
:108AB000880B990B0E9403E26887072F182F9C8B65
:108AC000262F372F482F592FB1018A819B810E9471
:108AD000F2E82B013C0120E030E0A9010E9476EA97
:108AE00087FF04C077FA709477F87094811491042A
:108AF000A104B10409F096C020E030E040E85FE353
:108B0000C301B2010E94FCE187FF10C09E85812C49
:108B1000912C5401992331F08AE9882E82E0982E15
:108B2000A12CB12C8C0C9D1CAE1CBF1CA981AA23AE
:108B300099F12C813D814E815F81211531054105DF
:108B4000510541F0D701C601821B930BA40BB50B55
:108B5000B7FD22C02885302F412F5C896F85788929
:108B600089899A890E94F2E820E030E040EC5FE3D6
:108B70000E94FCE187FD2AC0D701C601805A9541B9
:108B8000AF4FBF4F8C839D83AE83BF8398859F87F4
:108B9000088B198BAC89AA8B809152018823B1F084
:108BA00081149104A104B10409F408CFB0EDCB1AEB
:108BB000B7E0DB0AE108F108C818D908EA08FB08A1
:108BC000F7FCFCCE03C0081719070CF58091520181
:108BD000882309F443C01092520164960FB6F894AA
:108BE000DEBF0FBECDBFDF91CF911F910F91FF90E0
:108BF000EF90DF90CF90BF90AF909F908F907F903D
:108C00006F905F904F903F902F900C94B7BA2D2C9F
:108C10003E2CFA8288858B831982F9CE8FE30E94DD
:108C20006A3931CF20E030E040E450E4C301B201C2
:108C30000E9476EA18160CF079CF4601570176CFDC
:108C400083E50E945A308B8B811105C082E50E941A
:108C50005A30882319F00E94761C6ECE64960FB6A7
:108C6000F894DEBF0FBECDBFDF91CF911F910F9162
:108C7000FF90EF90DF90CF90BF90AF909F908F903C
:108C80007F906F905F904F903F902F9008952F921C
:108C90003F924F925F926F927F928F929F92AF928C
:108CA000BF92CF92DF92EF92FF920F931F93CF93D9
:108CB000DF93CDB7DEB7CB54D1090FB6F894DEBF42
:108CC0000FBECDBF2C968FAF2C97809147038D346C
:108CD00009F481C4843511F40C94CA5B873491F48F
:108CE00080914503909146038C31910509F434C27B
:108CF00008F06AC08430910509F4AEC130F40297DF
:108D000008F4F7C00E94DDBA77C18531910509F4F6
:108D100073C14B97B9F70E94EBBA81116DC18CE01A
:108D2000EEE5F1E0DE01119601900D928A95E1F7F2
:108D300070E060E080E50E94673040E050E068E469
:108D400072E44CA35DA36EA37FA340E050E060EA11
:108D500070E448A359A36AA37BA3813009F4B5C189
:108D6000823009F4D1C120E030E040E050E460916D
:108D70004C0B70914D0B80914E0B90914F0B0E94BC
:108D8000F3E87B018C0120E030E04AE753E40E94E5
:108D900076EA181624F4E12CF12C0AE713E4A984EE
:108DA000BA84CB84DC849701A801B501C6010E9476
:108DB00076EA181614F475018601C701D8018C8F64
:108DC0009D8FAE8FBF8FC2C18A35910509F4E6C36E
:108DD00060F58D31910509F43DC38A9709F092CF72
:108DE0008091A405813009F007C189E40E945A30BE
:108DF000082F10E0882319F00E94761C182F8AE4AF
:108E00000E945A30F82E882311F40C942C5C0E9496
:108E1000761C002309F421C3153010F40C941E5C59
:108E20008AE595E00E948239E7C08B35910509F407
:108E3000B8C38C35910509F065CF9AE6C92E91E04B
:108E4000D92EF12CE12C00E010E0D6018D916D01BE
:108E50000E945A30382E8823E1F10E947A1C4B017F
:108E60005C01133059F0F701EF5FF94F2081318138
:108E7000428153810E94F2E84B015C01F701EC5BF7
:108E8000F44F2081318142815381C501B4010E9498
:108E9000F2E82B013C012DEB37E346E855EB0E944D
:108EA00076EA87FD0AC02DEB37E346E855E3C301B8
:108EB000B2010E94FCE1181664F4133009F075C386
:108EC0008092500B9092510BA092520BB092530B88
:108ED000032D1F5FB4E0EB0EF11C143009F0B5CF89
:108EE000002321F080E59BE00E9483830E94148E82
:108EF00083C08091A405813009F07EC06DEEC62E3E
:108F000063E0D62E74E4E72E7BE0F72EE1E0AE2E90
:108F1000E6E0BE2E10E088E5810F0E945A308823DB
:108F200009F47EC00E947A1C2B013C01812F0E9413
:108F30003217882309F46AC0D7012D913D914D91D4
:108F40005C91C301B2010E94F3E8D6016D937D9359
:108F50008D939C9313971F5FF4E0CF0ED11C24E0F8
:108F6000E20EF11C34E0A30EB11C1330A1F685E42F
:108F70000E945A30882309F45EC00E947A1C6B015B
:108F80007C0183E00E943217882371F02091500BFE
:108F90003091510B4091520B5091530BC701B601C8
:108FA0000E94F3E86B017C01C092F903D092FA03AE
:108FB000E092FB03F092FC0386E40E945A3088237F
:108FC000C9F00E947A1C20E030E0A9010E9476EAF4
:108FD000181684F40E947A1C20E030E040E752E446
:108FE0000E9476E96093210170932201809323010E
:108FF000909324010E945E892C96FFAD2C97F1116D
:109000000C947B510E9490390C947B51F501208186
:10901000318142815381C301B2010E94F2E895CFB0
:10902000F70180819181A281B381F60180839183D0
:10903000A283B38390CF8091500B9091510BA0915C
:10904000520BB091530B8093F9039093FA03A093C2
:10905000FB03B093FC03B0CF80E50E945A30C12CD3
:10906000D12C7601882321F00E94561C6B017C01D3
:1090700083E50E945A30882361F00E947A1C20E028
:1090800030E04AE754E40E9462E20E94EFE96B019B
:109090007C010E949E7780916B12811105C060E077
:1090A00081E595E00E94771F0E9482C1C60ED71EFF
:1090B000E81EF91E0E9482C16C197D098E099F0964
:1090C00097FF9ACF0E941340F5CFBE01605E7F4F9D
:1090D000CE0109960E943486E0904C0BF0904D0B27
:1090E00000914E0B10914F0B2D813E814F81588581
:1090F00069817A818B819C81DE0194966D010E9449
:109100007C850E94148E78CF29853A854B855C85B5
:1091100060914C0B70914D0B80914E0B90914F0BC9
:109120000E94F3E86B017C0120E030E04AE753E461
:109130000E94FCE187FD06C0C12CD12C5AE7E52E28
:1091400053E4F52ECC8EDD8EEE8EFF8EBE01605E7A
:109150007F4FCE014C96BECF87E00E944B8588237F
:1091600009F464C10E949E77109228016091010465
:109170008CE40E947530982E80E00E949A300E9404
:1091800082C16093E8057093E9058093EA059093A6
:10919000EB058091210190912201A0912301B091D2
:1091A00024018093380390933903A0933A03B0933A
:1091B0003B0380911F01909120019093370380938E
:1091C000360384E690E09093200180931F0181E0B4
:1091D000809392050E94118F8AE50E94251CA82E7B
:1091E00088E50E94251C182F89E50E94251CB82EB1
:1091F000181308C0B12EA11205C011E0BB24B3940E
:10920000AA24A39482E50E945A30882309F416C147
:109210000E947A1C3B01882EC92E20E030E0A90173
:109220000E94FCE1882309F444C0111103C0BB2053
:1092300009F4D0C0D0904C0BE0904D0BF0904E0B49
:1092400000914F0B9301482D5C2D6D2D7E2D8F2DA0
:10925000902F0E9476EA181624F0D62CE72CF82CD2
:109260000C2D80E090E0A0E8B0E48C8F9D8FAE8F55
:10927000BF8F20E030E04AE753E46D2D7E2D8F2D27
:10928000902F0E94FCE187FD05C0D12CE12C2AE73C
:10929000F22E03E48D2D9E2DAF2DB02F89839A835E
:1092A000AB83BC83BE01645E7F4FCE0101960E94FA
:1092B0003486112309F489C0BB2009F483C01092BD
:1092C000440B1092450B1092460B1092470B1092D4
:1092D000480B1092490B10924A0B10924B0B0E94B4
:1092E0005386E9E9F6E1C590D590E590F490EDE973
:1092F000F6E14590559065907490A7019601C301E1
:10930000B2010E94FCE187FFA0C0A7019601C30142
:10931000B2010E9476E99B01AC010E9462E220E06A
:1093200030E040E85FE30E94F3E80E94B4EA20E006
:1093300030E048E452E40E9462E269837A838B83DE
:109340009C8320914C0B30914D0B40914E0B5091D2
:109350004F0B28A739A74AA75BA720E030E040ECD5
:109360005FE3C301B2010E9462E22B013C0177FA84
:10937000709477F8709420E030E040EC5FE3C70130
:10938000B6010E9462E29058AE014F5F5F4F6A01E2
:10939000E8A4F9A40AA51BA5A30192010E947C855B
:1093A0000E942C901092440B1092450B1092460B89
:1093B0001092470B1092480B1092490B10924A0BD7
:1093C00010924B0B80E00E94C38CBB2019F081E00F
:1093D0000E94C38CAA2019F082E00E94C38C0E94D4
:1093E00053868091910580939205892D0E949A3031
:1093F0008091380390913903A0913A03B0913B03D7
:109400008093210190932201A0932301B093240122
:1094100080913603909137039093200180931F0130
:1094200083E0809353010E94148EE6CD60E08FE4C8
:109430000E947530882309F495CEDECD612C712C05
:1094400030E8832E40E4C42EF0CEA3019201C70180
:10945000B6015FCF0E94AD5CCFCD853008F0E0CC87
:1094600090E1E4E4FBE0ADEEB3E001900D929A955B
:10947000E1F70023A1F054E01502F0011124E756B2
:10948000FA4E40815181628173814093ED03509384
:10949000EE036093EF037093F003FF2091F094E0EC
:1094A0008902F0011124EB57FA4E80819181A2814B
:1094B000B3818093F1039093F203A093F303B093ED
:1094C000F40386E40E945A30811151C0C12CD12C82
:1094D00076018090210190902201A0902301B0900C
:1094E000240120E030E0A901C701B6010E94FCE19F
:1094F000882341F0C0922101D0922201E092230101
:10950000F092240100911F011091200184E690E067
:109510009093200180931F01C0905801D090590171
:10952000E0905A01F0905B0180E090E0A0E8BFE39A
:109530008093580190935901A0935A01B0935B0115
:109540000E945E898092210190922201A0922301C3
:10955000B09224011093200100931F01C092580182
:10956000D0925901E0925A01F0925B0145CD0E94E0
:109570007A1C6B017C0120E030E0A9010E9476EAB0
:1095800018160CF0A3CF20E030E040E752E4C7010A
:10959000B6010E9476E96B017C019BCF10924003DB
:1095A0002BCD8FE08093400327CDF701EF51FC4F87
:1095B0005F01A301920160817181828193810E9488
:1095C000F3E8D5016D937D938D939C931397812F31
:1095D0000E942B857ECC8091450390914603823773
:1095E000910511F40C94FB5408F080C18934910565
:1095F00009F445C608F0D9C08831910509F498C42A
:1096000008F06CC08231910511F40C940A5400F5F5
:109610008230910508F411C4419709F073CB8BE0B7
:1096200092E00E94011C882309F45BC488E50E9433
:10963000251C81115E9889E50E94251C81115E9888
:109640008AE50E94251C882309F4D6CC1598D4CC31
:109650008531910509F456C458F5449709F052CB69
:109660008091C61683FF47C48EE995E00E94823937
:109670008091C61683FF17C08EEE94E10E94A16D03
:109680008BE1EEEEF4E1DE01119601900D928A95E8
:10969000E1F770E060E0CE0101960E949BD0CE0120
:1096A00001960E94A66D8FE895E00E948239A4CCB5
:1096B0008631910509F429C4479709F023CB80919D
:1096C000410390914203FC012191222309F42AC411
:1096D0002032D1F7DF0111971C92F6CF8C31910522
:1096E00009F4A5C420F58A31910509F44FC408F4A2
:1096F0002EC483E40E94251C882309F467C489ECE6
:1097000095E00E9482398091BB14882309F459C4E2
:10971000BE016F5F7F4F88EB94E10E946C6CCE01BD
:1097200001960E94B7CB8AE00E946A3965CC8E31DF
:10973000910509F48BC408F482C48F31910509F4B2
:10974000F4C4809709F0DECA8091C61682FD0E949B
:109750009E778091C61683FF4FCC60E080E50E9423
:109760007530182F682F80914103909142030E9419
:1097700071CF83E50E945A30882381F00E94661CD5
:10978000AB01BC014093C2165093C3166093C4163C
:109790007093C51688EB94E10E9412CC0E94B0C76A
:1097A00011112ACC0E94879027CC8C35910511F499
:1097B0000C945E5408F049C08135910511F40C9465
:1097C000E55378F48C34910509F469C58D3491051D
:1097D00009F47AC58B34910509F094CA0E948790E8
:1097E0000BCC8335910511F40C94025410F40C94B5
:1097F000FA538435910511F40C940A54853591057A
:1098000009F080CA83E50E94251C882309F4F4CB63
:109810000E9482C16093E8057093E9058093EA0590
:109820009093EB050E947A1C20E030E04AE754E474
:109830000E9462E20E94EFE960933C0370933D0353
:1098400080933E0390933F03D7CB8C36910509F468
:10985000D3CBE8F58936910509F43EC540F5883645
:10986000910509F04FCA8091FB0A83FDC5CB0E9488
:109870004B3A87FDC1CB89E40E945A30882311F40A
:109880000C94EB5B0E94363090E01816190614F425
:1098900081E090E026E0289FF001299FF00D11243F
:1098A000E255FA4F808191810E944AA0A5CB8A3669
:1098B000910509F43AC58B36910509F023CA80E574
:1098C0000E9440BB811198CB1092370695CB8E3603
:1098D000910509F45EC508F4FBC48F36910509F4BF
:1098E0006BC58037910509F487CB0CCA8232E1E061
:1098F0009E0711F40C94C25708F0AAC18E3B910543
:1099000009F4C7C508F094C08737910511F40C9489
:10991000505588F48537910511F40C94035510F0D7
:109920000C9415558337910509F0ECC988EB96E046
:109930000E94823961CB8937910511F40C945D55F1
:1099400010F40C9454558C38910509F476C581397E
:10995000910509F0D7C983E50E945A30882311F494
:109960000C9465550E94761C823010F00C94695559
:109970008C01112788E40E945A308823D1F00E947C
:10998000761C8A3A910514F40C9471550E94761C49
:10999000843B914014F00C9475550E94761C26E08F
:1099A000209FF001219FF00D1124E255FA4F918381
:1099B000808382E40E945A308823C9F00E94761C7A
:1099C000059714F40C9479550E94761C8D389105F6
:1099D00014F00C947D550E94761C26E0209FF00127
:1099E000219FF00D1124E255FA4F9383828386E480
:1099F0000E945A30882309F4FFCA0E94761C97FF00
:109A000002C00C9481550E94761C8F3F910519F07D
:109A100014F00C9485550E94761C26E0209FF001DE
:109A2000219FF00D1124E255FA4F95838483E4CAF7
:109A30008D3C910511F40C94215608F070C0893CBE
:109A4000910511F40C948C5590F5883C910509F022
:109A500059C90E944B3A182F87FDCECA00910604BF
:109A600084E40E945A30F82E8823C1F00E947A1CA8
:109A70004B015C0120E030E0A9010E94FCE1882359
:109A800011F40C94895524E01202F0011124EE5FC8
:109A9000FB4F80829182A282B3820F2D602F83E5DB
:109AA0000E947530809306040E94375FA5CA8B3CE4
:109AB000910511F40C94B6558C3C910509F022C91E
:109AC00083E092E00E94011C81110C94D9554091D1
:109AD000300B5091310B6091320B7091330B82EE51
:109AE00097E00E94283A4091340B5091350B6091D9
:109AF000360B7091370B8FED97E00E94283A40911A
:109B0000380B5091390B60913A0B70913B0B85E10A
:109B100098E10E94283A8AE00E946A396DCA833D22
:109B2000910511F40C94A25608F04DC045E9E42EBD
:109B300045E0F42E10E08E3C910509F0E3C888E57D
:109B4000810F0E94251C882351F00E947A1CF70186
:109B50006083718382839383812F0E942B851F5F93
:109B6000F4E0EF0EF11C133051F780E192E00E9417
:109B7000011C8111BBC940919505509196056091DA
:109B800097057091980584E298E00E94283A4091E8
:109B9000990550919A0560919B0570919C0587E10C
:109BA00097E20E94283A40919D0550919E05609150
:109BB0009F057091A00584E197E20E94283A8AE00F
:109BC0000E946A3919CA8C3D910511F40C946A57A8
:109BD0008D3D910509F096C80E944B3A082F87FDEC
:109BE0000BCA83E50E945A30002E000C110B78013D
:109BF000EE0CFF1C882311F40C94A8570E94761CCD
:109C0000F701EB5DFE4F91838083000F111F000F62
:109C1000111F9801285A3E4F7901BC01990F880BFA
:109C2000990B0E9403E22AE037ED43E25CE30E94D5
:109C300062E203501C4FD8012D913D914D915C91F2
:109C40000E9462E2F7016083718382839383D4C9A7
:109C50008C3A21E0920711F40C94DE5A08F083C08C
:109C60008F3241E0940711F40C94E35810F58D32D3
:109C7000A1E09A0711F40C941C5810F00C949D5814
:109C80008C32914009F03EC864E071E083E50E94A7
:109C900067308C0168EE73E080E50E946730893898
:109CA000F3E19F0710F088E893E1B8010E949A94CD
:109CB000A3C98A39F1E09F0709F49EC938F48039B5
:109CC000914009F01FC80E949E7796C9843A41E0EE
:109CD000940711F40C94E758853A914011F00C94D4
:109CE000824688E50E94251CC82E89E40E94251C16
:109CF000A82E882311F40C94455A0E94761C082F34
:109D000089E50E94251CF82E8AE40E94251CE82E75
:109D1000882311F40C94705A0E94761C182F8AE53F
:109D20000E94251CD82EB12C811104C081E50E940F
:109D3000251CB82EA11001C0E12C8E2D90E0C11081
:109D400001C0F12C8F0D911D019731F4D1100C94AD
:109D50009B5AB1100C949B5A0E94433A85E299E0B9
:109D60000E94823949C9883FA1E09A0711F40C94F6
:109D7000985B18F5853FE1E09E0711F40C94905B29
:109D800040F4843F914011F00C9482460E94697423
:109D900033C9863F31E0930711F40C94945B873FFD
:109DA000914011F00C94824661E083E50E94753089
:109DB00091E089270E9484A01FC9803A53E095074B
:109DC00009F4A5C178F48C30924011F00C948246CD
:109DD0008091C61682FD02C00C94AB5B80648093B8
:109DE000C6160AC9873EE3E09E0711F40C94B35BE4
:109DF000893E934011F00C9482468091BC168111EB
:109E00000C94C35B0E943A906D33710581059105F6
:109E100020F088EA99E00E943B5C84EA99E00E9485
:109E20003B5C84EE8093CA0380E999E00E9482390A
:109E30008CE899E00E943B5CDFC880E50E945A30C4
:109E4000C12CD12C7601882321F00E94561C6B0175
:109E50007C0183E50E945A30882361F00E947A1CBD
:109E600020E030E04AE754E40E9462E20E94EFE919
:109E70006B017C010E949E77809141039091420387
:109E80000097E1F00E9459B881E080939103C114DA
:109E9000D104E104F10431F00E9482C1C60ED71E44
:109EA000E81EF91E809191038823B1F0C114D104FA
:109EB000E104F10449F40E941340F4CF60E083E729
:109EC00095E00E94771FE0CF0E9482C16C197D0946
:109ED0008E099F0997FDEFCF109291030E94B7BAA8
:109EE0008BC860E086E895E00E94771F5E985E98D8
:109EF00015985E9881C80E94473A8FEA95E00E94C3
:109F000082397AC80E94D2D177C88091C61682FD64
:109F100073C80E94A1C78091C616877F8062809314
:109F2000C6166AC860E00E9471CF1092CA0364C866
:109F30000E94E033882321F00E94B0C70E948790DE
:109F40008DE99CE00E9480B50E94B7BA55C8809107
:109F5000C61682FF03C08B7F8093C61680910006D1
:109F6000813069F482E0809300060E9482C1609390
:109F7000DD037093DE038093DF039093E0030E9480
:109F8000B7BA89EB95E00E9480B536C88091C616B5
:109F900083FF32C883E50E945A30882309F42CC815
:109FA0000E94661CAB01BC014093C2165093C316BD
:109FB0006093C4167093C51688EB94E10E9412CC8E
:109FC0001BC88FEB95E00E948239ADCB8091C616FD
:109FD00082FF27C0C090C216D090C316E090C4166E
:109FE000F090C51688ED95E00E9482394AE0C701DD
:109FF000B6010E942DC78FE20E946A396091BE1699
:10A000007091BF168091C0169091C1164AE00E94CF
:10A010002DC78DE00E946A398AE00E946A390C944B
:10A02000FC478AEE95E00E9482390C94FC478091AF
:10A030004103909142030E9429CF0C94FC478091E8
:10A04000C6168E7F8093C6160C94FC478091C61668
:10A0500083FD02C00C94FC470E94F8CB8091C61689
:10A0600083FD02C00C94FC47409141035091420390
:10A07000BE01645E7F4F80E00E9437B78C0100977D
:10A0800011F40C94FC476C8D7D8D19821C8222E0AA
:10A09000AC01CE0101960E94AC6D811119C0F12C6A
:10A0A000CE0101960E94A66DB801FF2031F186E134
:10A0B00096E00E9409408AE00E946A391092C21616
:10A0C0001092C3161092C4161092C5160C94FC4739
:10A0D000CE0101960E94A6CC882309F361E0CE014F
:10A0E00001960E94526C0097D1F225EEDC012C9370
:10A0F0001C820E9447C8F82ED3CF8EEF95E00E94B5
:10A1000009408BEF95E00E9482390C94FC47209126
:10A110004103309142039091C61692609093C61607
:10A12000C9010E9429CF0C94FC470E943A907B0100
:10A130008C0120E831E541E050E00E9444E8C9018B
:10A140006DE671E00E949AE84B015C01C801B7011D
:10A1500020E13EE040E050E00E9444E8CA01B9013D
:10A1600028E130E040E050E00E9444E8762E672E7F
:10A17000C62ED72E8CE3282E312C412C512CC80111
:10A18000B701A20191010E9444E8F62EE72ECA0110
:10A19000B901A20191010E9444E8CB018E010F5F39
:10A1A0001F4F8114910431F1EF92FF927F936F93CF
:10A1B0006F927F92BF92AF929F928F928CE496E0C3
:10A1C0009F938F931F930F930E9493E10FB6F89480
:10A1D000DEBF0FBECDBFC8010E9459B80E94473AEA
:10A1E000B80180E696E00E9409408AE00E946A3940
:10A1F0000C94FC47A114B10489F0EF92FF927F9375
:10A200006F936F927F92BF92AF928CE396E09F9391
:10A210008F931F930F930E9493E1D8CFCD2879F0AD
:10A22000EF92FF927F936F936F927F9280E396E01D
:10A230009F938F931F930F930E9493E1C7CF892B16
:10A2400069F0EF92FF927F936F9388E296E09F937D
:10A250008F931F930F930E9493E1B8CFEF92FF92D9
:10A2600084E296E09F938F931F930F930E9493E154
:10A270000F900F900F900F900F900F90ACCF80E544
:10A280000E94251C882311F40C94FC470E94363050
:10A29000853608F084E68093CA030C94FC478091CD
:10A2A0000006813011F00C94FC4782E08093000698
:10A2B0000E9482C16093DD037093DE038093DF030D
:10A2C0009093E0030C94FC470E94AB900C94FC47E5
:10A2D0000E9460440C94FC470E944B3A182F87FD63
:10A2E0000AC08DE696E00E948239812F0E94337168
:10A2F0008AE00E946A39C55BDF4F0FB6F894DEBF73
:10A300000FBECDBFDF91CF911F910F91FF90EF90C6
:10A31000DF90CF90BF90AF909F908F907F906F9085
:10A320005F904F903F902F90089580E50E9440BB32
:10A3300081110C94FC4781E40E94251C6091370632
:10A34000062F10E0811102C00FEF10E089E40E9497
:10A350005A30882311F40C94F65B0E94363090E05A
:10A360001816190614F481E090E026E0289FF00109
:10A37000299FF00D1124E255FA4F048115810F3FFA
:10A38000110519F010F00FEF10E0009337060C9450
:10A39000FC478EE40E945A30882311F40C94FC4749
:10A3A0000E94661C6093D60B7093D70B8093D80BDA
:10A3B0009093D90B0C94FC4783E50E94251C8823BD
:10A3C00029F083E50E9440BB8093FB0A0E94473A34
:10A3D0008EE796E00E9482398091FB0A882351F132
:10A3E00010E000E020E08091FB0A90E0B0E0A0E007
:10A3F000002E04C0B695A795979587950A94D2F735
:10A4000080FF12C0FF24F394F20E222319F08CE295
:10A410000E946A39F801EE0FFF1FEC58F94F859141
:10A4200094910E9482392F2D0F5F1F4F0530110527
:10A43000D1F679C980E796E0C6CD8091FB0A83FF0B
:10A4400002C00C94FC4789E40E945A30882311F41E
:10A450000C94025C0E94363090E01816190614F431
:10A4600081E090E026E0289FF001299FF00D112463
:10A47000E255FA4F828193818C38910514F08CE873
:10A4800090E09093AC058093AB050E946A620C94B7
:10A49000FC478091FB0A83FF02C00C94FC4789E4CF
:10A4A0000E945A30882311F40C940D5C0E943630BF
:10A4B00090E01816190614F481E090E026E0289F39
:10A4C000F001299FF00D1124E255FA4F828193810A
:10A4D0001CAA8C38910514F08CE890E09093AC05A0
:10A4E0008093AB050E946A622091AB053091AC0568
:10A4F0008091A9059091AA05821793070CF03BC1A2
:10A5000088E996E060E00E94771F81E08093520125
:10A510001DAA1EAA1FAA18AE1BAE1CAE1DAE1EAEF3
:10A5200021961FAE21979CE322969FAF2297ACE124
:10A530002496AFAF2497B6E42896BFAF2897312C66
:10A54000212CE0E8ECA7FFEBF8AB18A621E02FAF39
:10A55000812C912C54010091AB051091AC05B801F0
:10A56000012E000C880B990B0E9403E26B017C0109
:10A57000232D322D4CA558A90E94FCE1882389F097
:10A580008091A9059091AA053CA93111F7C041E03D
:10A5900048A7081719070CF018A63C2C2D2CECA680
:10A5A000F8AA0E9482C16B017C01DC01CB012BADBA
:10A5B0003CAD4DAD5EAD821B930BA40BB50BB7FD4F
:10A5C0002FC0D701C60188519C4FAF4FBF4F8BAFF3
:10A5D0009CAFADAFBEAF80E00E94337185E896E0DE
:10A5E0000E94823981149104A104B10409F4DBC0F2
:10A5F000C501B40168577C4E8F4F9F4F6C197D0980
:10A600008E099F0928EE33E040E050E00E9444E8C4
:10A61000CA01B9014AE00E94DA3B8AE00E946A3925
:10A620000E9413400E9482C16093E8057093E9057F
:10A630008093EA059093EB056091A9057091AA05B6
:10A64000072E000C880B990B0E9403E269AF7AAFCA
:10A650008C019B01AC01632D722D8CA598A90E94E1
:10A66000F2E82B013C0120E030E0A9010E9476EAEB
:10A6700087FF04C077FA709477F87094811491047E
:10A68000A104B10409F093C020E030E040E85FE3AA
:10A69000C301B2010E94FCE187FF10C09FADA2E898
:10A6A0008A2EA6E09A2EA12CB12C911103C0812CE8
:10A6B000912C54018C0C9D1CAE1CBF1CA8A5AA2378
:10A6C00009F442C02DA93EA94FA958AD2115310565
:10A6D0004105510541F0D701C601821B930BA40B24
:10A6E000B50BB7FD31C029AD3AADA80121966FADCC
:10A6F000219722967FAD229724968FAD2497289696
:10A700009FAD28970E94F2E820E030E040E85FE348
:10A710000E94FCE187FD35C0D701C601805A9541F2
:10A72000AF4FBF4F8DAB9EABAFABB8AF99AD2196DE
:10A730009FAF2197AAAD2296AFAF229724960FAF75
:10A74000249728961FAF2897809152018823C9F03B
:10A7500081149104A104B10461F0B8E8CB1AB3E10B
:10A76000DB0AE108F108C818D908EA08FB08F7FE77
:10A7700008C01FAEF0CE89E896E0C4CE08171907CE
:10A7800064F480915201882311F40C94FC471092D8
:10A7900052010E94B7BA0C94FC473C2C2D2CECA61D
:10A7A000F8AA18A6FECE8FE30E946A3936CF20E0C1
:10A7B00030E040E450E4C301B2010E9476EA18168A
:10A7C0000CF07CCF4601570179CF0E94E0710E94C6
:10A7D000AE770E94AB901092370668EE73E080E08F
:10A7E00090E00E94A83360E087EA96E00E94771F1D
:10A7F0000C94FC47809140038F7D806180934003DF
:10A800000C94FC47809140038F7E806280934003CC
:10A810000C94FC4783E50E945A308823F1F00E9493
:10A8200082C16093E8057093E9058093EA059093EF
:10A83000EB050E947A1C20E030E04AE754E40E94D5
:10A8400062E20E94EFE960930B0170930C01809328
:10A850000D0190930E010C94FC478BE092E00E9456
:10A86000011C882339F10E949E7788E50E94251CEF
:10A87000882331F05E9A809194058E7F80939405B1
:10A8800089E50E94251C882331F05E9A8091940509
:10A890008D7F809394058AE50E94251C882311F4FE
:10A8A0000C94FC47159A809194058B7F80939405B6
:10A8B0000C94FC470E94AE770C94FC470E944B3AE4
:10A8C00087FF02C00C94FC478BE092E00E94011CC1
:10A8D000882309F48BC0EAE6CE2EE1E0DE2EFCEF01
:10A8E000EF2EFAE0FF2E10E0F60181916F010E9439
:10A8F0005A30882309F465C0133009F06DC00E94F6
:10A900007A1C4B015C0120E030E040EA51E40E94F7
:10A91000FCE187FF4EC0A501940160911C0B709172
:10A920001D0B80911E0B90911F0B0E9476E92B014D
:10A930003C01AC019B0160911B0670911C0680914B
:10A940001D0690911E060E9462E260931B067093A2
:10A950001C0680931D0690931E06A3019201609130
:10A960002C0B70912D0B80912E0B90912F0B0E9430
:10A9700062E260932C0B70932D0B80932E0B9093BF
:10A980002F0B60912B0670912C0680912D069091D3
:10A990002E060E9401E2A30192010E9462E20E943F
:10A9A000EFE960932B0670932C0680932D0690930D
:10A9B0002E0680921C0B90921D0BA0921E0BB09243
:10A9C0001F0B1F5FB4E0EB0EF11C143009F08CCFAD
:10A9D0000E947A770C94FC470E947A1CD701549607
:10A9E0006D937D938D939C935797EBCF81E00E945D
:10A9F0007CBA0C94FC470E9417BA80E295E10E9451
:10AA0000BA730C94FC4780914103909142030097E4
:10AA100041F0FC012081222321F00E9459B80C94BE
:10AA2000FC470E94B7BA0C94FC4700914103109177
:10AA3000420394E0F12C40E0915009F1D8018C914F
:10AA4000282F2B7F2134A1F411962C912133B9F4B6
:10AA5000813419F1853409F441E098012E5F3F4FAC
:10AA600089012F5F3F4FD8018C918032C9F3E4CF29
:10AA7000803529F4F801818180538A3070F34111C7
:10AA80000E94473AFF2021F08AEB97E00E9482392A
:10AA9000C8010E9471390C94FC47FF24F394DDCF68
:10AAA0000E94F68E0C94FC4781E08093920580937F
:10AAB00091050E94118F0C94FC4710929205109200
:10AAC00091050E94118F0C94FC4790E080E00C945B
:10AAD000B84C0E94433A8DEB97E00E9482390C9467
:10AAE000FC478AEA90E00C94CF4C83EB91E00C9405
:10AAF000CF4C85E090E00C94ED4C8CE890E00C9409
:10AB0000ED4C90E080E00C940D4D8FEF90E00C94B4
:10AB10000D4D80E00C94524D0E944B3A87FF02C0CD
:10AB20000C94FC470AE611E06CEFE62E6AE0F62E84
:10AB30007EE6C72E71E0D72ED8018D918D010E943F
:10AB4000251C882359F00E947A1C0E94EFE9F70126
:10AB500060837183828393830E942C77F4E0EF0EED
:10AB6000F11CC016D10641F70C94FC470E944B3AE9
:10AB700087FF02C00C94FC475AE6E52E51E0F52E03
:10AB800010E000E0D7018D917D010E94251C8823F3
:10AB900049F00E947A1CF801E450F54F64A375A3B4
:10ABA00086A397A30C5F1F4F0031110559F70C9432
:10ABB000FC4783E50E945A30882391F00E947A1C5A
:10ABC0006093300B7093310B8093320B9093330B67
:10ABD0006093380B7093390B80933A0B90933B0B37
:10ABE00080E50E945A30882351F00E947A1C6093BD
:10ABF000300B7093310B8093320B9093330B82E5C3
:10AC00000E945A30882351F00E947A1C6093340BC2
:10AC10007093350B8093360B9093370B84E50E942D
:10AC20005A30882311F40C94FC470E947A1C6093DC
:10AC3000380B7093390B80933A0B90933B0B0C9429
:10AC4000FC4788E092E00E94011C882311F40C94D8
:10AC5000FC4782E40E94251C882351F00E94561C68
:10AC600060930C0B70930D0B80930E0B90930F0B56
:10AC700083E50E94251C882351F00E947A1C609372
:10AC80003C0B70933D0B80933E0B90933F0B84E500
:10AC90000E94251C882351F00E947A1C6093400B6F
:10ACA0007093410B8093420B9093430B88E50E9475
:10ACB000251C882351F00E947A1C60930F06709324
:10ACC0001006809311069093120689E50E94251CB8
:10ACD000882351F00E947A1C609313067093140627
:10ACE00080931506909316068AE50E94251C8823FA
:10ACF000B1F00E947A1C6093170670931806809337
:10AD0000190690931A062DEC3CEC4CEC5DE30E9486
:10AD1000FCE1181624F082EF97E00E94823985E466
:10AD20000E94251C882311F40C94FC470E947A1C75
:10AD300060931B0670931C0680931D0690931E065D
:10AD40000C94FC4740900106509002066090030668
:10AD5000709004062091290130912A0140912B0125
:10AD600050912C01C301B2010E94F3E868A779A7B2
:10AD70008AA79BA78090050690900606A0900706DC
:10AD8000B090080620912D0130912E0140912F01A5
:10AD900050913001C501B4010E94F3E86CA77DA772
:10ADA0008EA79FA7C0900906D0900A06E0900B06D8
:10ADB000F0900C0620913101309132014091330125
:10ADC00050913401C701B6010E94F3E868AB79AB3A
:10ADD0008AAB9BAB20913501309136014091370110
:10ADE00050913801C301B2010E94F3E82B013C01EC
:10ADF0002091390130913A0140913B0150913C0141
:10AE0000C501B4010E94F3E84B015C0120913D01B2
:10AE100030913E0140913F0150914001C701B60180
:10AE20000E94F3E86B017C010E94473A8DE398E0B1
:10AE30000E94823983E50E94251C882321F00E940C
:10AE40004A308093270180912701882309F43FC06D
:10AE500087EB98E00E94823985E398E00E9482396E
:10AE600048A559A56AA57BA586E897E10E94283ADE
:10AE70004CA55DA56EA57FA587E197E20E94283AC3
:10AE800048A959A96AA97BA984E197E20E94283AB6
:10AE900083E398E00E9482398BE298E00E94823935
:10AEA000B301A20186E897E10E94283AB501A40106
:10AEB00087E197E20E94283AB701A60184E197E270
:10AEC0000E94283A8AE00E946A390C94FC4783EB7E
:10AED00098E0C0CF82E40E94251C882341F0809135
:10AEE0001F01909120019093100180930F0182E542
:10AEF0000E94251C882341F080910F019091100140
:10AF00009093200180931F0183E50E945A3088238B
:10AF100031F00E94761C9093200180931F01E091F4
:10AF20004303F09144038081882311F40C94FC477F
:10AF300060911F01709120018DE498E00E94393AE0
:10AF400085E20E946A398AE00E946A390C94FC47C3
:10AF50000E94473A85E40E946A3980E3800F0E948C
:10AF60006A39F701EB5DFE4F6081718181E598E000
:10AF70000E94393A85E20E946A398AE00E946A3961
:10AF80000C94FC478AE50E945A30882331F10E94D4
:10AF90007A1C20E030E040E050EC0E94FCE187FDAC
:10AFA0003AC00E947A1C20E030E040E050E40E9469
:10AFB00076EA1816ACF10E947A1C2091180B309199
:10AFC000190B40911A0B50911B0B0E9462E20E94D8
:10AFD000E8E9CB010E94BBC105C083E50E945A305D
:10AFE0008111D5CF80E192E00E94011C81111DC02A
:10AFF0000E94473A40916B0450916C0460916D043B
:10B0000070916E0489E598E00E94283A8AE00E94D7
:10B010006A390C94FC4760E070E080E090ECCDCFA2
:10B0200060E070E080E090E4C8CF82E50E94251CDB
:10B030008111DECF0C94FC4785E40E9440BB811156
:10B0400074C080E50E94251C882351F00E947A1C60
:10B050006093AA147093AB148093AC149093AD14C6
:10B0600089E40E94251C882381F00E947A1C2CEA26
:10B0700035EC47E25EE30E9462E26093AE147093A7
:10B08000AF148093B0149093B11484E40E94251CF3
:10B09000882381F00E947A1C2CEA35EC47E25EE3BB
:10B0A0000E9476E96093B2147093B3148093B41441
:10B0B0009093B5140E94473A4091AA145091AB1452
:10B0C0006091AC147091AD148EE698E00E94283A1D
:10B0D0002CEA35EC47E25EE36091AE147091AF1458
:10B0E0008091B0149091B1140E9476E9AB01BC013B
:10B0F0008AE698E00E94283A2CEA35EC47E25EE3C3
:10B100006091B2147091B3148091B4149091B514FD
:10B110000E9462E2AB01BC0186E698E00E94283AF8
:10B120008AE00E946A390C94FC470E94433A82E705
:10B1300098E00E9482390C94FC4783E50E94251C0C
:10B14000182F882369F00E94761C9C0190935D0162
:10B1500080935C0191E0232B09F090E090934806E6
:10B1600080E50E94251C882361F020915C013091CC
:10B170005D01232B11F00E944A30809348060C9405
:10B18000FC4711110C94FC470E94473A80EA98E072
:10B190000E94823980914806882391F088E898E0DF
:10B1A0000E94823960915C0170915D018FE898E0A6
:10B1B0000E94393A8BE898E00E9482390C94FC474F
:10B1C00084E898E0EDCF0E940C3C0C94FC4783E5AA
:10B1D0000E94251C182F30900104882319F00E942A
:10B1E0004A30382E2091440B3091450B4091460B4C
:10B1F0005091470B27962CAF3DAF4EAF5FAF2797CF
:10B200004090480B5090490B60904A0B70904B0B4C
:10B2100080914C0B90914D0BA0914E0BB0914F0B28
:10B220002B968CAF9DAFAEAFBFAF2B97112329F0FC
:10B23000311003C080E00E949A3086E50E94251CF0
:10B2400021968FAF21970E94BB30882309F4B8C0A4
:10B2500083E40E94251C882309F49FC00E947A1C65
:10B260006B017C01A7E0B4E0B9ABA8ABB9A7A8A774
:10B27000F5E0FCA71AAE1BAE28EC2FAF02EC1CAA1F
:10B28000212C38EC3DAB42E449AF88A599A5239623
:10B290009FAF8EAF239715E02396AEADBFAD23973A
:10B2A0008D909D90AD90BD902396BFAFAEAF23978C
:10B2B0002CA9322D4DA959ADC501B4010E94FCE164
:10B2C00087FF04C08CAA292CADAAB9AE2AAD3BAD2C
:10B2D0004FAD502FC501B4010E9476EA181624F430
:10B2E0008AAE9BAEAFAE0B2D1150B1F6BCA5B150DE
:10B2F000BCA7E8A5F9A57496F9A7E8A7B111C5CF31
:10B300002AAD3BAD4FAD502F6CA9722D8DA999ADD3
:10B310000E94F3E820E030E040E05FE30E9462E258
:10B32000A70196010E94F3E86B017C012DEB37E346
:10B3300046E855EB0E9476EA87FD0AC02DEB37E31D
:10B3400046E855E3C701B6010E94FCE118162CF54A
:10B3500080E00E949A3015E0A8A8B9A805E0D501C0
:10B360006D917D918D919D915D014D01B4E08B1AA0
:10B370009108A70196010E94F2E8F40160837183AD
:10B3800082839383015059F7115028A939A92C5E63
:10B390003F4F39AB28AB1111DFCF21964FAD21972D
:10B3A000442351F00E94BB30882331F087EE98E0AF
:10B3B0000E9482390E94A939832D0E949A300DC0C3
:10B3C000311005C021963FAD21973323A9F30E9488
:10B3D000473A8DEF98E00E948239332051F08091F6
:10B3E0000104811106C00E94433A88EC98E00E9453
:10B3F00082390E94473A8AEB98E00E948239809114
:10B400000104882309F43EC087EB98E00E9482394A
:10B410008AE00E946A392091440B3091450B40919B
:10B42000460B5091470B27966CAD7DAD8EAD9FAD11
:10B4300027970E94FCE181110C9476472091480BDC
:10B440003091490B40914A0B50914B0BC301B20113
:10B450000E94FCE181110C94764720914C0B3091B5
:10B460004D0B40914E0B50914F0B2B966CAD7DAD1B
:10B470008EAD9FAD2B970E94FCE181110C94764715
:10B480000C94FC4783EB98E0C1CFC11003C00FEFD1
:10B490000C94804E0E947A1C209101063091020685
:10B4A00040910306509104060E94F2E820E030E04B
:10B4B00040E252E40E94F2E820E030E046E951E444
:10B4C0000E94F3E82EE034E74AED5CE30E9462E27A
:10B4D0000E94E8E9062F653010F40C94804ED7CF17
:10B4E000F11003C01FEF0C948F4E0E947A1C209124
:10B4F00005063091060640910706509108060E9405
:10B50000F2E820E030E040E252E40E94F2E820E07D
:10B5100030E046E951E40E94F3E82EE034E74AEDDA
:10B520005CE30E9462E20E94E8E9162F653010F4A5
:10B530000C948F4ED7CF07FD02C017FF08C00E94A2
:10B54000433A8CE099E00E9482390C94FC470E94B7
:10B550007A1CE02E000FFF08A12F110FBB0B20E07B
:10B5600030E0A901BB2091F025E02E9DF0012F9D38
:10B57000F00D1124EA0FFB1FEE0FFF1FEE0FFF1F50
:10B58000E95FFB4F2081318142815381E5E0EE9DEF
:10B590008001EF9D100D11240A0F1B1F000F111FBA
:10B5A000000F111F095F1B4F0E94F3E8D8016D9334
:10B5B0007D938D939C9313970C94FC470E94EBBA58
:10B5C00081110C94FC4798E6C92E96E1D92EE4E44B
:10B5D000FBE0F9A7E8A79E012F5F3F4F1901790112
:10B5E00010E000E0F6016591759185919491A8A510
:10B5F000B9A58D909D90AD90BD90B9A7A8A7A501C4
:10B6000094010E94F2E82B013C01F7014082518233
:10B610006282738220E030E040EA51EC0E9476EAD8
:10B6200087FD0AC020E030E040EA51E4C301B201E6
:10B630000E94FCE1181684F4F801E654F94DE491F7
:10B640001E1654F4B7FAB094B7F8B094D7018D929F
:10B650009D92AD92BC921397F70181909190A19029
:10B66000B1907F0120E030E040EA51ECC501B40127
:10B670000E9476EA87FD3FC020E030E040EA51E4D6
:10B68000C501B4010E94FCE11816ACF10F5F1F4F19
:10B69000F4E0CF0ED11C0330110509F0A3CF85E9EA
:10B6A000E82E85E0F82E10E0F10181919191A191B1
:10B6B000B1911F01F70181939193A193B1937F0100
:10B6C000812F0E942B851F5F133071F70E94148E0B
:10B6D00060E085E499E00E94771F63E972E084E608
:10B6E00090E00E949A946AEB72E084E690E00E94F7
:10B6F0009A940C94FC470E94433A83E699E00E9496
:10B70000823961E085E599E00E94771F0E946D1DF6
:10B7100068E270E088EC90E00E949A940C94FC47F8
:10B720000E9458A60C94FC470E941C8F0C94FC4766
:10B7300081E080936F040E944CA610926F048823CE
:10B7400011F40C94FC470E94473A81E899E00E946A
:10B7500082390C94FC4783FD02C00C94FC470E9484
:10B76000F8CB0C94FC4781E08093A40510929612CC
:10B7700060E083E50E94753081110C94FC470E94C3
:10B7800093B80C94FC470E942DD281110C94FC4775
:10B790000C94024F109145030E9482C16093E8050A
:10B7A0007093E9058093EA059093EB05112311F45A
:10B7B0000C94FC470E94473A84E50E946A39812F25
:10B7C0000E9494C780E20E946A398CEA99E00E9444
:10B7D00082390C94FC4783E50E945A30882311F487
:10B7E0000C94FC470E94761C0C94544C83E50E94F8
:10B7F0005A30882311F40C94BF510E94661C8B01AF
:10B800000C94BF5183E50E945A30882311F40C94A4
:10B81000FC470E94761C0C943C5283E50E945A30EF
:10B820008CAB811107C082E50E945A30882311F445
:10B830000C94FC470E94761C0C946952F1100C94F5
:10B840002D4A90E1E4E4FBE0ADEEB3E001900D920F
:10B850009A95E1F70C943B4A80E001110C940C4757
:10B8600080E1E4E4FBE0ADEEB3E001900D928A9557
:10B87000E1F70C94614A4F925F926F927F928F92A0
:10B880009F92AF92BF92CF92DF92EF92FF920F936F
:10B890001F93CF93DF93CDB7DEB77C014DB65EB675
:10B8A0006090F1057090F2058DB69EB66AE070E08A
:10B8B000C7010E943EE16C018C010E191F09892B02
:10B8C00021F4C7010E9449E18C01C80101962DB7FE
:10B8D0003EB7281B390B0FB6F8943EBF0FBE2DBFE5
:10B8E0008DB79EB701965C01A801B7010E946AE17D
:10B8F000F501E00FF11F1082C5010E94302F81E099
:10B900000E944746C114D10451F076019FEFE91A15
:10B91000F90A0FB6F8949EBE0FBE8DBEC5CF0FB606
:10B92000F8949EBE0FBE8DBEC3010E94302F0FB68D
:10B93000F8945EBE0FBE4DBEDF91CF911F910F9167
:10B94000FF90EF90DF90CF90BF90AF909F908F903F
:10B950007F906F905F904F9008954F925F926F929B
:10B960007F928F929F92AF92BF92CF92DF92EF928F
:10B97000FF920F931F93CF93DF93CDB7DEB7289736
:10B980000FB6F894DEBF0FBECDBF83E50E9440BB6B
:10B99000863028F087E295E00E94823949C08330E2
:10B9A00009F46EC1E8F4813071F1823009F45AC0B3
:10B9B00084E195E00E9482390E94BB308823F1F037
:10B9C00080910104811117C083EB98E00E948239B5
:10B9D0008AE00E946A390E94A9390E94148E28C008
:10B9E000843009F493C1853019F780E00E949A30C1
:10B9F0000E948A30F2CF87EB98E0E8CF86E095E0AE
:10BA00000E948239EACF0E948A3010920A01109275
:10BA100009018091D203811125C08EE40E94251C6A
:10BA200081111DC084EF94E09093A2058093A1053D
:10BA300028960FB6F894DEBF0FBECDBFDF91CF9131
:10BA40001F910F91FF90EF90DF90CF90BF90AF903C
:10BA50009F908F907F906F905F904F9008958AEFA6
:10BA600094E0E2CF8091090190910A0197FF03C011
:10BA70008BEC94E091CF009709F0A8C01D821E8244
:10BA80001F8218868DEC9CECACE4BEE389839A831C
:10BA9000AB83BC83BE016B5F7F4FCE0101960E94DA
:10BAA00034868091090190910A01893191050CF049
:10BAB000B3C021E0209328019C012F5F3F4F3093BA
:10BAC0000A012093090165E00E948CE880FF03C011
:10BAD00024E0291B922F24E09202F0011124E75662
:10BAE000FA4E80809180A280B38094E08902F001B8
:10BAF0001124EB57FA4E40805180628073808DECA8
:10BB00009CECACE4BEE38D839E83AF83B88719823F
:10BB10001A821B821C82CE0101966C01E12CF12C51
:10BB200000EA10E4A3019201C501B4010E947C85E2
:10BB300019821A821B821C82B601CE0105960E94D0
:10BB400034868092440B9092450BA092460BB092A3
:10BB5000470B4092480B5092490B60924A0B7092EF
:10BB60004B0B1092D2030091090110910A0189E157
:10BB7000E82EF12C093111050CF47801B70184E6A7
:10BB800094E00E94393A69E170E08FE594E00E9408
:10BB9000393A8AE00E946A39101611060CF01DCF5E
:10BBA0001F9289E18F93FF92EF9288E494E09F9334
:10BBB0008F9386E594E09F938F931F920E945E1F60
:10BBC0000FB6F894DEBF0FBECDBF07CF815065E042
:10BBD0000E948CE880FF03C024E0291B922F25E0FF
:10BBE0009202F0011124E80FF11D87FDFA95EE0F86
:10BBF000FF1FEE0FFF1FE95FFB4F80914C0B9091F1
:10BC00004D0BA0914E0BB0914F0B80839183A2837B
:10BC1000B3831092280145CF80E090E0A0EAB0E421
:10BC200080934C0B90934D0BA0934E0BB0934F0B06
:10BC300081E291E00E9461850E949E778FEF9FEFE5
:10BC400090930A018093090187EB94E00E94823966
:10BC500085EA94E00E9459B863E972E084E690E0D6
:10BC60000E949A946AEB72E084E690E00E949A94B3
:10BC70008FE994E00E943B5C81E00E949A3071CF92
:10BC800089E40E945A30882371F00E94761C182F94
:10BC9000853068F064E070E08CE894E00E94393A06
:10BCA00089E894E079CE8AE40E94A339C1CE8AE47F
:10BCB0000E945A308823B9F30E94761C082F8530E1
:10BCC00048F064E070E086E794E00E94393A83E748
:10BCD00094E062CE8AE50E945A308823A9F00E943F
:10BCE0007A1C25E01202F0011124E00FF11D07FD7E
:10BCF000FA95EE0FFF1FEE0FFF1FE95FFB4F60830A
:10BD000071838283938369CE8AE5CECF8AE50E94D0
:10BD10005A308823C9F30E947A1C60936B04709395
:10BD20006C0480936D0490936E0457CECF93DF9391
:10BD3000C0913E0C81E6C89FE0011124C05CD34F46
:10BD40008091FB0A80FF05C00E94473ACE010E9405
:10BD50007139CE010E94302F80E0DF91CF910C9499
:10BD600047460F931F93CF93DF93CDB7DEB760970E
:10BD70000FB6F894DEBF0FBECDBF8C01DC01ED9194
:10BD8000FC910280F381E02DBE016F5F7F4F09952A
:10BD9000882309F464C08981807CC9F56F81637050
:10BDA00070E0762F6627770F770F8885B4E08B9F3A
:10BDB000C0011124682B792B8985829586958695FB
:10BDC0008370682B6F5F7F4F90E080E02A8523703F
:10BDD000220F3B8537FB332730F9232B3E813F7001
:10BDE000230F3327331F2750310904C0660F771FF5
:10BDF000881F991F2A95D2F760960FB6F894DEBF78
:10BE00000FBECDBFDF91CF911F910F910895803468
:10BE100019F568856695669570E090E080E0CB0145
:10BE2000772766272A85622B098510E0102F0027C7
:10BE3000012E000C220B330B602B712B822B932BCA
:10BE40006F5F7F4F8F4F9F4F4AE0660F771F881FAE
:10BE5000991F4A95D1F7D0CF8BE0F801848360E039
:10BE600070E0CB01C9CF0895FC0182810895CF9283
:10BE7000DF92EF92FF9280910604882309F457C065
:10BE8000C0900204D0900304E0900404F0900504F4
:10BE900020E030E0A901C701B6010E94FCE188233F
:10BEA00009F445C020E030E040E05FE3C701B6019F
:10BEB0000E9462E29B01AC010E9462E22BED3FE036
:10BEC00049E450E40E9462E29B01AC0160E070E052
:10BED00080E89FE30E9476E96B017C01C092FD033C
:10BEE000D092FE03E092FF03F092000460912501DE
:10BEF00070912601072E000C880B990B0E9403E21B
:10BF00002AE037ED43E25CE30E9462E2A70196017A
:10BF10000E9462E2609358017093590180935A0124
:10BF200090935B01FF90EF90DF90CF900895C12C2C
:10BF3000D12C80E8E82E8FE3F82ED0CF2F923F92BD
:10BF40004F925F926F927F928F929F92AF92BF9229
:10BF5000CF92DF92EF92FF920F931F93CF93DF93D5
:10BF6000CDB7DEB766970FB6F894DEBF0FBECDBF74
:10BF7000DC01CD90DD90ED90FC90139714962D91FF
:10BF80003D914D915C9117972B873C874D875E873C
:10BF900020E030E040E252E4C701B6010E94F2E83E
:10BFA0002EE034E74AED5CE30E9462E20E94E8E999
:10BFB00064300CF428C163E0662E660F7708F30145
:10BFC000EE0FFF1FEE0FFF1FE756FA4E80809180A5
:10BFD000A280B380F3013196FA83E98320E030E058
:10BFE00040E252E46B857C858D859E850E94F2E857
:10BFF0002EE034E74AED5CE30E9462E20E94E8E949
:10C0000064300CF404C163E0062F660F110BF801D5
:10C01000EE0FFF1FEE0FFF1FE756FA4E2081318112
:10C02000428153812B833C834D835E83A8014F5F04
:10C030005F4F5E8B4D8BA5E0A69DC001A79D900D27
:10C040001124988B8F87FC01E00FF11FEE0FFF1F6B
:10C05000EE0FFF1FE95FFB4F208131814281538149
:10C060002F83388749875A87E981FA81EE0FFF1FAE
:10C07000EE0FFF1FE756FA4EA50194016081718112
:10C08000828193810E94F2E8698B7A8B8B8B9C8BE7
:10C09000A5019401C701B6010E94F2E82B013C0101
:10C0A00085E049815A81849F1001859F300C1124BD
:10C0B000F101E00FF11FEE0FFF1FEE0FFF1FE95F11
:10C0C000FB4F2F81388549855A8560817181828136
:10C0D00093810E94F2E829893A894B895C890E9400
:10C0E00076E9A30192010E9462E22F813885498599
:10C0F0005A850E94F3E86B017C01EF85F889AD89D0
:10C10000BE89EA0FFB1FEE0FFF1FEE0FFF1FE95F57
:10C11000FB4F80809180A280B380FD01E20DF31D72
:10C12000EE0FFF1FEE0FFF1FE95FFB4FA50194010C
:10C1300060817181828193810E94F2E829893A8924
:10C140004B895C890E9476E9A30192010E9462E218
:10C15000A50194010E94F3E8A70196010E94F2E86C
:10C160004B015C01ED89FE89EE0FFF1FEE0FFF1FF3
:10C17000E756FA4E2B813C814D815E816081718151
:10C18000828193810E94F2E89B01AC01C501B40158
:10C190000E9476E94B015C012B813C814D815E81DF
:10C1A0006B857C858D859E850E94F2E89B01AC01A4
:10C1B000C501B4010E9462E2A70196010E94F3E862
:10C1C00020916B0430916C0440916D0450916E0489
:10C1D0000E94F3E866960FB6F894DEBF0FBECDBF9F
:10C1E000DF91CF911F910F91FF90EF90DF90CF9053
:10C1F000BF90AF909F908F907F906F905F904F9087
:10C200003F902F90089567FFD7CE60E0D5CE67FFAF
:10C21000FBCE60E0F9CE8F929F92AF92BF92CF9209
:10C22000DF92EF92FF92FC01C080D180E280F38028
:10C2300020E030E040E251E4C701B6010E9462E232
:10C2400020E030E040E251E40E9462E24B015C01F8
:10C2500020E030E0A901C701B6010E94FCE120E026
:10C2600030E040EA50E487FF04C020E030E040EADC
:10C2700050ECC501B4010E94F3E820E030E040E258
:10C2800051E40E9476E90E94E8E99B018BE237FFC6
:10C2900005C022273327261B370B8DE28093D60358
:10C2A000C90168EE73E00E94AEE8CB01EAE0F0E07D
:10C2B000BF010E94AEE8805D8093D703C90164E6A8
:10C2C00070E00E94AEE8CB01BF010E94AEE8805D45
:10C2D0008093D803C901BF010E94AEE8282FCB018B
:10C2E000BF010E94AEE8805D8093D9038EE2809307
:10C2F000DA03205D2093DB0386ED93E0FF90EF905F
:10C30000DF90CF90BF90AF909F908F90089524E6DC
:10C31000829FC001112481589F4F6FEF70E00E94EF
:10C32000AEE8262F81E3643609F080E28093D803DB
:10C3300090E22A3040F03AE0822F632F0E9480E89A
:10C340000E9480E8905D9093D903822F6AE00E945A
:10C3500080E8905D9093DA0385E28093DB0388EDBB
:10C3600093E008956091250170912601072E000C3D
:10C37000880B990B0E9403E22AE037ED43E25CE36D
:10C380000E9462E22091FD033091FE034091FF0381
:10C39000509100040E9462E2609358017093590129
:10C3A00080935A0190935B0108958091E505811176
:10C3B00004C08091C0058093370608958091BB1614
:10C3C0008823C1F081508093BB16EEEEF4E1882300
:10C3D00051F08150990B2BE1289FF001299FF00D1E
:10C3E0001124E355FA4E8BE1A3EDB4E101900D92D7
:10C3F0008A95E1F72091BB16211105C08091C616E0
:10C4000080628093C61681E090E0A0E0B0E0211148
:10C4100003C080E090E0DC018093CE059093CF05CF
:10C42000A093D005B093D1051092C70581E0809309
:10C43000DE0583E0809353010895CF93DF93EC01F1
:10C44000CB01BA010E9403E220E030E0A9010E9482
:10C45000F3E80E94E8E979836883DF91CF9108953A
:10C46000CF93DF93EC01CB01BA010E9403E229ECE8
:10C4700038EC48EC5EE30E9476E920E030E040E0F2
:10C480005FE30E94F3E80E94EFE96883DF91CF91B8
:10C4900008950E9403E229EC38EC48EC5EE30E9428
:10C4A00076E920E030E040E05FE30E94F3E80E949C
:10C4B000EFE9862F0C948761E091E50586E0E802BC
:10C4C000F0011124E255FA4F8091C00590E0958368
:10C4D000848308952091AB053091AC052115310579
:10C4E000E9F08091A9059091AA050296245031099E
:10C4F000821793079CF49093100580930F050E9478
:10C5000082C1605E70448D4F9F4F609311057093A0
:10C510001205809313059093140508951092110548
:10C520001092120510921305109214050895CF93DE
:10C53000DF93EC018D810E94C93B60E08B81DF912C
:10C54000CF910C948BC0DF92EF92FF920F931F93C9
:10C55000CF93DF938C01C62FD22FF32EE42ED52E4E
:10C560000E9497620E9401C28C2F80640E94BD3B92
:10C570008D2D0E94BD3B8E2D0E94BD3B8F2D0E94B4
:10C58000BD3B8D2F0E94BD3B87E8C11101C085E9ED
:10C590000E94BD3BCC3011F40E94C23BC0E00E941F
:10C5A000C23BF801868387FF04C0CF3F11F0CF5F05
:10C5B000F6CFDF91CF911F910F91FF90EF90DF9019
:10C5C000089561E0FC0183810E948BC08FEF0C9481
:10C5D000BD3B0F931F93CF938C010E9497620E94E3
:10C5E00001C2C82F882371F08DEF0E94BD3B0E94CD
:10C5F00001C2C82FC8010E94E1628C2FCF911F9108
:10C600000F91089582E1F8018483F4CF8F929F9275
:10C61000AF92BF92CF92DF92EF92FF920F931F9350
:10C62000CF93DF93EC016A017B01590120E030E0F8
:10C63000A90167E30E94A362A501980167E1CE0109
:10C640000E94A362811127C08F81833039F089E075
:10C65000CC0CDD1CEE1CFF1C8A95D1F7A7019601BE
:10C6600069E1CE010E94A36211E0882319F010E075
:10C6700087E08C83CE010E94E162812FDF91CF9110
:10C680001F910F91FF90EF90DF90CF90BF90AF90F0
:10C690009F908F90089589E08C8310E0EBCFCF932B
:10C6A000DF93EC016EBDFA01CA019E5F0DB407FE77
:10C6B000FDCF20812EBD0DB407FEFDCF21812EBD03
:10C6C0003296E817F90791F70DB407FEFDCF8FEF0B
:10C6D0000E94BD3B8FEF0E94BD3B0E94C23B8E83F8
:10C6E0008F71853049F083E18C83CE010E94E16235
:10C6F00080E0DF91CF91089581E0FBCF0F931F93EE
:10C70000CF93DF93EC018B010E9497620E9401C2DC
:10C7100081110CC085E18C8310E0CE010E94E162A2
:10C72000812FDF91CF911F910F910895A8016CEF98
:10C73000CE010E944F63182F882361F3EECF0F9331
:10C740001F93CF93DF93EC0189018F81833039F000
:10C7500089E0440F551F661F771F8A95D1F79A010C
:10C76000AB0168E1CE010E94A36281112AC0A80139
:10C770006EEFCE010E944F63182F8823B1F00E9404
:10C7800001C2182F8823D1F020E030E0A9016DE02C
:10C79000CE010E94A362882321F086E18C8310E001
:10C7A00004C00E94C23B8111F8CFCE010E94E16219
:10C7B000812FDF91CF911F910F91089587E18C8395
:10C7C000F4CF86E0EBCF1F93CF93DF93EC010E9471
:10C7D000976220E030E0A9016CE0CE010E94A362E4
:10C7E00011E0882319F010E083E08C83CE010E94D1
:10C7F000E162812FDF91CF911F9108951F93CF9315
:10C80000DF93EC018F81833039F089E0440F551FAD
:10C81000661F771F8A95D1F79A01AB0162E1CE01BD
:10C820000E94A36211E0882319F010E085E08C8358
:10C83000CE010E94E162812FDF91CF911F91089577
:10C840008F929F92AF92BF92EF92FF920F931F939E
:10C85000CF93DF938C01EB017A010E9482C14B01DF
:10C860005C012CE2820E21E0921EA11CB11C0E94F0
:10C87000C23BF80186838F3F69F40E9482C1681928
:10C8800079098A099B0997FDF2CF81E1F801848338
:10C89000C0E021C08E3F71F5F1E0EF1AF1088FEF93
:10C8A0008EBDFE012FEF0DB407FEFDCF8EB5819337
:10C8B0002EBDCF018C1B9D0B8E159F05A0F30DB4D3
:10C8C00007FEFDCF8EB5CE0DDF1D88830E94C23BD3
:10C8D0000E94C23BC1E0C8010E94E1628C2FDF913F
:10C8E000CF911F910F91FF90EF90BF90AF909F90CD
:10C8F0008F9008958FE0CACF0F931F93CF93DF934C
:10C90000EC018B010E94976240E052E0B801CE0139
:10C91000DF91CF911F910F910C9420640F931F937F
:10C92000CF93DF93EC0189018F81833039F089E067
:10C93000440F551F661F771F8A95D1F79A01AB01E7
:10C9400061E1CE010E94A36281110AC040E052E081
:10C95000B801CE01DF91CF911F910F910C9420640B
:10C9600084E08C83CE010E94E16280E0DF91CF9170
:10C970001F910F9108958F929F92AF92BF92CF9285
:10C98000DF92EF92FF920F931F93CF93DF93EC010F
:10C99000162F1F821C824B830E9482C16B017C0177
:10C9A00020EDC20E27E0D21EE11CF11CA89561E02B
:10C9B0008B810E948BC08B810E943AB8249A2C9A5A
:10C9C000279A2698259A81E00E94C93B85E08D83AD
:10C9D0000E94C93B0AE08FEF0E94BD3B0150D9F78E
:10C9E000A89520E030E0A90160E0CE010E94A3629A
:10C9F0008E83813081F00E9482C16C197D098E097D
:10CA00009F0997FDEECF81E08C83CE010E94E16209
:10CA10001A8280E06AC0A8952AEA31E040E050E03E
:10CA200068E0CE010E94A362853041F581E08F83EA
:10CA3000A8958F81812C912C5401823029F4812C6E
:10CA4000912CA12C80E4B82E20E030E0A90167E30E
:10CA5000CE010E94A362A501940169E2CE010E9469
:10CA6000A3628E838823F1F00E9482C16C197D0934
:10CA70008E099F0997FDE8CF8AE0C6CF04E00E94A7
:10CA8000C23B8E830150D9F78A3A11F482E0CFCFAE
:10CA90000E9482C16C197D098E099F0997FDBCCF48
:10CAA00082E0B2CF8F818230C1F420E030E0A90172
:10CAB0006AE3CE010E94A362882311F088E0A4CF2C
:10CAC0000E94C23B807C803C11F483E08F830E94F3
:10CAD000C23B0E94C23B0E94C23BCE010E94E16267
:10CAE00081E08A83173070F41D83DF91CF911F910D
:10CAF0000F91FF90EF90DF90CF90BF90AF909F90FD
:10CB00008F90089588E18C8384CF0F931F93CF93E8
:10CB1000DF93EC018B0120E030E0A90169E00E9485
:10CB2000A36281110AC040E150E0B801CE01DF915B
:10CB3000CF911F910F910C94206480E18C83CE01E2
:10CB40000E94E16280E0DF91CF911F910F910895E3
:10CB5000CF93C82FCB010E9482398FEF95E10E94BD
:10CB6000823980EF95E1CC2311F085EF95E10E94A9
:10CB700082398AE0CF910C946A390C948EC10C945E
:10CB80008EC140916F0421E042276CE070E00C946C
:10CB9000E1B940916F0421E0422764E070E00C9419
:10CBA000E1B940916F0421E0422761E070E00C940C
:10CBB000E1B940916F0421E0422762E070E00C94FB
:10CBC000E1B940916F0421E0422761E070E00C94EC
:10CBD000E1B940916F0421E0422768E070E00C94D5
:10CBE000E1B940916F0421E042276CE070E00C94C1
:10CBF000E1B941E061E070E00C94E1B940916F046B
:10CC000021E042270C94E1B962E070E00C941AC173
:10CC10006CE070E00C941AC164E070E00C941AC1EE
:10CC200061E070E00C941AC161E070E00C941AC1EC
:10CC30006CE070E00C941AC10F931F93CF93811195
:10CC400013C0C42F8B010E94473A8DEE96E10E94DB
:10CC50008239C8010E948239CC2331F08AE0CF9119
:10CC60001F910F910C946A39CF911F910F910895E4
:10CC7000CF93DF9380911E1590911F15891B80958E
:10CC80008F7019F40E941340F5CF80911E158F5FAD
:10CC90008F70A0911E159BE4A99FD0011124FD0166
:10CCA000E55BF94FEF0119929A95E9F798E09083C7
:10CCB000A05AB94F90E1E0E2F5E101900D929A950A
:10CCC000E1F720911E1590911F15291303C094E6DA
:10CCD00090931B1580931E15DF91CF910C94E33038
:10CCE00020E040E070E060E088E397E60E94B21C3C
:10CCF00081E08093C6051092EF051092EE0508952D
:10CD000020E040E070E060E08EE499E60C94B21C14
:10CD100080914806811114C080915C0190915D0161
:10CD200001972091A5143091A6142817390744F4CF
:10CD300020E040E070E060E083E599E60C94B21CEE
:10CD40000C94806621E02093C605FC0180819181CE
:10CD5000A281B38180931B0190931C01A0931D01BC
:10CD6000B0931E0120E040E070E060E08091BE05DD
:10CD70009091BF050C94B21CCF93DF9300D000D0EC
:10CD8000CDB7DEB78DEC9CECACECBCE389839A8329
:10CD9000AB83BC83CE0101960E94A2660F900F90D8
:10CDA0000F900F90DF91CF910895CF93DF9300D034
:10CDB00000D0CDB7DEB78DEC9CECACECBDE3898345
:10CDC0009A83AB83BC83CE0101960E94A2660F902A
:10CDD0000F900F900F90DF91CF910895CF93DF9335
:10CDE00000D000D0CDB7DEB780E090E0A0E8BFE390
:10CDF00089839A83AB83BC83CE0101960E94A2668D
:10CE00000F900F900F900F90DF91CF910895CF93D7
:10CE1000DF9300D000D0CDB7DEB780E090E0A0E295
:10CE2000B1E489839A83AB83BC83CE0101960E94CF
:10CE3000A2660F900F900F900F90DF91CF91089501
:10CE400081E08093C6051092940510927E0420E044
:10CE500040E070E060E089EE9BE60E94B21C8AE44C
:10CE600095E19093A2058093A10508950C94861DE9
:10CE70008F929F92AF92BF92CF92DF92EF92FF92EA
:10CE8000CF938091C4051092C405882369F0109255
:10CE9000C605CF91FF90EF90DF90CF90BF90AF90FD
:10CEA0009F908F900C94861D4091CE055091CF0598
:10CEB0006091D0057091D10541155105610571054D
:10CEC00099F01092CE051092CF051092D0051092D5
:10CED000D10581E0809353012AE0249FC001259F62
:10CEE000900D11240E94BBC180915301882309F445
:10CEF000AEC06091EE057091EF05072E000C880B17
:10CF0000990B0E9403E22091400630914106409126
:10CF10004206509143060E9462E26B017C0120E0D0
:10CF200030E040E251E40E9462E220E030E04AE773
:10CF300054E40E9462E24B015C0120E030E0A90170
:10CF4000C701B6010E94FCE120E030E040EA50E475
:10CF500087FF04C020E030E040EA50ECC501B40196
:10CF60000E94F3E820E030E040E251E40E9476E9DC
:10CF70000E94E8E96B017C018BE2F7FE09C0F094A6
:10CF8000E094D094C094C11CD11CE11CF11C8DE232
:10CF90008093D503C701B60120E137E240E050E0BD
:10CFA0000E94C2E88AE0882E912CA12CB12CCA01E3
:10CFB000B901A50194010E94C2E8605D6093D603A7
:10CFC000C701B60128EE33E040E050E00E94C2E81D
:10CFD000CA01B901A50194010E94C2E8605D609395
:10CFE000D7038EE28093D803C701B60124E630E070
:10CFF00040E050E00E94C2E8CA01B901A5019401D5
:10D000000E94C2E8605D6093D903C701B601A50123
:10D0100094010E94C2E8C62FCA01B901A50194017A
:10D020000E94C2E8605D6093DA03C05DC093DB03D9
:10D0300065ED73E08CEA95E1CF91FF90EF90DF9082
:10D04000CF90BF90AF909F908F900C948C23CF91F6
:10D05000FF90EF90DF90CF90BF90AF909F908F9018
:10D0600008956FEF8091C0050C9441C04F925F927C
:10D070006F927F928F929F92AF92BF92CF92DF92E8
:10D08000EF92FF920F931F93CF93DF930091C00510
:10D090000E9495BDC091C70510E0000F111F0558F3
:10D0A0001A4E95E0592E5C0E21E6E22E25E1F22E75
:10D0B000D3E0DC1B31E3C32E38E6D32E43E5A42EA8
:10D0C00045E1B42E82E0782E7C1A58E8852E55E191
:10D0D000952E81E0682E6C1A4C2E4194C11137C0F8
:10D0E0008091C9058823B1F080915301882359F0BC
:10D0F00081E09091C905911180E024E04FE655E16F
:10D10000642D0E9469BCCF5F5C12E8CF84E08093FD
:10D11000C8050CC08091C4051092C405882321F372
:10D120000E94861D8091DE058823F1F2DF91CF9168
:10D130001F910F91FF90EF90DF90CF90BF90AF9035
:10D140009F908F907F906F905F904F900895C13027
:10D1500059F5F801859194919093E7058093E60540
:10D160008091C905813081F080915301882359F263
:10D170001F929F928F926F9281E09091C90591309A
:10D1800009F474C080E072C08091C4051092C40597
:10D19000882351F38091C005682F0E9441C080917F
:10D1A000DE05882309F3C2CFC23009F042C0F8017E
:10D1B000859194919093E7058093E6058091C90548
:10D1C0008230D1F080915301882309F49CCFDF9203
:10D1D000CF92BF92AF927F9281E09091C905923039
:10D1E00009F080E08F930E94A41C0F900F900F9085
:10D1F0000F900F900F9087CF8091C4051092C405B7
:10D20000882301F30E9431688091DE058823D1F2E2
:10D210008DCF8091C4051092C4058823C1F0609120
:10D22000C0058FEF0E9441C08091DE05882379F010
:10D230007DCFC33009F067CFF80185919491909329
:10D24000E7058093E6058091C905833011F380914D
:10D250005301882309F457CF1F92FF92EF92DF9377
:10D2600081E09091C905933009F08CCF8F930E9493
:10D27000A41C0F900F900F900F900F9044CF6EEC66
:10D280007BE682E00C946ED463ED7BE681E00C9447
:10D290006ED468ED7BE680E00C946ED465E879E6A8
:10D2A00083E00C946ED4EF92FF920F931F9388EF5C
:10D2B000E82E84E1F82E0AEF14E126E337E640E891
:10D2C00056E66AE075E18FE095E10E94A0C41F91E7
:10D2D0000F91FF90EF900895EF92FF920F931F939D
:10D2E0008AE3E82E84E1F82E0DEA14E126E337E61E
:10D2F0004EED5FE16CE374E181E494E10E94A0C42F
:10D300001F910F91FF90EF900895CF93DF9300D07E
:10D3100000D0CDB7DEB78091C4051092C405882334
:10D3200059F01092C6050E94861D0F900F900F9025
:10D330000F90DF91CF9108956091CE057091CF0548
:10D340008091D0059091D1056115710581059105F8
:10D3500061F10E9403E220911B0130911C01409178
:10D360001D0150911E010E9462E22091500B3091EC
:10D37000510B4091520B5091530B0E94F3E8609374
:10D38000500B7093510B8093520B9093530B83E08F
:10D390000E94432081E0809353011092CE051092A9
:10D3A000CF051092D0051092D105809153018823AA
:10D3B00009F4BBCF2091BA053091BB054091BC0563
:10D3C0005091BD056091500B7091510B8091520BA3
:10D3D0009091530B0E94F2E869837A838B839C833C
:10D3E000CE0101960E940B61BC018BE896E20E947F
:10D3F0008C239BCF2F923F924F925F926F927F929E
:10D400008F929F92AF92BF92CF92DF92EF92FF9254
:10D410001F93CF93DF93CDB7DEB72C970FB6F89459
:10D42000DEBF0FBECDBF1C01162F8091C405109228
:10D43000C4058823E1F01092C6050E94861D2C9633
:10D440000FB6F894DEBF0FBECDBFDF91CF911F9115
:10D45000FF90EF90DF90CF90BF90AF909F908F9014
:10D460007F906F905F904F903F902F9008958091A4
:10D47000CE059091CF05A091D005B091D1058D83B7
:10D480009E83AF83B887892B8A2B8B2B09F460C0CE
:10D4900080912701882309F4BDC080912801811162
:10D4A000B9C0613009F494C0623009F4A2C0809020
:10D4B000290190902A01A0902B01B0902C01C090DE
:10D4C0003501D0903601E0903701F0903801612E9F
:10D4D000712C6D817E818F8198850E9403E220915D
:10D4E0001B0130911C0140911D0150911E010E94B1
:10D4F00062E2D301AA0FBB1FAA0FBB1FBC87AB8779
:10D50000AC5BB44FBA87A9872D913D914D915C9149
:10D510000E94F3E82B013C018D819E81AF81B8858B
:10D52000B7FF8FC0A5019401C301B2010E94FCE1C5
:10D5300087FD7FC0EB85FC85EC5BF44F4082518218
:10D5400062827382812F0E94432081E08093530185
:10D550001092CE051092CF051092D0051092D105F1
:10D5600080915301882309F46ACFF4E01F9FC00122
:10D570001124FC01EC5BF44F8F5F994FDC012D917E
:10D580003D914D915C9160817181828193810E9476
:10D59000F3E86B017C01C982DA82EB82FC822DEC1C
:10D5A0003CEC4CEC5DE360911B0170911C0180919F
:10D5B0001D0190911E010E9476EA87FD52C0CE01A6
:10D5C00001960E940B61BC01C1010E948C2337CFE0
:10D5D00080902D0190902E01A0902F01B0903001ED
:10D5E000C0903901D0903A01E0903B01F0903C01AD
:10D5F0006ECF8090310190903201A0903301B090B5
:10D600003401C0903D01D0903E01E0903F01F09088
:10D6100040015DCF812C30E5932E33ECA32E37EC07
:10D62000B32EC12C40E5D42E43ECE42E47E4F42E77
:10D630004ECFA985BA858D929D92AD92BC921397DB
:10D6400081CFA7019601C301B2010E9476EA1816A4
:10D650000CF070CFE985FA85C082D182E282F38234
:10D6600071CF20E030E040E251E4C701B6010E94F2
:10D6700062E220E030E04AE754E40E9462E24B01BB
:10D680005C0120E030E0A901C701B6010E94FCE185
:10D6900020E030E040EA50E487FF04C020E030E0C2
:10D6A00040EA50ECC501B4010E94F3E820E030E00C
:10D6B00040E251E40E9476E90E94E8E96B017C01B6
:10D6C000F7FC62C020EA36E841E050E00E94C2E880
:10D6D000CA01B9012AE030E040E050E00E94C2E80F
:10D6E000605D6093D503C701B60120E137E240E0F9
:10D6F00050E00E94C2E88AE0882E912CA12CB12C27
:10D70000CA01B901A50194010E94C2E8605D60935D
:10D71000D603C701B60128EE33E040E050E00E9496
:10D72000C2E8CA01B901A50194010E94C2E8605D86
:10D730006093D7038EE28093D803C701B60124E635
:10D7400030E040E050E00E94C2E8CA01B901A50102
:10D7500094010E94C2E8605D6093D903C701B601DD
:10D76000A50194010E94C2E8162FCA01B901A501C2
:10D7700094010E94C2E8605D6093DA03105D10932B
:10D78000DB0385ED93E01FCFF094E094D094C09438
:10D79000C11CD11CE11CF11C6DE2A3CF62E084E945
:10D7A00096E20C94FA6961E08BE996E20C94FA69CE
:10D7B00060E082EA96E20C94FA696DE172E683E930
:10D7C00092E90C94CC2460E372E689E492E60C942E
:10D7D000CC2480915301882331F041E060E773E16C
:10D7E00082E00E940CBC80917E048770873041F4F7
:10D7F00020E040E070E060E08FE690EA0C94B21C1C
:10D8000008950F931F93CF93DF93CDB7DEB72A9779
:10D810000FB6F894DEBF0FBECDBF809153018823B1
:10D82000F1F01F9289E18F938091D30390E00196EC
:10D830009F938F938DE493E19F938F938E010F5F5E
:10D840001F4F1F930F930E9493E1B80182E493E16D
:10D850000E948C230FB6F894DEBF0FBECDBF84E0CC
:10D86000809353018091D203811108C020E040E0F1
:10D8700070E060E08BE094E20E94B21C2A960FB642
:10D88000F894DEBF0FBECDBFDF91CF911F910F91F6
:10D890000895CF93DF93EC010E94C3CB1B82DF91ED
:10D8A000CF910895CF93DF93EC01462F41706C85A3
:10D8B0007D858E859F850E9490C8882351F0888938
:10D8C00020E2829FC001112489569D4EDF91CF91A5
:10D8D000089590E080E0FACFCF93DF93EB01FC0155
:10D8E0002381211104C080E0DF91CF91089522505F
:10D8F000223028F48FE28883198281E0F5CF60E03E
:10D900000E94526C009779F3DC0160E080E09EE2B7
:10D910002D91203299F0883031F49E01260F311D6F
:10D92000F90190836F5F9E01260F311DAD014150BB
:10D930005109FA014081F90140836F5F8F5F8B309D
:10D9400039F7FE01E60FF11D1082D7CF3F924F92BB
:10D950005F926F927F928F929F92AF92BF92CF927F
:10D96000DF92EF92FF920F931F93CF93DF93CDB788
:10D97000DEB72C970FB6F894DEBF0FBECDBF5C01AB
:10D98000DC0159968D909C90F40181859285A38548
:10D99000B4859C01AD012F5F3F4F4F4F5F4F2987EB
:10D9A0003A874B875C87D50114964D905D906D90BA
:10D9B0007C901797411451046104710409F459C013
:10D9C000BFEF4B1A5B0A6B0A7B0A312C73016201B1
:10D9D0001D821E821F821886F40181859285A3858F
:10D9E000B4852D813E814F815885281739074A0714
:10D9F0005B0708F056C089859A85AB85BC858C1578
:10DA00009D05AE05BF0550F482E0C82ED12CE12C57
:10DA1000F12C92E0492E512C612C712C9E012F5F2C
:10DA20003F4FB701A601C4010E94CACA8823C9F1A9
:10DA300089819A81AB81BC81892B8A2B8B2B01F147
:10DA4000260137019FEF491A590A690A790A2D817F
:10DA50003E814F8158852F5F3F4F4F4F5F4F2D8342
:10DA60003E834F8358873FEFC31AD30AE30AF30A72
:10DA7000B3CF408051806280738033243394A6CF2B
:10DA8000C414D504E604F70411F70FEF1FEF2FEFCE
:10DA90003FE0B701A601C4010E9438CA782E811167
:10DAA0001AC0712C872D2C960FB6F894DEBF0FBECE
:10DAB000CDBFDF91CF911F910F91FF90EF90DF903D
:10DAC000CF90BF90AF909F908F907F906F905F901E
:10DAD0004F903F900895F50144815581668177818B
:10DAE000411551056105710539F097018601C401A1
:10DAF0000E9438CA8823A9F2D5011496CD92DD92EE
:10DB0000ED92FC921797332051F0D701C601019690
:10DB1000A11DB11DF40180839183A283B383F5011C
:10DB200085899689A789B08D892B8A2B8B2B09F043
:10DB3000B9CFC58AD68AE78AF08E818180688183D1
:10DB4000B1CF40E050E0BA010C9412CCFC0123812B
:10DB500021110C94496C08952F923F924F925F923D
:10DB60006F927F928F929F92AF92BF92CF92DF92ED
:10DB7000EF92FF920F931F93CF93DF93CDB7DEB752
:10DB8000C354D1090FB6F894DEBF0FBECDBF4C0110
:10DB90005B016A01222E19821C821C8E1F8E611568
:10DBA000710521F510E0CE014C960E94A66DCE01C4
:10DBB00001960E94A66D812FCD5BDF4F0FB6F894C2
:10DBC000DEBF0FBECDBFDF91CF911F910F91FF90B0
:10DBD000EF90DF90CF90BF90AF909F908F907F900D
:10DBE0006F905F904F903F902F900895FC0183813C
:10DBF0008111D8CFFA0180818F32A1F18B01CE0142
:10DC000001967C013C0180E2382E2E019CE1490EF8
:10DC1000511C2396EFAE23972496FFAE24972296AD
:10DC20003FAE229721963FAE21973FAE3EAE3DAE2E
:10DC30003CAE3BAE3AAE39AE38AE3FAA960190E06C
:10DC400047E0D9018D91882309F447C08F3209F448
:10DC500044C08E3209F54A3009F4A4CF98E04AE076
:10DC60009D01EFCFFB01838182508B01823060F0F8
:10DC7000618D728DCE014C960E9482D18E01045E20
:10DC80001F4F882309F48ECFC6016C010196F6015F
:10DC900020812F32D1F3B3CFEAECF2E22491222398
:10DCA00021F031968213FACF7DCF491708F47ACF4D
:10DCB000813208F477CF8F3709F474CF3FE9380FFA
:10DCC0003A3108F420EEE7E3F0E0EC0FFD1FE90F36
:10DCD000F11D820F80839F5FC3CF8FA9803209F42B
:10DCE00061CF6901F90180812F5F3F4F8F32C9F306
:10DCF000882301F121E0AE01495C5F4FB801C70103
:10DD00000E94A0D2882309F44DCF0A151B0519F0F3
:10DD1000C8010E94496C942D852D6E147F0431F04A
:10DD200023969FAD239724968FAD24978701E92EE4
:10DD3000F82E75CF222DAE01495C5F4FB801C401AA
:10DD40000E94A0D2182F2FCF2F923F924F925F9216
:10DD50006F927F928F929F92AF92BF92CF92DF92FB
:10DD6000EF92FF920F931F93CF93DF93CDB7DEB760
:10DD7000ED970FB6F894DEBF0FBECDBF8091CA05F8
:10DD8000882369F18091C61600E010E083FF23C06C
:10DD900083ED94E10E94A16D8BE1E3EDF4E1DE01FE
:10DDA000919601900D928A95E1F710E000E0BE0196
:10DDB0006F5F7F4FCE0181960E9433CE18163CF4E0
:10DDC000CE0101960E9416C8080F111DF0CFCE019A
:10DDD00081960E94A66D00937304109374040E94B0
:10DDE00095BD1091C7051CAF85E0810F8DAF312E19
:10DDF00031948EEDC82E81E6D82E96EEA92E94E1B0
:10DE0000B92E81E0782E711A2AEE822E24E1922E0C
:10DE1000111113C08091C905882391F1809153019C
:10DE2000882359F081E09091C905911180E024E0A8
:10DE300043EF54E1632D0E9469BC8091C61685FFB3
:10DE400055C01130D9F48091C9058130F1F180912C
:10DE50005301882309F45BC11F929F928F927F9296
:10DE600081E09091C905913009F080E08F930E9484
:10DE7000A41C0F900F900F900F900F9082E066C03F
:10DE80008091C4051092C405882341F20E94861D2A
:10DE90008091DE05882311F2ED960FB6F894DEBF6F
:10DEA0000FBECDBFDF91CF911F910F91FF90EF90EB
:10DEB000DF90CF90BF90AF909F908F907F906F90AA
:10DEC0005F904F903F902F9008958091C4051092DD
:10DED000C405882309F4BBCF1092C7050E94D2D194
:10DEE0008091DE05882309F4B2CFD6CF83FF2DC001
:10DEF000113021F68091C9058130D1F08091530114
:10DF0000882309F404C1DF92CF92BF92AF927F922F
:10DF100081E09091C905913009F080E08F930E94D3
:10DF2000A41C0F900F900F900F900F900F90A6CF02
:10DF30008091C4051092C405882301F30E94DE611C
:10DF40008091DE058823D1F2A7CF81E09091530123
:10DF5000992309F4DDC0582E082FF12CE12C412E15
:10DF60009CAD491A802F2091730430917404E216FD
:10DF7000F30608F0CDC00113A5C083ED94E10E9423
:10DF8000A16D202E25188BE1E3EDF4E1DE019196E1
:10DF900001900D928A95E1F7612CBE016F5F7F4F72
:10DFA000CE0181960E9433CE18167CF4CE010196E4
:10DFB0000E9416C8882389F326106BC0BE016F5FCC
:10DFC0007F4F83EF95E00E9431C8CE0181960E9479
:10DFD000A66D8091C6169091C90584FF78C09113F3
:10DFE00066C08091C4051092C405882309F45FC0FF
:10DFF00019821C828091D6146EEE74E1882311F090
:10E0000063ED74E121E043EF55E0CE0101960E94FB
:10E01000AC6D882309F43FC08BE1FE013196A3ED7E
:10E02000B4E101900D928A95E1F78091C6168F7D3B
:10E030008093C616A091BB16AA3080F481E08A0FA7
:10E040008093BB168BE18A9FD0011124A355BA4E51
:10E05000E3EDF4E101900D928A95E1F7CE0101968E
:10E060000E94A66D1092C70582E090E0A0E0B0E0AB
:10E070008093CE059093CF05A093D005B093D105A2
:10E0800081E08093DE051092D40383E080935301F6
:10E0900003CF639482CF0E94473A63EF75E080ED2F
:10E0A00094E10E9409408AE00E946A39D7CF8091AA
:10E0B0005301882339F081E0911380E041E0642D21
:10E0C0000E94AABC8FEFE81AF80A0F5F4BCF911796
:10E0D00059F0809153018823A9F381E09091C905FB
:10E0E000911380E040E0EBCF8091C4051092C4050D
:10E0F000882379F383EF95E00E94B8C70E946D1DD5
:10E100000E94B7BA8091DE05882319F3C5CE82E05C
:10E110001F5F9DAD91137CCE8093C805BDCE8F92BD
:10E120009F92AF92BF92CF92DF92EF92FF92CF93E6
:10E130006B017C01B42E20E030E0A9010E94FCE1DB
:10E1400087FF07C08DE20E946A39F7FAF094F7F86A
:10E15000F094C0E060E070E080E09FE3CB1541F018
:10E160002DEC3CEC4CEC5DE30E9462E2CF5FF6CF1D
:10E17000A70196010E94F3E86B017C010E94EFE980
:10E180004B015C014AE00E942DC7CC2379F1C50107
:10E19000B4010E9401E29B01AC01C701B6010E94DB
:10E1A000F2E86B017C018EE20E946A39C150F0F006
:10E1B00020E030E040E251E4C701B6010E9462E293
:10E1C0006B017C010E94EFE94B015C014AE00E9477
:10E1D0002DC7C501B4010E9401E29B01AC01C7013A
:10E1E000B6010E94F2E86B017C01E0CFCF91FF9075
:10E1F000EF90DF90CF90BF90AF909F908F90089559
:10E20000EF92FF920F931F93CF937C018B01C2E497
:10E210004F3F09F0C4E580E20E946A398C2F0E94CA
:10E220006A398AE30E946A39F701608171818281CB
:10E23000938142E00E948F708EEB92E20E948239BD
:10E24000F801608171818281938142E00E948F7028
:10E2500062E070E080E090E0CF911F910F91FF901D
:10E26000EF900C94E7C01F93CF93DF93CDB7DEB749
:10E2700028970FB6F894DEBF0FBECDBF182F609160
:10E28000A7147091A814072E000C880B990B0E94FC
:10E2900003E26D837E838F8398876091A5147091CC
:10E2A000A614072E000C880B990B0E9403E26983C9
:10E2B0007A838B839C834AEFBE016B5F7F4FCE01D5
:10E2C00001960E9400716091AB057091AC05072E1C
:10E2D000000C880B990B0E9403E26D837E838F8371
:10E2E00098876091A9057091AA05072E000C880BEC
:10E2F000990B0E9403E269837A838B839C834FEF9F
:10E30000BE016B5F7F4FCE0101960E94007160914C
:10E31000AD051F3F39F085E11802F0011124EF55DA
:10E32000FB4E608570E086EC92E20E94393A609183
:10E33000AD0570E081EC92E20E94393A28960FB662
:10E34000F894DEBF0FBECDBFDF91CF911F9108952E
:10E350000F930FB70F9300916E000B7F00936E0029
:10E3600078940F930BB70F930CB70F921F922F93C4
:10E370003F934F935F936F937F938F939F93AF934D
:10E38000BF93EF93FF9311240E94657AFF91EF9161
:10E39000BF91AF919F918F917F916F915F914F91BD
:10E3A0003F912F911F900F900CBF0F910BBF0F91BA
:10E3B0000460F89400936E000F910FBF0F911895B1
:10E3C000CF93DF93C1EAD4E11F821E820E948EC1E7
:10E3D00018865D98C5EAD5E01F821E820E946A6297
:10E3E00018865C98DF91CF910895109237060E94AD
:10E3F000E0710C946D1D4F925F926F927F928F929D
:10E400009F92AF92BF92EF92FF920F931F93CF9381
:10E41000DF93B0E2A0E06A2F70E0AB014B0F511D1B
:10E4200055954795411117C0E2EEF1E2859194911F
:10E43000282F822FDF91CF911F910F91FF90EF90A6
:10E44000BF90AF909F908F907F906F905F904F9014
:10E450000895B42FE2CFA41711F0B41303C0EEE572
:10E46000F2E2E4CF9A0121503109220F331F220F2B
:10E47000331FF901E052FE4DE590F490F901EC51A3
:10E48000FE4D059114918E159F051CF3A42F0817BE
:10E4900019070CF4C0CFBC01F901EE51FE4DC59136
:10E4A000D491F901EA51FE4DA590B4906E197F09FF
:10E4B000072E000C880B990B0E9403E22B013C01F4
:10E4C000B5016C1B7D0B072E000C880B990B0E946D
:10E4D00003E29B01AC01C301B2010E9462E24B0165
:10E4E0005C01B8016E197F09072E000C880B990B8F
:10E4F0000E9403E29B01AC01C501B4010E9476E9D0
:10E500004B015C01BE01DD0F880B990B0E9403E2F9
:10E510009B01AC01C501B4010E94F3E80E94E8E947
:10E52000262F972F86CFCF93DF93C1EAD4E18A813C
:10E530009B810E9498B69D838C83C5EAD5E08A8131
:10E540009B810E94FB719D838C83A895109272041D
:10E55000DF91CF910895EF92FF920F931F93CF9386
:10E56000DF93C82F7B018A018091A4058130A1F43B
:10E570000E94433AC7010E94823986E991E20E94D3
:10E580008239C7FD33C08C2F0C2E000C990B0E94D2
:10E5900030B78AE00E946A390E94E071A8958091A4
:10E5A000F504811132C081E08093F50480E8809306
:10E5B000A4050E94E071D5E1D150149AE1F069E11F
:10E5C00070E080E090E00E94E7C0A895149868E2AF
:10E5D00070E080E090E00E94E7C0A89568E270E0FB
:10E5E00080E090E00E94E7C0A895E6CF82E991E242
:10E5F0000E948239CECF6BE871E2CF3F11F06FE815
:10E6000071E240E0C8010E94703ADF91CF911F9102
:10E610000F91FF90EF9008954F925F926F927F92CB
:10E620008F929F92AF92BF92CF92DF92EF92FF9222
:10E630000F931F93CF93DF93EC016B014A01B22E2E
:10E64000FA014080518062807380A30192016D8144
:10E650007E818F8198850E94FCE18823A1F04D8204
:10E660005E826F827886AA24A39420E030E0A9011C
:10E67000F40160817181828193810E9476EA18168B
:10E680000CF0A12CAC828C818230A1F0833009F493
:10E690005AC08130C9F52D813E814F815885F601E0
:10E6A00060817181828193810E94FCE187FD2CC091
:10E6B00082E08C83B701FF0C880B990B0E9403E268
:10E6C0009B01AC016D817E818F8198850E94F2E86B
:10E6D0009B01AC01F60160817181828193810E946E
:10E6E00076EA87FD22C00E9482C16B017C019801FD
:10E6F000A8EEB3E00E9471E8C60ED71EE81EF91E10
:10E70000C882D982EA82FB82DF91CF911F910F915B
:10E71000FF90EF90DF90CF90BF90AF909F908F9041
:10E720007F906F905F904F9008950E9482C1088102
:10E7300019812A813B81601B710B820B930B97FD22
:10E74000E3CF83E08C8340E652E260E772E28B2DF8
:10E75000DF91CF911F910F91FF90EF90DF90CF90BD
:10E76000BF90AF909F908F907F906F905F904F90F1
:10E770000C94AB72CF93DF93EC01488159816A818D
:10E780007B8181E891E20E94FB3B4C815D816E813F
:10E790007F8189E297E20E94FB3B488559856A8523
:10E7A0007B8585E297E20E94FB3B8AE0DF91CF9177
:10E7B0000C946A39BC012091D6043091D704409161
:10E7C000D6045091D7042417350731F481E0261779
:10E7D000370709F080E008959A01F1CF0F930FB742
:10E7E0000F9300916E000F930B7F00936E000091CA
:10E7F0006F000D7F00936F000F930BB70F930CB753
:10E800000F921F922F933F934F935F936F937F933A
:10E810008F939F93AF93BF93EF93FF9311240E9425
:10E82000FA7BFF91EF91BF91AF919F918F917F9173
:10E830006F915F914F913F912F911F900F900CBF5F
:10E840000F910BBF0F910260F89400936F000F912E
:10E8500000936E000F910FBF0F91189500000000FC
:10E86000000000008091930580FF27C0459A8FEF3C
:10E8700080938C0480919305869580FF21C0479AF0
:10E880008FEF80938D04809193058695869580FF08
:10E890001AC02A988FEF80938E04809193058695F5
:10E8A0008695869580FF12C0289A8FEF80938F04FB
:10E8B00000000000000000000895459881E0D8CFD6
:10E8C000479881E0DECF2A9A81E0E5CF289881E061
:10E8D000EDCFCF92DF92EF92FF920F931F93CF93E2
:10E8E000DF93CDB7DEB7C658D1090FB6F894DEBFB7
:10E8F0000FBECDBFC358DF4F188219821A821B8208
:10E90000CD57D0408091140290911502A09116022B
:10E91000B0911702CF57DF4F88839983AA83BB83B7
:10E92000C158D04084E690E090930E0680930D0687
:10E930001092B7141092B61410928B0464E070E039
:10E94000CE018F579F4F0E941AC180910D06909162
:10E950000E06029690930E0680930D061092B71441
:10E960001092B61481E0CA57DF4F8883C658D04052
:10E97000CE018A579F4F0E94146668E470E08CEFC6
:10E980009AE00E941AC160E170E08FE096E00E9478
:10E990001AC18AE097EDA3EABCE3C358DF4F88832E
:10E9A0009983AA83BB83CD57D040CE0183589F4F14
:10E9B0000E940C6685E995E00E9418667E018DE64E
:10E9C000E80EF11C8FEFD7018C93C7010E941466EB
:10E9D00019821A821B821C828E010F5F1F4FC80191
:10E9E0000E940C6619821A821B821C82C8010E9436
:10E9F0000C6685E08983F70180838BE694E00E94B2
:10EA00000C66C8010E941466C7010E94146664E681
:10EA100070E087E094E00E941AC18CE0D8011D925A
:10EA20008A95E9F7C8010E941866C358DF4F18821B
:10EA300019821A821B82CD57D0403AE0D32EDA9445
:10EA4000DD2031F0CE0183589F4F0E940C66F7CF36
:10EA500088E0F701982F11929A95E9F7D8011D9255
:10EA60008A95E9F783E0CB57DF4F8883C558D040BC
:10EA7000EA968FAFEA97CE018B579F4F0E9414669C
:10EA8000CE0187589F4F0E94146668E070E0C8016D
:10EA90000E941AC168E070E0C7010E941AC1C35801
:10EAA000DF4F188219821A821B82CD57D0402AE08C
:10EAB000C22ED12CB1E0CB1AD10831F0CE0183584F
:10EAC0009F4F0E940C66F6CF19828FEFF70180836B
:10EAD000C8010E941066C7010E94146680E1D82E0A
:10EAE000D801ED2D1D92EA95E9F760E170E0C801CB
:10EAF0000E941AC11982C8010E9410666CE070E081
:10EB00008EEA95E00E941AC1198A1A8A1B8A1C8A09
:10EB100080E090E0A0E8BFE38D879E87AF87B88B49
:10EB20008091AA149091AB14A091AC14B091AD1443
:10EB300089839A83AB83BC832CEA35EC47E25EE39E
:10EB40006091AE147091AF148091B0149091B11493
:10EB50000E9476E96D837E838F8398872CEA35EC5B
:10EB600047E25EE36091B2147091B3148091B414E3
:10EB70009091B5140E9462E269877A878B879C879F
:10EB800064E170E0C8010E941AC184E190E09A83B8
:10EB90008983C8010E9404668CE0E6E9F1E0D801AF
:10EBA00001900D928A95E1F7C8010E9408668CE0F9
:10EBB000E6E9F1E0D80101900D928A95E1F7C801EC
:10EBC0000E9408661982C8010E9414668FE790E0CF
:10EBD0009A838983C8010E94046685E0E2EAF1E035
:10EBE000D80101900D928A95E1F765E070E0C801C7
:10EBF0000E941AC11982C8010E94106680E2E7EAE9
:10EC0000F1E0D80101900D928A95E1F760E270E0A1
:10EC1000C8010E941AC1D7011C92C7010E94106648
:10EC200086E094E00E94106682E094E00E940C6608
:10EC3000C358DF4F188219821A821B82CD57D040E9
:10EC4000CE0183589F4F0E940C6680E2F80111921A
:10EC50008A95E9F760E270E0C8010E941AC1FE01DE
:10EC6000F99688E0DF011D928A95E9F744E650E0C5
:10EC700060E070E049835A836B837C834D835E83BD
:10EC80006F83788783E090E0A0E0B0E089879A877F
:10EC9000AB87BC874D875E876F87788B498B5A8B94
:10ECA0006B8B7C8B8D8B9E8BAF8BB88F898F9A8F64
:10ECB000AB8FBC8F8D8F9E8FAF8FB8A38EE190E00E
:10ECC000A0E0B0E089A39AA3ABA3BCA38DA39EA3AD
:10ECD000AFA3B8A789A79AA7ABA7BCA78DA79EA7E4
:10ECE000AFA7B8AB89AB9AABABABBCAB8DAB9EABB4
:10ECF000AFABB8AF60E470E0C8010E941AC1F80180
:10ED00008D2D11928A95E9F760E170E0C8010E94AB
:10ED10001AC1D8011D92DA94E9F760E170E0C801E8
:10ED20000E941AC1C358DF4F188219821A821B82AF
:10ED3000CD57D040CE0183589F4F0E940C669CE077
:10ED4000D92EF8018D2D11928A95E9F76CE070E0CB
:10ED5000C8010E941AC18CE6D8011D928A95E9F774
:10ED60006CE670E0C8010E941AC18FE794E00E942F
:10ED70000866F701108211821282138214821582B2
:10ED80001682178268E070E0C7010E941AC1F7017D
:10ED90001192DA94E9F7CB57DF4F1882C558D0406B
:10EDA00080E090E0A0E4B0E4ED968CAF9DAFAEAF14
:10EDB000BFAFED97C7010E941866CE018B579F4FDA
:10EDC0000E941466CE0187589F4F0E940C66809166
:10EDD0008B04811124C000910D0610910E068091C4
:10EDE000B6149091B714D7018D939C9384E690E06C
:10EDF00090930E0680930D0664E070E083ED91E041
:10EE00000E941AC1C7010E94046691E00D341340AC
:10EE100009F490E080918B04892B80938B0480917E
:10EE20008B04811105C060E089EC96E10E94771F98
:10EE300090918B0481E08927CA57DF4F0FB6F89471
:10EE4000DEBF0FBECDBFDF91CF911F910F91FF901D
:10EE5000EF90DF90CF900895AF92BF92CF92DF9264
:10EE6000EF92FF920F931F93CF93DF93CCEFDAE0F3
:10EE70000FE116E08CE0A82E8BE0B82EC12CD12C2F
:10EE80007601C39469917991899199910E9401E2E7
:10EE9000288939894A895B890E9462E20E94EFE9E8
:10EEA000F80161937193819391938F01C616D706F0
:10EEB000E806F90610F46B017C01AC16BD0611F7EB
:10EEC0006FEF7FEFCB01A70196010E9444E82093EA
:10EED0002F06309330064093310650933206DF916F
:10EEE000CF911F910F91FF90EF90DF90CF90BF9047
:10EEF000AF9008950F931F93CF93DF9300E11BE032
:10EF0000C8E3D6E0F80121913191419151918F01EF
:10EF100060E070E080E89FE30E9476E9699379936E
:10EF200089939993F6E0C834DF0761F70E949BB993
:10EF3000DF91CF911F910F910C942C7790911E151A
:10EF400080911F15981306C08091490690914A063A
:10EF5000892B19F00E941340F1CF089590911E154E
:10EF600080911F15981308C08091490690914A0618
:10EF7000892B11F40C94CC330E941340EFCFCF9324
:10EF8000DF9320910104222379F0EC010E949E5F1F
:10EF90009B01AC01688579858A859B850E94F2E892
:10EFA000688779878A879B87DF91CF910895CF9370
:10EFB000DF9320910104222379F0EC010E949E5FEF
:10EFC0009B01AC01688579858A859B850E94F3E861
:10EFD000688779878A879B87DF91CF9108954F92C1
:10EFE0005F926F927F928F929F92AF92BF92CF92D9
:10EFF000DF92EF92FF920F931F93CF93DF93CDB7E2
:10F00000DEB76A970FB6F894DEBF0FBECDBF9A8FFA
:10F01000898F5B018A01DC01D6966D917D918D917E
:10F020009C91D9970E9401E26B017C01F50120813E
:10F030003181428153810E9462E20E945FE92B018B
:10F040003C01D8012D913D914D915C91C701B601D4
:10F050000E9462E20E945FE94B015C01C301B201C0
:10F060000E94EFE9698B7A8B8B8B9C8B68377105DB
:10F070008105910540F428E730E040E050E0298B1D
:10F080003A8B4B8B5C8BC501B4010E94EFE96D8715
:10F090007E878F87988B683771058105910540F4CD
:10F0A00088E790E0A0E0B0E08D879E87AF87B88BBF
:10F0B000E98DFA8DEE5BFF4F2081318142815381D2
:10F0C00029833A834B835C83CA01B9010E9403E21E
:10F0D0002B013C0169897A898B899C890E9401E214
:10F0E00069877A878B879C8720E030E0A901C3017C
:10F0F000B2010E94FCE1882309F43BC1A7019601FB
:10F10000C701B6010E9462E24B015C0129853A8584
:10F110004B855C85CA01B9010E9462E29B01AC018A
:10F12000C501B4010E94F2E84B015C01A301920108
:10F13000C301B2010E94F3E89B01AC01C501B40117
:10F140000E9476E90E945FE90E94EFE96D837E8369
:10F150008F83988769817A818B819C819095809536
:10F16000709561957F4F8F4F9F4F0E9403E24B0137
:10F170005C016D857E858F8598890E9401E2698397
:10F180007A838B839C8320E030E0A901C501B40120
:10F190000E94FCE1882309F4F0C029813A814B8167
:10F1A0005C81CA01B9010E9462E26D8B7E8B8F8BFC
:10F1B000988FA7019601C701B6010E9462E29B01E8
:10F1C000AC016D897E898F89988D0E94F2E86B0170
:10F1D0007C01A5019401C501B4010E94F3E89B01E3
:10F1E000AC01C701B6010E9476E90E941EEAA98D12
:10F1F000BA8D95968D909D90AD90BC909897750125
:10F2000064012D813E814F815885C21AD30AE40AD8
:10F21000F50A0E94EFE9C61AD70AE80AF90AF7FECA
:10F220006EC020E030E0A901C301B2010E94FCE100
:10F23000882309F4A6C0C501B4010E9401E26B0154
:10F240007C01A3019201C301B2010E94F3E89B017A
:10F25000AC01C701B6010E9462E26B017C01298505
:10F260003A854B855C85CA01B9010E9462E29B0127
:10F27000AC01C701B6010E94F2E86B017C01298153
:10F280003A814B815C81CA01B9010E9462E29B0113
:10F29000AC01C701B6010E94F3E86B017C0120E0DC
:10F2A00030E040E850E4C301B2010E9462E29B01F9
:10F2B000AC01C701B6010E9476E90E945FE96B01CB
:10F2C0007C0120E030E0A9010E9476EA18161CF0CB
:10F2D000C12CD12C7601C701B6010E94EFE96D83E4
:10F2E0007E838F83988786169706A806B90620F432
:10F2F0008D829E82AF82B886C12CD12C76018D8101
:10F300009E81AF81B885E98DFA8D81A792A7A3A7C9
:10F31000B4A7C80ED91EEA1EFB1EC5A6D6A6E7A630
:10F32000F0AA29893A894B895C8922AF33AF44AF6F
:10F3300055AFFE962D853E854F85588920833183B4
:10F34000428353836A960FB6F894DEBF0FBECDBFDB
:10F35000DF91CF911F910F91FF90EF90DF90CF90B1
:10F36000BF90AF909F908F907F906F905F904F90E5
:10F37000089560E070E0CB01E5CE60E070E0CB0185
:10F3800034CF60E070E0CB0198CF90916F0081E0C6
:10F3900091FD02C080E0089590916F009D7F909351
:10F3A0006F000895CF93C82F0E94C57994E0C99F3C
:10F3B00090011124F901E752FB4F2B513B4FD9012A
:10F3C0004D915D916D917C914083518362837383F4
:10F3D00091E09093D804882319F0CF910C94E330F6
:10F3E000CF910895CF92DF92EF92FF9280917D04AA
:10F3F000329B60C0816080937D0480917D04339B4B
:10F400005BC0826080937D0480917D04349B56C0F4
:10F41000846080937D04C090C904C0FE10C08091B8
:10F42000930580FF0CC080917D0480FF08C080910F
:10F43000A30581608093A30580E00E94D279D12C3E
:10F44000F12CE12CD701C601B695A7959795879524
:10F4500080FF11C080919305869580FF0CC080913C
:10F460007D0481FF08C08091A30582608093A3057D
:10F4700081E00E94D27982E0F694E794D794C79411
:10F480008A95D1F7C0FE1CC080919305869586951C
:10F4900080FF16C080917D0482FF12C08091A30579
:10F4A00084608093A30582E0FF90EF90DF90CF907F
:10F4B0000C94D2798E7F9FCF8D7FA4CF8B7FA9CFE5
:10F4C000FF90EF90DF90CF9008950F931F93CF930D
:10F4D000DF93809147018F3708F447C08F57909191
:10F4E000A91490931805992309F43DC05D9A909151
:10F4F000AD0590931705992309F441C05C9A8F5F7D
:10F50000809347018091160591E089278093160525
:10F5100081110E94F21F80914601C1E0C80F853021
:10F520000CF0C0E0823009F4D3C05CF5882309F404
:10F530003EC0813009F4C1C0C0934601809192055C
:10F5400081110E94F2798091490690914A060097B4
:10F5500029F0019790934A0680934906DF91CF9155
:10F560001F910F9108955D98C2CF9091180589174A
:10F5700008F05D9890911705891708F4C0CF5C9842
:10F58000BECF843009F4BBC00CF4B5C08530A1F601
:10F5900090911505911102C0809315058091150574
:10F5A000815080931505882339F2C5E0C5CF80913D
:10F5B00045018F5F80311CF480934501BDCF1092CF
:10F5C000450180917204811113C08091A114909122
:10F5D000A2149093A4148093A3148091A5059091F4
:10F5E000A6059093A8058093A70581E080937204F7
:10F5F0001092A2141092A1141092A6051092A505C3
:10F600000091A3141091A4148091A7149091A814B0
:10F61000D1E0181619062CF08091A914811101C0AF
:10F62000D0E080914C0190914D01081719073CF4EE
:10F6300040E852E26DE872E280E00E94AB72DD23A6
:10F6400071F080914A0190914B01801791073CF431
:10F650004FE952E26CEA72E280E00E94AB720091E4
:10F66000AB051091AC052091A7053091A8058091BC
:10F670008F0590919005281739073CF440E852E235
:10F680006DE872E28FEF0E94AB72101611060CF05B
:10F6900053CF2091A7053091A80580914801909102
:10F6A0004901821793070CF047CF4FE952E26CEA09
:10F6B00072E28FEF0E94AB723FCF10927B0087E423
:10F6C00080937C0080917A00806480937A0034CFAC
:10F6D00080917A0086FD26C02091780030917900D3
:10F6E0008091A1149091A214820F931F9093A21461
:10F6F0008093A11421CF10927B0086E4E1CF80910A
:10F700007A0086FD11C020917800309179008091B7
:10F71000A5059091A605820F931F9093A60580934F
:10F72000A5050ACFC2E008CFC4E006CF0E94C57984
:10F730001092330610923406109235061092360657
:10F7400081110C94E33008950F931F9380911E153F
:10F7500090911F15891B8F7009F449C090911B155A
:10F76000992361F0833040F48FEF890F29F0809363
:10F770001B1590E080E038C010921B1580911F157A
:10F780002BE4829FC0011124855B994FFC012081ED
:10F7900020FDEFCF4091330650913406609135063D
:10F7A00070913606E95BFF4F008111812281338120
:10F7B000401B510B620B730B40933306509334067E
:10F7C000609335067093360620911F152F5F2F70BA
:10F7D00020931C1530911F1520911D15321304C064
:10F7E00020911C1520931D151F910F9108950E94C3
:10F7F000967BBFCF2F923F924F925F926F927F92F4
:10F800008F929F92AF92BF92CF92DF92EF92FF9230
:10F810000F931F93CF93DF9300D000D0CDB7DEB707
:10F820008FEF9FEF90938900809388000AE009830F
:10F83000312C212C78948091D2049091D304A09102
:10F84000D404B091D504892B8A2B8B2B09F0C4C129
:10F850008091D8048823E1F08091D6049091D70458
:10F860001092D804892B09F4B7C11092D7041092D2
:10F87000D6041092C90490911E1580911F159817F7
:10F8800009F4AAC180911F158F5F8F7080931F1597
:10F890008091D6049091D704892B09F49DC14091A1
:10F8A000CE045091CF046091D0047091D104809126
:10F8B000CA049091CB04A091CC04B091CD040091E6
:10F8C000BC0410E030E020E0841B950BA60BB70BC6
:10F8D000081719072A073B0710F4D901C8018A83C2
:10F8E000840F951FA61FB71F8093CE049093CF045B
:10F8F000A093D004B093D104E1E0C0909404D090E0
:10F900009504E0909604F09097048091A40490915F
:10F91000A504A091A604B091A704C80ED91EEA1EA2
:10F92000FB1EC092A404D092A504E092A604F0921B
:10F93000A704F7FC33C040918C04042E000C550B37
:10F94000660B770B8091E5049091E604A091E704A3
:10F95000B091E804840F951FA61FB71F8093E5049C
:10F960009093E604A093E704B093E8048091900498
:10F9700090919104A0919204B0919304A7019601F3
:10F98000281B390B4A0B5B0BDA01C9018093A404D5
:10F990009093A504A093A604B093A70400919804A3
:10F9A0001091990420919A0430919B048091A804AD
:10F9B0009091A904A091AA04B091AB04080F191F5B
:10F9C0002A1F3B1F0093A8041093A9042093AA04A4
:10F9D0003093AB0437FD33C080918D04082E000CAA
:10F9E000990BAA0BBB0B4091E9045091EA0460917A
:10F9F000EB047091EC04840F951FA61FB71F809332
:10FA0000E9049093EA04A093EB04B093EC04809192
:10FA1000900490919104A0919204B0919304B90143
:10FA2000A801481B590B6A0B7B0BDB01CA018093B1
:10FA3000A8049093A904A093AA04B093AB044091A6
:10FA40009C0450919D0460919E0470919F0480914C
:10FA5000AC049091AD04A091AE04B091AF04480FF6
:10FA6000591F6A1F7B1F4093AC045093AD046093F1
:10FA7000AE047093AF0477FD33C080918E04082EDE
:10FA8000000C990BAA0BBB0B8090ED049090EE0438
:10FA9000A090EF04B090F004880D991DAA1DBB1D25
:10FAA0008093ED049093EE04A093EF04B093F004E0
:10FAB0008091900490919104A0919204B09193044C
:10FAC0002A013B01481A590A6A0A7B0AD301C2017A
:10FAD0008093AC049093AD04A093AE04B093AF04B4
:10FAE0008090A0049090A104A090A204B090A304E0
:10FAF0008091B0049091B104A091B204B091B3048C
:10FB0000880D991DAA1DBB1D8093B0049093B1046C
:10FB1000A093B204B093B304B7FD33C040908F04F8
:10FB2000042C000C5508660877088090F10490902A
:10FB3000F204A090F304B090F404840C951CA61C6D
:10FB4000B71C8092F1049092F204A092F304B09258
:10FB5000F4048090900490909104A0909204B0904E
:10FB600093042C013D01481859086A087B08530189
:10FB700042018092B0049092B104A092B204B0927B
:10FB8000B304E11104C0E0918400F0918500F7FE18
:10FB90005F9A37FF469A77FF2B9AB7FF299AE09131
:10FBA0008400F0918500E0918400F0918500F7FEDB
:10FBB0005F9837FF469877FF2B98B7FF29985A80B0
:10FBC000552021F080918400909185000A81015098
:10FBD0000A83E0E0011191CE80905401909055018C
:10FBE000A0905601B090570181149104A104B10472
:10FBF00009F047C08091EC059091ED05009709F45C
:10FC00002FC023B1247015980000000000000000F0
:10FC1000181619060CF0D7C02A9A00000000000040
:10FC200000002B9A34E03A950000E9F72B98000089
:10FC3000000000000000222309F4C7C02A9A000037
:10FC4000000000000000181619060CF0C0C08091DA
:10FC5000EC059091ED0501979093ED058093EC05EF
:10FC60000E949133882309F4B8C080ED97E0A0E0AA
:10FC7000B0E08093540190935501A0935601B09346
:10FC800057018091D2049091D304A091D404B091F3
:10FC9000D504892B8A2B8B2B09F053C4E091D60411
:10FCA000F091D704309709F427C58091CE04909144
:10FCB000CF04A091D004B091D1044091CA045091D6
:10FCC000CB046091CC047091CD0484179507A607EE
:10FCD000B70708F486C01092D7041092D604109289
:10FCE000C90490911E1580911F15981709F404C539
:10FCF00080911F158F5F8F7080931F1580EDC82E28
:10FD000087E0D82EE12CF12C8091D6049091D70475
:10FD1000892B09F00EC40E94A47B9093D704809392
:10FD2000D604892B09F405C44090D6045090D7041A
:10FD30005C824B82D2018C9183FFB3C2F201858D2C
:10FD4000968DA78DB0A1418D528D638D748D0589DF
:10FD500016892789308D0093E5041093E6042093DB
:10FD6000E7043093E8044093E9045093EA04609375
:10FD7000EB047093EC048093ED049093EE04A09355
:10FD8000EF04B093F00481A192A1A3A1B4A1809348
:10FD9000F1049093F204A093F304B093F40410924E
:10FDA000D7041092D6041092C90490911E15809128
:10FDB0001F15981709F4AFCF80911F158F5F8F70B3
:10FDC00080931F15A8CF2A9828CF2A9838CF8091E2
:10FDD000EC059091ED0501963FCF8FEF9FEFDC0191
:10FDE00048CF4091C5045091C6046091C7047091FA
:10FDF000C804481759076A077B0708F4DEC08091DA
:10FE0000C1049091C204A091C304B091C40441A95B
:10FE100052A963A974A91127859F412C969F90012F
:10FE2000A69F300DA59F200D311D869F400C211DE2
:10FE3000311F959F400C211D311FA49F400C211D97
:10FE4000311F949F410C211F311F4694211F311FE8
:10FE5000789F200D311D799F300D112442AD53AD97
:10FE600064AD75AD420F531F611D711D4093BD04FC
:10FE70005093BE046093BF047093C00406A917A9F1
:10FE800020AD31AD041715072607370740F400935E
:10FE9000BD041093BE042093BF043093C00440906F
:10FEA000BD045090BE046090BF047090C00421E671
:10FEB00031E201E00A83F901459155916591749110
:10FEC000441555056605770570F476946794579444
:10FED00047941A81110F1A832C5F3F4F4DE751E26F
:10FEE0004217530741F75A815093BC0460E246160B
:10FEF00051046104710428F410E2412E512C612C4C
:10FF0000712C70E2471A5108610871084114E8E049
:10FF10005E066104710408F42EC0F4E05F9E900157
:10FF200011242F59324EF901329645915491042DE6
:10FF3000EE27059FB001049F610D7E1F06946E1F82
:10FF40007E1F1124AB0170E060E0F901C590D490F0
:10FF5000F12CE12CC41AD50AE60AF70A8C0D9D1D76
:10FF6000AE1DBF1D8093C1049093C204A093C3042F
:10FF7000B093C404C9CEB301A20176956795579595
:10FF800047959A012C7F2F59364EF901C590D49090
:10FF9000F901329645915491142D1770149F9001D8
:10FFA000159F300D1124F3E036952795FA95E1F76A
:10FFB000C21AD30AF12CE12CD1CF4091B804509150
:10FFC000B9046091BA047091BB04481759076A07D5
:10FFD0007B0708F0D4C08091B4049091B504A0913F
:10FFE000B604B091B70441A952A963A974A9222704
:10FFF000859F312D969F8001A69F100DA59F000D16
:020000021000EC
:10000000111D869F300D011D121F959F300D011D82
:10001000121FA49F300D011D121F949F310D021F4E
:10002000121F3695021F121F789F000D111D799F18
:10003000100D112430E020E04091BD045091BE0429
:100040006091BF047091C004FE9640805180628030
:100050007380041715072607370758F4401B510B08
:10006000620B730B441655066606770610F42A01D8
:100070003B0121E631E241E04A83F9014591559186
:1000800065917491441555056605770570F476946D
:100090006794579447945A81550F5A832C5F3F4F6A
:1000A0006DE771E26217730741F77A817093BC04C0
:1000B000E0E24E1651046104710428F400E2402E7F
:1000C000512C612C712CF0E24F1A51086108710813
:1000D000411408E050066104710408F42EC014E0D5
:1000E000519E900111242F59324EF90132964591BB
:1000F0005491F42DEE27F59FB001F49F610D7E1F02
:1001000006946E1F7E1F1124AB0170E060E0F901C0
:10011000C590D490F12CE12CC41AD50AE60AF70A4E
:100120008C0D9D1DAE1DBF1D8093B4049093B5042E
:10013000A093B604B093B704E7CDB301A2017695BE
:100140006795579547959A012C7F2F59364EF9019F
:10015000C590D490F901329645915491042D0770C1
:10016000049F9001059F300D112413E036952795CB
:100170001A95E1F7C21AD30AF12CE12CD1CF809164
:10018000410190914201A0914301B0914401B7FF18
:100190005DC0C6A8D7A8E0ACF1AC81E691E221E051
:1001A000FC0145915591659174914C155D056E0565
:1001B0007F0558F4F694E794D794C794220F0496D9
:1001C0004DE751E24817590759F72093BC0450E214
:1001D000C516D104E104F10428F470E2C72ED12C35
:1001E000E12CF12C60E2C61AD108E108F108C11433
:1001F00078E0D706E104F10408F431C0A4E0DA9E07
:10020000C00111248F59924EFC01329625913491F0
:10021000BC2D6627B39FA001B29F410D561F0694C7
:10022000461F561F112470E060E0FC0185919491F7
:10023000B0E0A0E0841B950BA60BB70B80934101A7
:1002400090934201A0934301B0934401C0904101B7
:10025000D0904201E0904301F090440155CDD70188
:10026000C601B695A795979587958C7F8F59964E21
:10027000FC0125913491FC01329645915491EC2D6D
:10028000E770E49FC001E59F900D112463E096950F
:1002900087956A95E1F7281B390BC901B0E0A0E00A
:1002A000CDCFAB81BC8155960D911D912D913C9187
:1002B000589781E0011511052105310509F480E009
:1002C000EB81FC81C18CD28CE38CF48CC114D10401
:1002D000E104F10409F08260AB81BC815D964D912F
:1002E0005D916D917C919097411551056105710566
:1002F00009F084608093C9041092B4041092B5048C
:100300001092B6041092B7041092C1041092C20465
:100310001092C3041092C404EB81FC8185A196A1C4
:10032000A7A1B0A58093CA049093CB04A093CC045A
:10033000B093CD04442455243201481A590A6A0A5C
:100340007B0A4092A4045092A5046092A604709285
:10035000A7044092A8045092A9046092AA04709243
:10036000AB044092AC045092AD046092AE04709223
:10037000AF044092B0045092B1046092B204709203
:10038000B30441A052A063A074A0440C551C661C89
:10039000771C000F111F221F331F0093940410932A
:1003A00095042093960430939704CC0CDD1CEE1C2E
:1003B000FF1CC0929804D0929904E0929A04F092A3
:1003C0009B04440F551F661F771F40939C04509356
:1003D0009D0460939E0470939F044092A0045092E9
:1003E000A1046092A2047092A304880F991FAA1F0F
:1003F000BB1F8093900490939104A0939204B093B8
:1004000093041092CE041092CF041092D004109254
:10041000D10481A592A5A3A5B4A58093C50490930A
:10042000C604A093C704B093C80485A596A5A7A544
:10043000B0A98093B8049093B904A093BA04B09380
:10044000BB0485A990919305891721F080939305AA
:100450000E942E748091920581110E94F2794424A9
:100460004A94542C320140924101509242016092D0
:10047000430170924401AB81BC81DA964D915D914C
:100480006D917C91DD974093BD045093BE046093C1
:10049000BF047093C00481E691E2A1E0FC010591E4
:1004A000159125913491041715072607370758F43D
:1004B0007695679557954795AA0F0496EDE7F1E273
:1004C000E817F90759F7A093BC04403251056105BC
:1004D000710520F440E250E060E070E040525109C4
:1004E000610971094115F8E05F076105710508F4BC
:1004F000DAC004E0509FC00111248F59924EFC01D4
:10050000329625913491AA27439FF001429FE10D35
:10051000FA1F0694EA1FFA1F1124AF0170E060E091
:10052000FC01C590D490F12CE12CC41AD50AE60A3E
:10053000F70AC092D204D092D304E092D404F0928D
:10054000D50489288A288B28C9F48091D2049091F7
:10055000D304A091D404B091D5048A3F9105A1059C
:10056000B10560F42AEF30E040E050E02093D2047F
:100570003093D3044093D4045093D5044091540154
:100580005091550160915601709157010091D2042C
:100590001091D3042091D4043091D5044F3F8FEFB4
:1005A00058076807780799F0D901C801B695A7954B
:1005B00097958795481759076A077B0740F48093FA
:1005C000540190935501A0935601B0935701409167
:1005D00054015091550160915601709157014F3F60
:1005E0009FEF59076105710508F07DC04B835A8361
:1005F000F62FE72F8B819A81AF2FBE2F081719078F
:100600002A073B0710F4D901C801081B190B2A0B54
:100610003B0B0093D2041093D3042093D404309363
:10062000D5044F3FEFEF5E076E077E0761F0481B72
:10063000590B6A0B7B0B4093540150935501609307
:10064000560170935701F8942091840030918500F1
:10065000205F3F4F098101500983002309F44AC0FC
:10066000280E391E2216330610F40C941A7C309290
:1006700089002092880078940F900F900F900F902F
:10068000DF91CF911F910F91FF90EF90DF90CF906E
:10069000BF90AF909F908F907F906F905F904F90A2
:1006A0003F902F900895DB01CA01B695A7959795C5
:1006B00087958C7F8F59964EFC01C590D490FC0194
:1006C0003296259134914770429FC001439F900D0F
:1006D0001124A3E096958795AA95E1F7C81AD90A3F
:1006E000F12CE12C26CFAFEFAB83BFEFBA83F0E064
:1006F000E0E080CF1901BBCF80EDC82E87E0D82E77
:10070000E12CF12C08CBFC01208131814281538105
:1007100060911C0B70911D0B80911E0B90911F0B13
:100720000E9462E20E947BEA60932C1570932D1563
:1007300080932E1590932F1590911E1580911F1563
:1007400098130C9438660E949E770E94C579409158
:100750002C1550912D1560912E1570912F154093E9
:10076000F1045093F2046093F3047093F404811144
:100770000C94E33008954F925F926F927F928F9224
:100780009F92AF92BF92CF92DF92EF92FF920F9320
:100790001F93CF93DF93EC018B015A01F901209154
:1007A0001C0B30911D0B40911E0B50911F0B608153
:1007B0007181828193810E9462E20E947BEA6B01D7
:1007C0007C012091180B3091190B40911A0B50911C
:1007D0001B0BF50160817181828193810E9462E22D
:1007E0000E947BEA4B015C012091140B3091150BA8
:1007F0004091160B5091170BF80160817181828135
:1008000093810E9462E20E947BEA2B013C012091CD
:10081000100B3091110B4091120B5091130B68810A
:1008200079818A819B810E9462E20E947BEA6093C7
:1008300020157093211580932215909323154092D3
:1008400024155092251560922615709227158092D6
:10085000281590922915A0922A15B0922B15C092B6
:100860002C15D0922D15E0922E15F0922F15909107
:100870001E1580911F15981791F0DF91CF911F9150
:100880000F91FF90EF90DF90CF90BF90AF909F902F
:100890008F907F906F905F904F900C9438660E947D
:1008A0009E770E94C5794091281550912915609135
:1008B0002A1570912B150091241510912515209162
:1008C000261530912715C0902015D0902115E09065
:1008D0002215F0902315C092E504D092E604E09230
:1008E000E704F092E8040093E9041093EA042093EB
:1008F000EB043093EC044093ED045093EE046093CA
:10090000EF047093F00440912C1550912D156091D7
:100910002E1570912F154093F1045093F2046093BB
:10092000F3047093F404882391F0DF91CF911F9129
:100930000F91FF90EF90DF90CF90BF90AF909F907E
:100940008F907F906F905F904F900C94E330DF9189
:10095000CF911F910F91FF90EF90DF90CF90BF90BC
:10096000AF909F908F907F906F905F904F90089581
:10097000CF92DF92EF92FF92CF93DF93C82F0E9426
:10098000C57994E0C99FE0011124FE01EB51FB4FB2
:10099000C080D180E280F38081110E94E330C85C86
:1009A000D94FC701B6010E9403E2288139814A81EB
:1009B0005B810E9462E2DF91CF91FF90EF90DF9028
:1009C000CF900895CF92DF92EF92FF92CF93DF9373
:1009D000C82F0E94C57994E0C99FE0011124FE014F
:1009E000E752FB4FC080D180E280F38081110E94EA
:1009F000E330C85CD94FC701B6010E9403E22881E9
:100A000039814A815B810E9462E2DF91CF91FF9040
:100A1000EF90DF90CF900895CF930E94C579C82FB3
:100A200080911F1580931E1580931D1580931C15B2
:100A300084E680931B150E94967B80ED93E0909353
:100A40004A0680934906C1110E94E33081E08093F9
:100A5000D804CF910895CF93DF9324E0829FC00103
:100A60001124EC01CF5FD94FFC01EB56FA4F8F51A7
:100A70009C4FDC012D913D914D915C916081718184
:100A8000828193810E94F3E8688379838A839B83C0
:100A9000DF91CF91089580FF04C090917E0490FD76
:100AA0008E7F81FF05C090917E04969590FD8D7F8D
:100AB00082FF06C090917E049695969590FD8B7F5F
:100AC0000895CF92DF92EF92FF920F931F93C12C64
:100AD000D12C76018C0120E53BE04CE45BE068E43E
:100AE0007BE084E49BE00E9439B91F910F91FF9055
:100AF000EF90DF90CF9008954F925F926F927F9228
:100B00008F929F92AF92BF92CF92DF92EF92FF921D
:100B10000F931F93CF93DF93CDB7DEB72C970FB60C
:100B2000F894DEBF0FBECDBF2B013C0129873A8769
:100B30004B875C8747015801F601E080F180028114
:100B4000138120E030E0A901B701C8010E94FCE157
:100B5000882309F484C05E2D4F2D302F212F852F3F
:100B6000942FA32FB22F89839A83AB83BC8320E079
:100B700030E0A901B701C8010E94FCE1811104C065
:100B8000E12CF12C08E413E4C701D8018D839E8386
:100B9000AF83B887A501940160914C0B70914D0B08
:100BA00080914E0B90914F0B0E94FCE187FF0CC08F
:100BB00080924C0B90924D0BA0924E0BB0924F0B2B
:100BC000CE0101960E9461854092440B5092450BE4
:100BD0006092460B7092470B89859A85AB85BC85E0
:100BE0008093480B9093490BA0934A0BB0934B0B07
:100BF000CE0105960E946185A501940160914C0B80
:100C000070914D0B80914E0B90914F0B0E9476EAA4
:100C1000181664F480924C0B90924D0BA0924E0BE0
:100C2000B0924F0BCE0101960E9461850E949E7783
:100C30002C960FB6F894DEBF0FBECDBFDF91CF91DB
:100C40001F910F91FF90EF90DF90CF90BF90AF90EA
:100C50009F908F907F906F905F904F90089550E09D
:100C600040E030E820E47BCFCF92DF92EF92FF921A
:100C70000F931F936B01FC01E080F18002811381CF
:100C8000E4E4FBE0248135814681578160817181F4
:100C9000828193810E947C851F910F91FF90EF903C
:100CA000DF90CF9008950C949BB92F923F924F9272
:100CB0005F926F927F928F929F92AF92BF92CF92EC
:100CC000DF92EF92FF920F931F93CF93DF93CDB7F5
:100CD000DEB76C970FB6F894DEBF0FBECDBF809124
:100CE0007104811150C18091700481113CC18091C7
:100CF0007204811119C06C960FB6F894DEBF0FBE56
:100D0000CDBFDF91CF911F910F91FF90EF90DF90BA
:100D1000CF90BF90AF909F908F907F906F905F909B
:100D20004F903F902F9008950E9493720E9482C12D
:100D30004B015C010091A5141091A6148091500103
:100D400090915101801791070CF448C26091A7144B
:100D50007091A814072E000C880B990B0E9403E2D7
:100D60006D837E838F839887B801110F880B990B51
:100D70000E9403E269837A838B839C832AE0E22EBC
:100D8000F12C0CE310E020E0AE014B5F5F4FBE01A1
:100D90006F5F7F4F89E095E10E940C730091A5146D
:100DA0001091A61480914E0190914F0180179107E8
:100DB0000CF4F0C060E06093A91480919D149091B0
:100DC0009E14A0919F14B091A0140097A105B105A5
:100DD00039F1A5019401281B390B4A0B5B0BDA0191
:100DE000C901B7FD1DC080919B1490919C140817F8
:100DF00019070CF413C28091A7149091A8140097BE
:100E000039F00E5F1F4F0497081719070CF41CC226
:100E100010929D1410929E1410929F141092A01480
:100E20008091A9059091AA05873991050CF0E2C13E
:100E30008091110590911205A0911305B0911405B0
:100E40000097A105B10561F1A5019401281B390B9B
:100E50004A0B5B0BDA01C901B7FD22C08091A905DD
:100E60009091AA0520910F053091100582179307E4
:100E70000CF4CCC12091AB053091AC0521153105A6
:100E800039F0029624503109821793070CF4EFC110
:100E9000109211051092120510921305109214056C
:100EA00080910B0590910C05A0910D05B0910E0558
:100EB000A5019401281B390B4A0B5B0BDA01C90110
:100EC000B7FD19CF38E8830E33E1931EA11CB11C86
:100ED00080920B0590920C05A0920D05B0920E0524
:100EE0006091AB057091AC05072E000C880B990B37
:100EF0000E9403E26D837E838F8398876091A905AA
:100F00007091AA05072E000C880B990B0E9403E232
:100F100069837A838B839C8382E0E82EF12C02E341
:100F200010E02FEFAE014B5F5F4FBE016F5F7F4F51
:100F300082E195E10E940C738091A9059091AA0528
:100F40009C01255031092239310508F05BC12091FF
:100F5000AB053091AC05821793070CF467C180E0B4
:100F60008093AD05C8CE109270040E940C850E943B
:100F70009E770E94D4B80E94538680917204882381
:100F800009F4B9CED1CE41E070E060E082ED91E2AB
:100F90000E94703A809150019091510108171907F1
:100FA0000CF008CFE090A714F090A814B801012E1F
:100FB000000C880B990B0E9403E21B012C01E11429
:100FC000F10409F43CC1B701601B710B072E000C42
:100FD000880B990B0E9403E26B017C0120E030E05A
:100FE00040E251EC0E94FCE187FD29C120E030E0A5
:100FF00040E251E4C701B6010E9476EA18160CF4EB
:1010000049C180910A05811149C1209102053091A1
:101010000305409104055091050529873A874B87C0
:101020005C878091060590910705A0910805B09115
:1010300009058D879E87AF87B88BA20191016091CA
:10104000F6047091F7048091F8049091F9040E94DD
:10105000F2E82091B2143091B3144091B41450913D
:10106000B5140E9462E229853A854B855C850E9411
:10107000F2E820ED3CEC4CE45DE30E9462E229855D
:101080003A854B855C850E94F3E8698B7A8B8B8B64
:101090009C8B6093020570930305809304059093E5
:1010A00005052091AE143091AF144091B0145091C9
:1010B000B1142D8B3E8B4F8B588F2D853E854F85E0
:1010C0005889C701B6010E94F3E8762E672E8987FA
:1010D0009D8720E030E0A9010E94FCE187FDE9C086
:1010E0002D893E894F89588D60E070E08FE793E449
:1010F0000E9476E9698F7A8F8B8F9C8F272D362DF2
:1011000049855D850E94FCE187FF06C0798C6A8C69
:101110003B8D39874C8D4D87872D962DA985BD85B3
:101120008093060590930705A0930805B0930905E1
:101130002091AA143091AB144091AC145091AD148D
:10114000C701B6010E9462E26B017C01C092FA0401
:10115000D092FB04E092FC04F092FD04272D362D82
:1011600049855D856D897E898F89988D0E9462E2AF
:101170009B01AC012093FE043093FF0440930005D3
:1011800050930105C701B6010E94F3E829893A8905
:101190004B895C890E94F3E820E030E0A9010E94BD
:1011A000F3E86B017C0120E030E0A9010E94FCE142
:1011B00087FD48C020E030E04FE753E4C701B601A7
:1011C0000E9476EA1816A4F56FE72092F604309292
:1011D000F7044092F8045092F904EDCD40E852E251
:1011E0006DE872E280E00E94AB720091A51410914C
:1011F000A614ACCD40E852E26DE872E28FEF0E9497
:10120000AB7216CE1092AD055C9875CD44EB51E2F1
:1012100063EC71E28FEF0E94AB7242CE44EB51E27D
:1012200063EC71E280E00E94AB72FACD8FE798CE5A
:10123000C701B6010E94E8E975956795C6CF81E0C0
:1012400080930A0560E0C1CF10939C1400939B1417
:101250000E9482C1605B7C438F4F9F4F60939D14BF
:1012600070939E1480939F149093A014D9CD909363
:10127000100580930F050E9482C1605E70448D4FFF
:101280009F4F6093110570931205809313059093FF
:10129000140506CE81E080930A0596CF10920A05C8
:1012A0001D861E861F86188A19861A861B861C862E
:1012B000C4CE712C612C19861D862ECF2F923F92A1
:1012C0004F925F926F927F928F929F92AF92BF9256
:1012D000CF92DF92EF92FF920F931F93CF93DF9302
:1012E000CDB7DEB7A6970FB6F894DEBF0FBECDBF61
:1012F00080912701882309F4CDC080917E04C82EF7
:10130000D12CF12CE12C80FF3CC0809029019090E1
:101310002A01A0902B01B0902C012091ED03309177
:10132000EE034091EF035091F003C501B4010E9418
:1013300076EA181644F48092ED039092EE03A092A0
:10134000EF03B092F0038090350190903601A090A9
:101350003701B09038012091ED033091EE034091B8
:10136000EF035091F003C501B4010E94FCE187FF37
:1013700008C08092ED039092EE03A092EF03B0922A
:10138000F003D701C601B695A7959795879580FF7D
:101390003CC080902D0190902E01A0902F01B09024
:1013A00030012091F1033091F2034091F303509109
:1013B000F403C501B4010E9476EA181644F4809241
:1013C000F1039092F203A092F303B092F4038090A1
:1013D000390190903A01A0903B01B0903C012091DE
:1013E000F1033091F2034091F3035091F403C501EE
:1013F000B4010E94FCE187FF08C08092F103909243
:10140000F203A092F303B092F40392E0F694E7940F
:10141000D794C7949A95D1F7C0FE3CC0C0903101D3
:10142000D0903201E0903301F09034012091F50327
:101430003091F6034091F7035091F803C701B601CC
:101440000E9476EA181644F4C092F503D092F6038F
:10145000E092F703F092F803C0903D01D0903E0176
:10146000E0903F01F09040012091F5033091F603A8
:101470004091F7035091F803C701B6010E94FCE1C7
:1014800087FF08C0C092F503D092F603E092F703FD
:10149000F092F8038091FB0A83FD7EC02091500BEF
:1014A0003091510B4091520B5091530B6091F903C5
:1014B0007091FA038091FB039091FC030E94FCE180
:1014C000882309F469C010914806111161C0809108
:1014D0005C0190915D0101972091A5143091A614B3
:1014E000281739073CF40E94473A8DE496E10E94A0
:1014F000823911E02091500B3091510B4091520BE9
:101500005091530B6091F9037091FA038091FB03A2
:101510009091FC030E94F2E86B017C0120E030E036
:10152000A9010E9476EA87FF04C0F7FAF094F7F861
:10153000F094209158013091590140915A015091F5
:101540005B01C701B6010E9462E220E030E84BE394
:1015500054E40E9476EA1816ECF40E94473A8EE2B0
:1015600096E10E9482398091F9039091FA03A0914B
:10157000FB03B091FC038093500B9093510BA0930D
:10158000520BB093530B89EF93E00E94838304C006
:1015900010E0B0CF1111E7CF2AE037ED43E25CE372
:1015A0006091210170912201809123019091240189
:1015B0000E9462E26B017C0160911F017091200129
:1015C000072E000C880B990B0E9403E29B01AC01D3
:1015D000C701B6010E9462E2698B7A8B8B8B9C8B70
:1015E00080910104882309F46CC02091440B309150
:1015F000450B4091460B5091470B6091ED03709164
:10160000EE038091EF039091F0030E94F2E86D8B5E
:101610007E8B8F8B988F2091480B3091490B409196
:101620004A0B50914B0B6091F1037091F203809142
:10163000F3039091F4030E94F2E8698F7A8F8B8F05
:101640009C8F20914C0B30914D0B40914E0B509143
:101650004F0B6091F5037091F6038091F703909121
:10166000F8030E94F2E86D8F7E8F8F8F98A32091F0
:10167000500B3091510B4091520B5091530B609194
:10168000F9037091FA038091FB039091FC030E948F
:10169000F2E86B017C0120E030E0A9016D897E89D0
:1016A0008F89988D0E94FCE181110FC020E030E00D
:1016B000A901698D7A8D8B8D9C8D0E94FCE1811131
:1016C00004C0C12CD12C76012CC12D893E894F89B3
:1016D000588DCA01B9010E9462E24B015C01298D5B
:1016E0003A8D4B8D5C8DCA01B9010E9462E29B016B
:1016F000AC01C501B4010E94F3E84B015C012D8DE2
:101700003E8D4F8D58A1CA01B9010E9462E29B0132
:10171000AC01C501B4010E94F3E84B015C01A701D3
:101720009601C701B6010E9462E29B01AC01C501AE
:10173000B4010E94F3E80E94B4EA4B015C012DEB76
:1017400037E346E855E30E94FCE187FF0FC020E045
:1017500030E0A901C701B6010E9476EA46015701AF
:1017600087FF04C0B7FAB094B7F8B0942DEB37E315
:1017700046E855E3C501B4010E94FCE187FDDEC0E7
:1017800020E030E040EA51E4C501B4010E9476E96E
:101790000E94EFE91B01672B19F422242394312CBA
:1017A000B10190E080E00E9401E29B01AC0160E0A9
:1017B00070E080E89FE30E9476E92B013C01AC01D8
:1017C0009B01C501B4010E9462E24B015C01A301CF
:1017D00092016D897E898F89988D0E9462E26D8B5E
:1017E0007E8B8F8B988FA3019201698D7A8D8B8D63
:1017F0009C8D0E9462E2698F7A8F8B8F9C8FA301F0
:1018000092016D8D7E8D8F8D98A10E9462E26D8F09
:101810007E8F8F8F98A3A3019201C701B6010E940A
:1018200062E269A37AA38BA39CA380E1E4E4FBE0DA
:101830008E010F5F1F4FD80101900D928A95E1F73D
:101840000E9482C12B013C0128EC420E511C611CFC
:10185000711C0DA31EA381E0281A310809F45FC092
:101860000E9482C18B019C010419150926093709C0
:1018700037FD86C02B013C0128EC420E511C611C37
:10188000711C0E9413402D893E894F89588D6981B2
:101890007A818B819C810E94F3E869837A838B83B0
:1018A0009C83298D3A8D4B8D5C8D6D817E818F81DE
:1018B00098850E94F3E86D837E838F8398872D8DB2
:1018C0003E8D4F8D58A169857A858B859C850E94B8
:1018D000F3E869877A878B879C8729A13AA14BA176
:1018E0005CA16D857E858F8598890E94F3E86D8760
:1018F0007E878F87988B750164018E010F5E1F4F65
:101900009E01235F3F4FAE01475F5F4FBE016B5F9C
:101910007F4F8DA19EA10E9439B981119CCF750185
:1019200064018E010F5E1F4F29EF33E045EF53E056
:1019300061EF73E08DEE93E00E9439B980E1EDEE46
:10194000F3E0A4E4BBE001900D928A95E1F7A6963E
:101950000FB6F894DEBF0FBECDBFDF91CF911F91C0
:101960000F91FF90EF90DF90CF90BF90AF909F903E
:101970008F907F906F905F904F903F902F90089541
:101980000E94558680CF2F923F924F925F926F9226
:101990007F928F929F92AF92BF92CF92DF92EF92FF
:1019A000FF920F931F93CF93DF93CDB7DEB761976D
:1019B0000FB6F894DEBF0FBECDBF898BE82EF12C99
:1019C000F701E654F94D6491062E000C770B880B55
:1019D000990B0E9403E24B015C011701220C331C9E
:1019E000220C331CF101EB55F94E259135914591AF
:1019F0005491C501B4010E9462E22B013C01F10146
:101A0000E756F94E659175918591949120E030E00B
:101A100040EC5FE30E9462E2A50194010E9462E251
:101A2000AB01BC0100E010E0980189890E9447BB2E
:101A300020E030E0A901C301B2010E94FCE188234B
:101A400009F441C0B301A201705800E010E0980110
:101A500089890E9447BBA3019201C301B2010E9480
:101A6000F3E82B013C01F701EA56F94E14911111EC
:101A700007C00E94473A84E796E10E9482391AE043
:101A80008989823008F0CBC060E070E88BE395E490
:101A900020E030E040E752E40E9476E96B017C01EF
:101AA000612F70E090E080E00E9401E29B01AC01B8
:101AB000C701B6010E9476E98B019C01B301A20126
:101AC00089890E9447BB81E090E0A0E0B0E00988EE
:101AD00004C0880F991FAA1FBB1F0A94D2F7209138
:101AE0009405282B2093940520917E04822B8093CB
:101AF0007E04F101E859F94E85919591A591B49133
:101B000081010C5B144FF80180839183A283B3831E
:101B1000F101EF51FC4F10821182128213828989E8
:101B20000E942B850E945386F801C080D180E280FC
:101B3000F380F101E351FC4FC082D182E282F38253
:101B40008CE0E7ECF1E0DE01119601900D928A95B0
:101B5000E1F7E1E0F0E0EC0FFD1FE20DF31D408046
:101B600051806280738020E030E0A901C301B2019E
:101B70000E94FCE18823D1F120E030E0A901C301FB
:101B8000B2010E9476EA87FF04C077FA709477F872
:101B9000709481010C5B144FA3019201C501B40143
:101BA0000E9462E29B01AC01C701B6010E94F2E80B
:101BB000F8016083718382839383F98960E070E820
:101BC0008BE395E4F23020F060E070E080E793E48E
:101BD00020E030E040E752E40E9476E96D877E879E
:101BE0008F87988BCE010D960E94618561960FB606
:101BF000F894DEBF0FBECDBFDF91CF911F910F9143
:101C0000FF90EF90DF90CF90BF90AF909F908F901C
